:1000000000200120F54E0200916C0200916C02006C
:10001000916C0200916C0200916C0200916C0200E4
:10002000916C0200916C0200916C0200916C0200D4
:0C003000916C0200916C020071F4000061
:10003C002DE9F04F99B0054680780224532800F240
:10004C00C785DFE810F054009900A800B800C8007C
:10005C00DA00EA000C011B01C5052A01380159011F
:10006C00C505C505C505C505C505C505C505C50534
:10007C00C505C505C505C505C505C505C505C50524
:10008C00C505C505C505650188019401A001AB0135
:10009C00BA01D401EB0107023A02C505C505C50535
:1000AC00C505C505C505600276028C02A202B80220
:1000BC00CD02DE020303C505C505C505C505C5058D
:1000CC00C50538034C036003C5056D037703950321
:1000DC009E03AA03B603C503CF03F2030F04340433
:1000EC003C044E045B0467048B0492049504EC1CE2
:1000FC00E97A2A7B002320461EF094F88DF818002C
:10010C0006AB65200021012222F0B2FADFF8180BB1
:10011C000078012800F25B85204629F0ACFC002811
:10012C0000F0558505460079012840F0508529F0EE
:10013C0035FA00274FF400018DF83F008DF8380098
:10014C00000ACDF83A108DF841708DF83E708DF89C
:10015C0040008DF839000EAE214606F10A0029F058
:10016C0008FD297815223346017069788770417033
:10017C004520FF2100F029BD29F0ADFC6979AA7951
:10018C000023002425F0FCF98DF838000EAB652017
:10019C00012100F053BC29F043FA29F0B9FB0146C8
:1001AC000EA8022229F043FC8DF8180006AB65203E
:1001BC00022100F043BC29F033FA29F0A9FB0146D7
:1001CC000EA8032229F033FC8DF8180006AB65202D
:1001DC00032100F033BC29F023FA29F099FBEA79CA
:1001EC0001460EA80023002427F058F88DF81800BB
:1001FC0006AB6520042100F021BC29F011FA29F08E
:10020C0087FB01460EA8052229F011FC8DF8180079
:10021C0006AB6520052100F011BC0020DFF8304A48
:10022C0029F0E0F8ADF85800681DA0478046E81D9D
:10023C00A04795F809B0824605F10A07BBF1100FEB
:10024C0000F2AE830EAC5E46002E00F0AC83384656
:10025C0029F0E0FC24F8020B013E0237F4E729F008
:10026C00DFF929F055FB01460EA8102229F0DFFB1F
:10027C008DF8180006AB65200721DFE329F0D0F9D3
:10028C0029F046FB01460EA8112229F0D0FB8DF86F
:10029C00180006AB65200821D0E329F01CFC6A7B12
:1002AC00691D0023002423F01FFE8DF838000EABCF
:1002BC0065200A21C2E302208DF8200029F00BFCF6
:1002CC00ADF81800681D29F0A5FCEA79064605F181
:1002DC0008018DF838200EAF781C28F053FF06A8C3
:1002EC0031463A460023002420F084FB8DF8580058
:1002FC0016AB65200B21A1E329F0EDFB00210024B6
:10030C0023F048F88DF838000EAB65200C2195E3EE
:10031C000020DFF83C4929F065F8ADF85800681D5D
:10032C00A047804695F80F9005F11000A04705F105
:10033C001304AD7C83460F2D00F247830EAE2F467F
:10034C00002F00F04583204629F064FC26F8020BB0
:10035C00013F0234F4E729F063F929F04AF828F058
:10036C0001FF40F0468306A829F003FC46E329F080
:10037C0057F929F03EF828F0F5FE40F04D8306A819
:10038C0029F0F7FB4DE329F0A6FB29F09EFA8DF836
:10039C0038000EAB6520232100F016BCDFF888185E
:1003AC00C8208DF81800E81C0978002900F081831A
:1003BC0028F065FB8DF81800A3E36879EE1CFE2885
:1003CC000BD1A879FF2808D12878082805D3304606
:1003DC0029F020FC314625F0FBFA0EA9304628F016
:1003EC0043F8002800F09183054600249FE3E81CA5
:1003FC00042126F08DF8E97929F02EFCDFF8441859
:10040C008DF83800022028F063FCDFF83C1803203C
:10041C0028F05EFC0EAB65202621D5E329F055FBB8
:10042C00044605F10E0029F0F5FB297C6A7C034695
:10043C00E878CDE90012AA1D214625F053FDDFF81E
:10044C0000188DF83800042028F042FC0EAB652013
:10045C002721B9E34FF00208E81C8DF8408029F001
:10046C00D9FBADF8380068798DF85800A81D29F033
:10047C00D1FB2E7A044600270935CDE9005716A882
:10048C000EA92246334621F0C7F829F0E7F810D11F
:10049C00DFF890078DF84080CDE9005722463346AF
:1004AC00C08AADF8380016A80EA921F0B5F88DF861
:1004BC00180006AB6520282186E30226E81C8DF87F
:1004CC00406029F0A7FB29F023FAED7904460EA829
:1004DC00002321462A4627F069FE29F0BFF80ED1E9
:1004EC00DFF840078DF8406021462A460023C08A79
:1004FC00ADF838000EA827F059FE8DF8180006ABA1
:10050C006520292160E329F08BF8ADF83800681DCF
:10051C00042125F0FDFF6A7AAB7A00240146009491
:10052C000EA825F00BFD8DF8180006AB65203021C8
:10053C0084E229F075F829F0CDF9312201238DF8E8
:10054C00580016A8CDE90004DFF8F0060EA921F03A
:10055C0063F88DF8180006AB652031216EE229F0A6
:10056C005FF829F0B7F9322201238DF8580016A84C
:10057C00CDE90004DFF8C4060EA921F04DF88DF882
:10058C00180006AB6520322158E229F049F829F011
:10059C00A1F9332201238DF8580016A8CDE90004E7
:1005AC00DFF898060EA921F037F88DF8180006AB85
:1005BC006520332142E229F033F8ADF83800687B2E
:1005CC000024691D0094C0F3400200F001030EA842
:1005DC0022F0C2FE8DF8180006AB652034212DE206
:1005EC0029F01EF86A7BADF83800691D0EA80023AF
:1005FC00002426F0F3F98DF8180006AB65203521A0
:10060C001CE22C4614F8030B04281ABFE8782C1DA6
:10061C0002208DF84000204629F0FCFADFF818661D
:10062C00A5780121E278ADF8380000230024317060
:10063C000EA829461EF066FE8DF818002846347068
:10064C0026F008FA06AB65203621F7E129F043FACB
:10065C00ADF83800687904218DF84000A81D25F00C
:10066C0057FF0446AE7AEF7A05F10C0029F0D2FA66
:10067C00DFF8B0850546214632463B4628F08FFE12
:10068C000EA820F0A5FF28F0E9FF10D1022021468A
:10069C0032463B468DF84000B8F81600ADF83800ED
:1006AC0028F07DFE0EA820F093FF8DF8180006AB05
:1006BC006520372188E26C7829F00DFA0146DFF8C5
:1006CC007405007820F070F98DF8380004F0E00023
:1006DC00202840F07C820EAB65203E2174E26C78C1
:1006EC0029F0F9F90146DFF84C05007821F07CFC83
:1006FC008DF8380004F0E000202840F068820EAB42
:10070C0065203F2160E200206C788DF83800DFF81E
:10071C0018050078411E022980F09481022095E191
:10072C0029F0D9F929F0D1F88DF838000EAB6520F5
:10073C00422149E2002006908DF83D00CDF83900A9
:10074C00E81C06A926F0BCFD8DF83800069850B1BF
:10075C0028F02CFE81788DF83B10C1788DF83C1078
:10076C0000798DF83D000EAB6520432106222CE26A
:10077C00E81C28F084F98DF838000EAB6520442174
:10078C0022E229F0A8F96979AA790DF0BBFF8DF85E
:10079C0038000EAB6520452116E229F09CF96979E9
:1007AC00AA791AF08FFC8DF838000EAB6520462123
:1007BC000AE2EC7829F089F90146204622F080FE05
:1007CC00B0FA80F0472140098DF838000EABC1E13A
:1007DC00E87800248DF8384023F0F6FB0EAB65204A
:1007EC0047212BE1E8780EA926F08EFD06468DF800
:1007FC00180040000130C5B2284629F00FFA002835
:10080C0000F0A381044600F8016B00219DF818202C
:10081C00914280F0BE809DF83830013100F8023BE7
:10082C009DF8393000F8013CF2E70EAC132120465C
:10083C0028F044FBEE7829F048F90146304626F0C2
:10084C0031F9002800F088810021231D8DF8381023
:10085C0028F0ACFDC11C827818468DF83B2028F09E
:10086C0091FC7CE10020EC78CDF84600CDF84200FC
:10087C00CDF83E00CDF83A0029F027F9AA79ADF869
:10088C0038000F2A28BF0F228DF83A2022B10EA86B
:10089C00E91D033028F076FC0EA9204601221CF03D
:1008AC00CBFF8DF8180006AB65204B218CE128F0AE
:1008BC0069FA8DF838000EAB65204C2184E1E8789C
:1008CC0029798DF838100EA9032800F05F810228D1
:1008DC0000F06281012840F06681522021F0C8FBB3
:1008EC0064E129F0F8F869790246A81D1BF054FA66
:1008FC008DF838000EAB65204E2165E129F0EBF840
:10090C000146687919F05AFF8DF838000EAB652056
:10091C004F2159E1C34D0822E88A05F13901ADF8A0
:10092C003800C24800788DF83A00A88CADF83B002E
:10093C00688BADF83D000EACE01D28F023FC04F1F3
:10094C000F0005F11C01082228F01CFC287E502108
:10095C00182223468DF84F00652036E1B248007806
:10096C00002800F0018112200AE120F07DFD2EE12B
:10097C0000208DF83800E878010606D5A94910F05A
:10098C007F0018BF012081F868000EAB6520532151
:10099C001AE1652049212A46234621F069FE39E1F6
:1009AC0080208DF863003E78102E52D80DF1180976
:1009BC00013734464D46002C4DD0384629F02AF9E3
:1009CC0025F8020B013C0237F5E780208DF8630017
:1009DC0027780F2F54D801340DF1180A3E46002EFB
:1009EC0050D0204629F016F92AF8020B013E0234A9
:1009FC00F5E7084629F00EF9ADF81800687E06A94F
:100A0C0028F0B8FB0EA921201BF018FB8DF858001C
:100A1C0016AB6520212111E0084629F0FBF8ADF852
:100A2C001800687E06A928F0A5FB0EA922201BF051
:100A3C0005FB8DF8580016AB65202221012221F010
:100A4C0017FEC5E0002840F0B580042008F002FE37
:100A5C00B3E080200DE0BBF1100F0CD80EA90020E4
:100A6C0052465B468DE84202039016A8414615F0AB
:100A7C0009FA8DF863000DF1630365200621A3E0EC
:100A8C0080200FE00F2D0FD80EA9002002974A46A8
:100A9C005B46CDE9005106A9CDE9031016A84146E5
:100AAC0015F098F98DF863000DF163036520202192
:100ABC008AE016A90EAD2A4618F076FD04469DF87C
:100ACC005800F0B1614904EB4400002641F8206065
:100ADC0001EB800046609DF94B00B0F1FF3F03DC59
:100AEC0005F1130022F07CFF0EAD1421284628F0EE
:100AFC00E5F90420214614222B4625F05BFC8DF8E9
:100B0C00186006AB652024215EE0182029F086F8D9
:100B1C00002800F083800446BDF83800002118221C
:100B2C00234628F0B1F90546002818BFC82519201E
:100B3C0029F074F8002867D007460130002D4BD0FF
:100B4C001821FF2228F0B4F950E0002049218DF83B
:100B5C00180006AB652037E001208DF838000EAB8D
:100B6C0065204A21132230E028F0B5FF044605F138
:100B7C000D0029F04FF80246691D204625F0F4F9C6
:100B8C008DF838000EAB652051211DE0522021F06C
:100B9C006FFA2748002104E0522021F069FA24481A
:100BAC000121017002E0522025F036FA0EAB6520CF
:100BBC004D2109E001208DF8380004F0E0002028D8
:100BCC0005D10EAB65204021012221F051FD0024FE
:100BDC00204619B0BDE8F08F3146082228F0D2FA31
:100BEC0007F109002146102228F0CCFA65202521B6
:100BFC0019223B463D7021F03BFD3846192128F067
:100C0C005DF9384629F008F8002CE0D02046182170
:100C1C0028F054F9204628F0FFFFD8E7C825FFF745
:100C2C00E4BB00BF407B002018260020C426002017
:100C3C00D527002096880020952700207C260020B0
:100C4C0059680200CD6D0200494E0100804300201E
:100C5C00219C02002DE9F04F99B080466FF00700FF
:100C6C00DFF8DCA80630ADF852009AF80000022834
:100C7C0014D1DFF8C808007880B9B8F8080010B1B2
:100C8C001020012101E0302000210AF03FFE00205D
:100C9C008DF81C0007A9522021F0EAF90DF11C096E
:100CAC0098F80810D8F804004A4610F001FAE8B198
:100CBC009DF81E609DF81F409DF82050BDF82670D1
:100CCC0028F066FC844211D127F003004FF6F8712E
:100CDC0080B288420AD0012D08D8022E06D29AF88A
:100CEC000000022808D19DF84D0028B1D32016F041
:100CFC000AF819B0BDE8F08FB8F82800ADF8480034
:100D0C00B8F83200ADF82A009DF82200D0B1D8F81E
:100D1C0004109DF81D209DF83830012027F0E4F9CF
:100D2C0008B1CF20E3E7DFF81C08C078012809D10F
:100D3C00B8F8280028F04BFE20B1417901F0E7010A
:100D4C00083141719DF8210068B1BDF82610FF20D3
:100D5C0025F0A8FE9DF82110E0B141F001012C26F0
:100D6C008DF8211017E09DF83900002800F0EB8079
:100D7C009DF83D10FF2902D0002940F02681DFF8B4
:100D8C00C807BDF82620C18A8A4240F0278101207D
:100D9C00222607E0082601F00300012808BF46F0D0
:100DAC00110601209AF800104FF6F877012908D89F
:100DBC003446B20758BF64F07F04002808BF34469D
:100DCC0000E034469DF82200DFF87C575FFA84FB84
:100DDC0030B9E87A20B10BF02200222840F0808054
:100DEC001BF0400004901CD0012903D8A87B80077D
:100DFC0000F1D880119801780C2900F2DB800122D7
:100E0C0041F298438A401A4200F0D480032902D15F
:100E1C0040780D2805D007A822F036F901283FF4B8
:100E2C0068AFA88CB8F8441081420AD198F84620D3
:100E3C00B8F84210B8F8280000230093002307F0FC
:100E4C00E5FC9DF82200F8B1B8F84210B8F828007B
:100E5C0022F0EAFB002800F08F800646D8F8040048
:100E6C009DF81D10F2780844417B8A421EBF002277
:100E7C007260F1700130042125F04AFB71688842E0
:100E8C00FFF437AF013070609AF80000022834D2BA
:100E9C00A87B80077FF52DAF9DF84D004FF6F876B7
:100EAC0060B1BDF8280027F06BFB002800F007812B
:100EBC00D8F80400417801F0DF0141709DF82E0054
:100ECC00002800F0DF80D8F80400817901398171A5
:100EDC008DF82E1004F07F00090640F0D680D3E088
:100EEC000BF0420042287FF41CAF1198007800F000
:100EFC00FE0006287FF415AF72E77FF4FAAE95F882
:100F0C002600092802D004287FF4F3AE5FEA8B6038
:100F1C0000F19E80049800283FF4EBAE11989DF8E8
:100F2C0038100078042808BF022900F045810728F2
:100F3C0008BF042900F009810C2840F04D8107A856
:100F4C0015F0AEFAD5E6BDF8260022F00DFE0238FB
:100F5C00DFF8F415B0FA80F0CA8A4109BDF8260012
:100F6C00904208BF023100293FD09DF81E20002A74
:100F7C0056D001F1400455E09DF84D00B8B3042063
:100F8C0026F06CF800283FF4B4AE01464FF4B27072
:100F9C000880B8F828004880DFF8B00500781EF00B
:100FAC007DF8A6E611980178A1F10C0212F10C0F54
:100FBC003FF62CAFE88ABDF8262082427FF496AE2D
:100FCC00BDF8280024F02CF990E6109A9DF83C000E
:100FDC0020F060FF30B101200026E3E690F82600F7
:100FEC000428F8D100260020DCE600241AE095F84D
:100FFC006C0001287FF448AF11980078062803D1C3
:10100C00049800287FF440AFF81DBDF82A1080B278
:10101C0081423FF46EAE07A841461EF0FFFA68E627
:10102C0001F1200422F0A0FD0138B0FA80F0400953
:10103C0044EA00069DF81E0000283FF4B2AE119859
:10104C00007827F0F1FA012818BF04F07E06A8E614
:10105C0098F8460028F080F99DF82E00012840F001
:10106C00B480B8F82800BDF82810814240F0AD805B
:10107C00BDF8260022F078FD022804BF00208DF870
:10108C002E00A2E004F07F000446210702D44FF0AA
:10109C00000A34E0E1B24A0722D4C9069DF82110B7
:1010AC0028D5C1F3820212B1072A18BF013A002ACF
:1010BC0008BF044601F0E30040EA820118E0D320A7
:1010CC0015F021FEDFF888040078002800F09F80DE
:1010DC00DFF8801451F82000C0EB0010810098E07C
:1010EC009DF8210000F0E00100F0E30040EAD1019E
:1010FC008DF82110D8F804004FF4805A017295F83D
:10110C002600092801D0042823D1E98ABDF826003D
:10111C0088420AD022F028FD022806D09DF8210032
:10112C0000F0030001287FF4E4AD9DF81E000028B8
:10113C0047D011989DF838100078042808BF022970
:10114C003AD0072848D1042946D107A817F040FF08
:10115C00CFE5E7B214F0610F46D0F80709D0B8F824
:10116C00281007A8A94615F0E3FB002864D004F06A
:10117C009F040025E7B2A00609D598F84600D8F8D8
:10118C003C2028F0E9F807A815A905F04DFC7806D5
:10119C0040F12681B8F8281007A80DF152022B4611
:1011AC0010F002F800286FD005461198007801283D
:1011BC0008BF4AF0100A13E107A9002010F068FFDD
:1011CC0097E598F8460028F0C7F8D8F83C2007A80F
:1011DC0015A905F029FC8CE503287FF48AAD07A836
:1011EC0000210FF0EFFC84E59DF81E0001285AD178
:1011FC0011980078032849D0052854D1B8F8281044
:10120C0007A80DF1520200230FF0CEFF71E5D14873
:10121C000168D1480268BDF82800904701287FF486
:10122C0068ADCE480168BDF828008847CC480168F5
:10123C00BDF8280088475CE526F0E4FA9DF82E10EE
:10124C000546BDF8280019B9B8F82810884291D085
:10125C00B9F81610814204D1BA48807800283FF4BE
:10126C0089AFB8F8281007A82A4609F027FA0028F1
:10127C0000F09B8038074AF0040ABDF8260048BFEE
:10128C00F01DADF8520075E70025A9E0BDF8260069
:10129C0027F076F938B1B8F8281007A80DF15202EA
:1012AC0000230FF081FF9DF82E0088B323F066FD1C
:1012BC0000287FF41EAD9DF83900A0B3109A9DF85C
:1012CC003C009DF83D1020F0E5FD002870D09DF805
:1012DC003D00002875D0109928F042FB9DF8243071
:1012EC00ADF8520011209DF823209DF821104AF0F2
:1012FC00400A002B08BF0920002A18BF083000291B
:10130C0018BF0130D8F804100A5C013A0A5462E0A4
:10131C009DF81E0001287FF47EAE119800780328FA
:10132C003FF4E7AC77E69DF82010BDF826000029C5
:10133C00ADF8520000F0D3804020BDF8261009F122
:10134C001D0200EAC4059DF820002B4618F0C2FDD2
:10135C0038B1D8F804004AF0200A017801F03F01B6
:10136C0001709DF8390048B1BDF8261009F1200034
:10137C0021F06CFE4AF0400AADF852009DF81E00B8
:10138C00012806D0BDF82810BDF82600002214F064
:10139C0085FFBDF82810BDF826002A4612F0BEFBCA
:1013AC00002818BF4AF0200A15E004F0DF04E0E63C
:1013BC00BDF82610BDF828000B2200231AF07AFC89
:1013CC0097E4BDF82600ADF8520028F000FB002889
:1013DC0008BF4AF0400A26F015FA05464FF6F87693
:1013EC00B01DBDF8521080B20F1A5E4818BF2F46C0
:1013FC000078012805D1F01DB8F8321080B2814276
:10140C002FD160B2B0F1FF3F3FF773AC002F3FF428
:10141C0070ACB8F8080028F001FC00283FF469AC67
:10142C00B8F80820D8F80410054627F0ABFE9DF854
:10143C001E10002098F80830B8F8282016908DF867
:10144C005410BDF8521015ACCDE9007ACDE9020468
:10145C00284610F0DDFB70B3284628F0DDFBFFF7C3
:10146C0048BCB8F828108142CBD0701CBDF826209F
:10147C0080B28242C5D2BDF828008142C1D028F08A
:10148C00A6FA0028BDD0017901390129B9D84088C4
:10149C0001218DF85410ADF8600015AD28461EF0F2
:1014AC002DFD0028ADD0281D1DF0F0FC0028A8D083
:1014BC0021F0DAFEA5E72348407800283FF419AC68
:1014CC0000208DF81870ADF81900DDF826004FEAF1
:1014DC003040059005A827F0CDFCFFF70ABC390772
:1014EC003FF52AAF9DF81E1001293FF425AF0021CE
:1014FC0018F0B0FC20B1407901380228FFF41CAF81
:10150C00B8F84410BDF8520022F08EF830B1807853
:10151C0026F0B8FB01380728FFF40EAFBDF8280001
:10152C0027F02EF818B104208DF8200004E7BDF840
:10153C002610BDF8280002223FE700BFD527002067
:10154C0018260020E8250020407B002098880020E9
:10155C00C727002060B70200942300209C230020A2
:10156C0098230020D32700202DE9F0438DB00546A9
:10157C0080780224252800F27380DFE810F0260022
:10158C00A400C400D700EA00F8000601B602B602B7
:10159C001D012E01B602B602B602B602B602460113
:1015AC004B01B602B602540158016101B602B602F3
:1015BC00B602B602B602B602B602B602B6026B01AB
:1015CC006E017101740178017F01DFF8D47500247C
:1015DC000E258DF804403878012807D801A81DF095
:1015EC00EDF804469DF8040005EB4005EEB23046DC
:1015FC0028F014FB002800F087824FF00008054605
:10160C00431C0021082280F80080012027F03CFCBC
:10161C0027F0C4FF6872000A0721A872DFF884055E
:10162C00E972007828733878012800F262829DF8FC
:10163C000420002A6A7300F05E8205F10E0000217E
:10164C002346914280F0578213F8022B013100F8A7
:10165C00022B13F8012C00F8012C9DF80420F0E764
:10166C00A0F140010D291FD8DFE811F00E00100188
:10167C003F023F021E012E013F023F023A0145018B
:10168C00500165013F02740101ACE91C0822201DC8
:10169C0027F078FD204619F0E1FFBDF80600402147
:1016AC00ADF828000AABEEE0632800F069816428ED
:1016BC0000F07681E02840F0188200244720E021D9
:1016CC00002200230FE2202028F0A8FA002800F0C6
:1016DC00C1812021FF22044627F0EAFB631C012074
:1016EC000021082227F0D0FB0546002818BF012551
:1016FC0001AB84200021042227F0C6FB002800F057
:10170C000582023506E2E81C28F084FAADF80400E4
:10171C00832028F09CF9014601AA832028F070F858
:10172C008DF828000AAB6720022190E1E81C042107
:10173C0024F0EEFE0190842028F089F9014601AADC
:10174C00842028F05DF88DF828000AAB672003216F
:10175C007DE1612028F07BF90146EA1C612028F02C
:10176C004FF88DF8040001AB672004216FE1622073
:10177C0028F06DF90146EA1C622028F041F88DF83A
:10178C00040001AB6720052161E100208DF8040005
:10179C00E81C28F03FFA6A7900F4F851002A00F0AE
:1017AC004981B1F5A06F04D04FF6FF71884240F02B
:1017BC004B814FF0FF3045E128F002FA044628F047
:1017CC00FDF9D949604301ACB0FBF1F1204628F09A
:1017DC008EF9672009210422ABE0DFF8B4632D7980
:1017EC00306840B901AC204627F09AFD0120214613
:1017FC000EF028FA3060052D00F06981002D00F004
:10180C006981642122F040F966E115F8032B672009
:10181C0010216EE0E87823F093FD8DF8040001AB05
:10182C006720112113E100246720142102E0002419
:10183C0067201521ADF80840019401AB062252E156
:10184C0000246720162109228DF80C40CDE90144B3
:10185C0001AB48E1F52020210BE0F520212108E027
:10186C00F520222105E04FF6F570232108E0F52044
:10187C0024218DF8040001AB6720E8E0F520252138
:10188C00ADF8040001AB67200222E1E0E81C28F06F
:10189C00C1F9ADF8060001AC204617F055FB231D2D
:1018AC00672041210822D3E0E81C0AA926F0DCFDC0
:1018BC0000288DF8040000F0CF8001A81821FF2229
:1018CC00013027F0F5FAF4E0E81C0AA926F0CCFD6B
:1018DC0000288DF8040000F0F1804FF0FF30EFE0AD
:1018EC0015F8030F697822F0B3F828806720482197
:1018FC0002222B46ACE0E87824F058FF01AC0146FC
:10190C00204618F0E7FC6720492111E0EC1C20462A
:10191C0026F066FA002818BF2046B5F80B1019F00F
:10192C00F1F901AC0146204618F0D4FC67204A219D
:10193C00242223468CE001ACE91C0822204627F027
:10194C0021FC204627F0D8F98DF828000AAB672037
:10195C004B217CE04FF0FF3095F80380691D01901E
:10196C00ADF81000CDE90200FE208DF806002879B4
:10197C0003288DF8300020D10AA828F0FAF821E0CD
:10198C000024E91C08228DF8284001AD284627F0D8
:10199C00F9FB28461DF07AFA0AAB67206321A1E017
:1019AC00B5F80B006A7B0024E91C8DF804400AF0A2
:1019BC0067F801AB6720642194E0084628F02AF907
:1019CC00ADF82800AF7B002F00F0DD807E0095F88D
:1019DC000D90304628F022F9002800F0D48005F153
:1019EC000F013246044627F0CDFB00940AA940466D
:1019FC004A463B460DF0F8F9002800F0BA8083788F
:101A0C0001784278057946798DF806308DF8041006
:101A1C008DF80520C3788DF809608DF808508DF885
:101A2C00073001A98B1D811D40794200184627F013
:101A3C00A9FBA5E0B1F5A06F03D04FF6FF7188426A
:101A4C0002D100205549086001AB67200621012214
:101A5C0020F00EFE002448E0182028F0DFF840B3F8
:101A6C00BDF828100446009006200022182324F00C
:101A7C008BFCB8B9BDF8285001AE21461022701C61
:101A8C0027F080FB444F05EB450506F1110057F894
:101A9C00251028F02CF807EB8500416806F115009D
:101AAC0028F025F82046182127F008FA204628F0BF
:101ABC00B3F801AB672044211922C9E7BDF828000F
:101ACC00ADF8050001AB672045210322C0E7314981
:101ADC0001220A7021F08BF9002467200A218DF86D
:101AEC00044001AB012220F0C3FD20460DB0BDE83F
:101AFC00F08385F80D806720002132462B4620F0BC
:101B0C00B7FD284628F088F87CBBA3E7019800BAFB
:101B1C00C4F809000AAB83200021022227F0B4F993
:101B2C0020B1043506E000BF40420F00BDF828008C
:101B3C00A4F80D0004F10F0361200021012227F00D
:101B4C00A3F9002818BF083504F110036220002106
:101B5C00102227F099F9002818BF1035234625705C
:101B6C0067200121202220F083FD204628F054F824
:101B7C0070E74FF6FF70ADF808006FF480300190FD
:101B8C00204628F049F801AB67204D210E225FE773
:101B9C00248800209227002018830020048800202D
:101BAC0018260020C42600202DE9F04F85B084783B
:101BBC000226362C00F2BE820546DFE814F06C01DA
:101BCC00740172007C017800BB02BB0281003700FB
:101BDC004C008C009F00AD00BB02B5009001BB0215
:101BEC00BB029A01AD01BB01BB02BB02BB02BB0233
:101BFC00BB02BB02BB0237004C00BB02BB02BB02E8
:101C0C00BB02BB02BB02BB02BB02BB02BB02BB02E0
:101C1C00BB02BB02BB02BB02BB02BB02BB02BD00D0
:101C2C00EB00CB01FF005B005B00DB0127F047FF03
:101C3C00242840F0AA8102AB352000210422002484
:101C4C0027F022F9002800F0FC81012002228DF8F7
:101C5C0010000020FCE100208DF8100027F02FFF71
:101C6C000646092C40F0ED8095F8059095F8068015
:101C7C000720EFE0DFF82465306880B1406A70B16E
:101C8C0002A927F025FF0546342C40F02C8228466B
:101C9C0027F0C0FF002800F02582042041E2032039
:101CAC003FE2DFF80835612002210A223FE202AC54
:101CBC00E220214624F0B0F961200421082288E1B9
:101CCC0027F0FDFE0446681D27F0A4FF242C40F0ED
:101CDC0087810020FBE1E878032800F29781281D1A
:101CEC0027F098FF0246E878DFF8B81431F81010A6
:101CFC00DFF8B404007827F0F7FE88E1E8780328D1
:101D0C0000F28981DFF89C1431F81010DFF8980488
:101D1C0000781CF067FE7FE127F018FEADF8080094
:101D2C0002AB61200C2103E1002661200E2101226F
:101D3C008DF8086002AB1BE2DFF8606401208DF8BF
:101D4C0010003068002800F02C810069002800F099
:101D5C00288102A927F0BCFE042124F0D9FB00281D
:101D6C0000F0EC81044627F059FF002800F01C819C
:101D7C002146054627F0A2F83068BDF80C10224623
:101D8C002B4606690298B0478DF81000284627F0BC
:101D9C0043FF09E1DFF804442068002800F00881C3
:101DAC008069002800F0048102A927F091FE2068C8
:101DBC00BDF80C10826902989047FAE0DFF8DC73EA
:101DCC003868002800F0FB80C069002800F0F7801C
:101DDC0002A927F07DFE9DF80850BDF80AB0BDF8A9
:101DEC000C90044627F016FFA6788046F72E28BFE5
:101DFC006FF00806B01C5FFA80FA504627F00EFF11
:101E0C00002800F09D81012D044608BFBBF1000F96
:101E1C0000F09A813868A11CF3B24246C569029859
:101E2C0000914946A8470746002840F093810027B7
:101E3C0061203321524623466670277020F018FC2F
:101E4C0088E1681D27F0E6FE8146E81D27F0E2FEDA
:101E5C008046092002AF242E18BF2F1808BF352644
:101E6C00304609EB080527F0F2FD854201D9022026
:101E7C0057E1B9F1000F04D1304641463A4622F001
:101E8C0047FA304641463A4627F0BAFC002800F0A3
:101E9C00E5800A2045E1E878012802D0002840F0CE
:101EAC00488127F0D7F940F259600121ADF80800BC
:101EBC0002AB61203CE00120EC1C8DF80800E22014
:101ECC00214620F0D5F830B901200821224627F010
:101EDC0097FC8DF8080002AB6120032126E1E8781D
:101EEC00291D012800F0E180002840F0E580E02069
:101EFC00DFE027F0E4FD0446681D27F08BFE242C60
:101F0C000FBF00200146204627F052FD8DF8080037
:101F1C0002AB6120122109E127F0D1FD24280CBF6E
:101F2C00002027F094FDADF8080002AB61201321CE
:101F3C000222FCE0E8788DF8080099488068D0F817
:101F4C00302402A9E02090478DF8100004AB6120EA
:101F5C001421EBE0914C206898B3806A88B302A9F5
:101F6C0027F0B6FD2068BDF80C10826A02989047E5
:101F7C00014627E0894C206868B3C06858B327F045
:101F8C009EFD2168C968884726E08046693800268E
:101F9C0080B2032838BF0126681D082C40D1057873
:101FAC0041E003208DF8100004AB61203021BDE02E
:101FBC0003208DF8100004AB61203121B6E003271B
:101FCC00CDE0002102AC204627F091FD61203221AA
:101FDC0004222346ABE0032027F095FC3621A5E034
:101FEC0005F10806ED790146A8426CD9204600227D
:101FFC0027F000FC09288DF808006AD1002D68D064
:10200C0020462946324627F0FBFB62E0022027F0EF
:10201C007AFC0A218AE0022027F075FC0B2185E06E
:10202C0027F0F8FD0546404627F011FD0227A8428F
:10203C0088BF7700CFB100268DF80870612021464B
:10204C0092E002988DF810400422ADF812000220A4
:10205C008DF8110004AB6120082168E0012E62D1DB
:10206C00E220394620F004F85BE0471BB8B2F728B1
:10207C0028BFF727B81CC6B2304627F0CFFD002882
:10208C0060D01FFA87FB00F1020982464846594688
:10209C0026F014FF404629465A464B4626F0F4FEDD
:1020AC000546002867D00A2770E00878022814D269
:1020BC0052201FF0DDFF00E002208DF8080002AB7B
:1020CC0061200F2132E02046324627F093FB8DF839
:1020DC00080002AB6120072128E002A9522023F05E
:1020EC009BFFECE702359DF8080015F8018BBDF855
:1020FC000C7001280ED1BDF80A0058B9384641467B
:10210C002A4622F005F9012F04D1E22029461FF0BE
:10211C00AFFF01273068394642462B46466A029883
:10212C00B0478DF8100004AB61202146012220F04D
:10213C009FFA0026304605B0BDE8F08F052031E748
:10214C0010270CE0102776E7A9F169000328BFF4EB
:10215C0061AE0227204627F05FFD002FE9D0002654
:10216C008DF80870612033218DF8096002AB0222D2
:10217C0020F07EFADEE78AF8017000276120214604
:10218C00324653468AF8007020F072FA504627F017
:10219C0043FD002D7FF44FAFCBE700BF5C27002041
:1021AC000C01002064BC02009688002000BC0200D8
:1021BC002DE9F04F8FB00C4648070FD4200441D4C2
:1021CC00E00400F19781200600F1C081A00700F126
:1021DC00D481200500F1F3810020B4E1DFF8200563
:1021EC000178062900F2AD81DFE811F007009401B7
:1021FC00AB01AB019901AB01A001DFF81055DFF881
:10220C0004152A7891F82B30022A02D19E0600F18F
:10221C0098815E0700F19D819B0740F19281042318
:10222C00037091F82C30DB0700F08B8191F82E3085
:10223C00002B00F0528225F03CFE0420012102F01C
:10224C00A3FA57E2DFF8C8040394DFF8BCB4DFF854
:10225C00B094DFF8C474DFF8AC44DFF8B054DFF8A6
:10226C00BCA448F20208008802909BF800001CF005
:10227C00E7FB002800F03A8106460078D3282DD1E0
:10228C00F089404540F019813878002800F015811C
:10229C0099F80000012840F0108126F0BBFE0028C0
:1022AC0040F00B817088002840F00781A24604ACF6
:1022BC001221204626F002FE27F0ACF930462146CA
:1022CC0018F02EFCBDF81C00B0F5285FC0F088801B
:1022DC00012002211FF078FA54462AE099F80010E8
:1022EC00884217D1012834D0032840F0E6802878A2
:1022FC000138012800F2E180B078012851D0002883
:10230C0040F0DB807078002800F0BF8000201DF0CA
:10231C000DFFD2E00A2811D194F82B00BA46B71C55
:10232C003071A16909B138468847384625F03AFA28
:10233C005746DFF8D853DFF8E4A3BEE0297800292C
:10234C0040F0BB80092840F0B880A168B01C8847D9
:10235C00B3E028780138012800F2AF80707860B1C2
:10236C0094F8330094F83410013084F83300C0B280
:10237C00884202D9012000219DE099F80100032830
:10238C0058D0022871D0012840F097803878002866
:10239C0000F08C8026F03EFE002800F09280012098
:1023AC0085E07078002875D027F0F8F84FF6FE71AC
:1023BC00884203D1BAF81600884207D0AAF8161042
:1023CC00ADF8281053200AA91FF052FE1EF04CFD48
:1023DC0025F048FA00208AF826001DF0C5FB6CE0B9
:1023EC00CF48006809A90AAA17F0DEF80746029838
:1023FC005446C64DDFF824A3874212D29DF838000C
:10240C0010B1FD208DF838000420394614220AAB97
:10241C0023F0D0FFC34907EB470001EB80000121FB
:10242C0041720020012184F83200012002F0ACF945
:10243C00B94F42E0A2460AACAB20002122461CF068
:10244C00F9FC042004945446DFF8D0A2AF4D8DF86B
:10245C00140004A80FF038FD27F0DCF89BF80000FE
:10246C004FF4805141F288321DE0012020714FF46D
:10247C008060ADF828000AA819F0B6F827F0CAF861
:10248C00A4484FF4805102680BE010F0C1FB606966
:10249C0098B9A2E702204FF4805140F6B83289F87F
:1024AC0002009BF8000027F01FFB06E0002084F8D8
:1024BC0032000120012102F067F9304625F0CCFCF6
:1024CC00D3E694F8350020B1E0690028F5D08047B8
:1024DC00F3E70020002102220023ADF8280002209F
:1024EC008DF830000AA825F061FEB5E7039880F45A
:1024FC00004028E0854800780138012859D88048E8
:10250C00017803294DD0012953D1417800201FF0C7
:10251C005BF94EE0012001211FF056F911E025F086
:10252C00C8FC0420012102F02FF90AE0002132221C
:10253C000170744880F82A1073480421007827F041
:10254C00D3FA84F004000FB0BDE8F08F84F0800063
:10255C00F9E70522027091F82C2092072CD591F8FE
:10256C002E204ABB052202600120487000201CF07E
:10257C004DFB022024F0DAFEE3E7644800780138D2
:10258C0001280BD80020CDE90A000AA812F00EFD94
:10259C0020B15D48022100781BF054FD84F002004C
:1025AC00D1E78178022904D10121817000201FF02C
:1025BC00E7F884F48050C6E705200021B3E75348C0
:1025CC000078002840F08680DFF838A1DAF80C504B
:1025DC00002D79D004A80DF1280B01300BF1040665
:1025EC000390002D6DD0A87A18B10138A87200069E
:1025FC0046D19AF83180B8F1000F11D00020A91CF7
:10260C0008228DF82800304626F0BCFD584619F0FB
:10261C0025F828B12A88BDF82A00314623F0A4FCFD
:10262C00AF1C0DF127015A46384616F0BDFF814606
:10263C00384609A923F0E3F9B8F1000F05D09DF84D
:10264C00380040F0020002281CD1DAF80800A0B1D2
:10265C0003983946082226F095FD022000220C230F
:10266C008DF81000BDF82400ADF81A00264800784B
:10267C0004A90091092120F0F8FB28461EF052FA1B
:10268C00ED68AEE7384623F097FF9DF82700012848
:10269C00DBD15846142126F011FC224A09EB4900E3
:1026AC0000215B4642F8201002EB800014224160AE
:1026BC004172FF2049468DF83800042023F07AFE41
:1026CC00C3E7DAF80C0028B90F484FF40061007822
:1026DC001CF088F984F4006035E7013A012A09D826
:1026EC00032202600120487001201CF08FFA0120A7
:1026FC0024F01CFE287800287FF423AF04205CE72C
:10270C0008880020AC2200209F880020182600207A
:10271C00C6BC020064270020AA270020407B0020B2
:10272C00DC870020804300202DE9F04F9DB004464B
:10273C00DFF84005406818B18047002800F0798226
:10274C00DFF834A5DFF834B50D940DF138099AF89B
:10275C000000411E002C0B9118BF01218BF80F10AB
:10276C009BF802800BF118049BF801100027002540
:10277C000C91C0B287421ED2B84517D0FEB20021D0
:10278C004A460423304626F0C5FC0E9810F4403F10
:10279C0040F0040018BF0135C0B27C2806D1304689
:1027AC000621F82225F030FCF82020709AF8000061
:1027BC000C340137DDE7E9B201380022884204D13C
:1027CC009BF80500002800F05182CDF82880DDF838
:1027DC0034804FF001094046B8F1000F08BF1020BB
:1027EC00059015AD00200190DDE90B74002638042E
:1027FC0000F0F9819BF80F0008B98BF80F90E0B24C
:10280C0000210EAA042326F085FC0E98B8F1000FC7
:10281C0018D010F4403F18D04FF400509AF8001024
:10282C000136013FABF810009BF80F0001388BF814
:10283C000F0059FA84F0B0FBF1F202FB11048BF893
:10284C000D40D4E70021049102E0CDE90B7404960D
:10285C00C0B20A9E4FF00009702804D00C98702169
:10286C00C0B221F0FDFEF4B200210EAA04232046D2
:10287C0026F050FC9DF83800FE2803D02046FE219F
:10288C0021F0EEFE20460621FE2225F0BDFB4FF482
:10289C0000500C9F0BF116010022ABF814908BF832
:1028AC000C60A146ABF81000FF208BF80E00F8B2BC
:1028BC008BF80D70400050FA87F001EB8000B0F8F7
:1028CC0006A0DFF8B00302706000ABF812A050FA5B
:1028DC0086F09BF80F6001EB8002FE20114601F898
:1028EC00020F32F8060F03910890E3480292047825
:1028FC0014A821F0A9F956FA87F0CDF824900138E4
:10290C0090FBF4F101FB140000905FFA87FB0C972D
:10291C00CB4500F06081ABEB0900B0FA80F04009C8
:10292C0007900020069000204FF00109C00740F0EE
:10293C009D801FFA8AF4162C71D9CE480078002895
:10294C0040F07181AAF1070758460FAAB9B216F0E8
:10295C00AFFEBDF84A6006F11000A0420FD89DF8FA
:10296C00460096280BD1A7EB06099DF84520314669
:10297C005B461FFA89F840461AF0CAF918B3AAF157
:10298C00010A4FF001095446A0B2172864D3362827
:10299C00A4F1160658462A4688BF2026A41BB3B2BB
:1029AC00A1B226F0B7FB3004EED015FA86F010F881
:1029BC00010C962801D0013EF5E7DDF8348006EBDA
:1029CC00040A0020B2E79DF84700C10701D1800737
:1029DC0004D40020CA46DDF83480A5E7F01D83B28C
:1029EC00089813FA80F4B4F5005F01D90120F2E7DE
:1029FC0080B2A54918440A1A5846414626F08AFB6B
:102A0C0006980130B4F5005F069004D101204FF414
:102A1C0000510891DEE70020CA460894DBE70698CF
:102A2C0010B1964926F0D0FC0098C0B2834500F056
:102A3C00D88091490C98097859FA80F0DDF82490E7
:102A4C00B0FBF1F202FB11078C4907EB470001EBDD
:102A5C008000B0F81CA058E78948149900684268B7
:102A6C00884890470020DDF8348005E0069810B1C6
:102A7C00824926F0A9FC002007900C980A907D480A
:102A8C000078002840F0CF8008981021C0F5005243
:102A9C00103883B20998C1F2001221F0F1F8754A8E
:102AAC00117808431499107075480068426875488D
:102ABC00904707980A9A88B16F4800780BEB000191
:102ACC00013991FBF0F202FB10126C49D0B24000BC
:102ADC0050FA82F001EB8000B0F81CA0DFF89CB13A
:102AEC0008990298099C01238BF80E200180ABF801
:102AFC001010BBF912209BF80D102046ABF814A057
:102B0C0023F040F9BBF914209BF80E102046022349
:102B1C0023F038F9BBF81000049CB8F1000FC0F595
:102B2C00005007D00599DFF850A18842A4BF0121BD
:102B3C00019101E0DFF840A1059988424FF07C013A
:102B4C00B8BF7821099E304621F08AFD0DF01EFB9E
:102B5C0007469BF80F000621FC22C01B8BF80F00C8
:102B6C00304625F051FA0399FC209BF80E30087082
:102B7C009BF8021017FA84F00C9301449AF80000A9
:102B8C00B1FBF0F202FB10118BF802100A9101312B
:102B9C00CAB2B2FBF0F202FB10118BF8011003EB7E
:102BAC0043010BEB8101898B102906D10C99013162
:102BBC00B1FBF0F202FB10100C900B98C01BB8F19B
:102BCC00000F0B903FF410AE019880F00100C0078D
:102BDC007FF40AAE07E00120CB464FF001090790C5
:102BEC004DE700984AE77C2021F054FD0446FF286D
:102BFC0025D17E2021F04EFD0446FF281FD19BF8E5
:102C0C00014004EB44000BEB8000807DFF2812D0C8
:102C1C009AF800009BF802100144013991FBF0F284
:102C2C0002FB10140BE01648149900684268154812
:102C3C00904700221AE020467E2121F011FDE0B2DF
:102C4C00FE218BF80340400050FA84F00BEB80001F
:102C5C00808BABF806009BF8020021F001FD0020F0
:102C6C008BF80500BBF81000C0F5005210B21DB077
:102C7C00BDE8F08FA023002097880020A0800020C2
:102C8C00D801001000400340002000112DE9F04F46
:102C9C0089B021F05DFADFF810158122DFF8148578
:102CAC00DFF814A5DFF82045DFF814E50A70DFF82B
:102CBC00FC140860DFF8F804FF2101700020DFF835
:102CCC000415A8F800008AF80000DFF8F004096881
:102CDC00007891F808B04FF6FE718EF80000594458
:102CEC008AB2A168D1F80031DB899A4200F267817F
:102CFC000422DFF8DC54A8F80020DFF8D024126896
:102D0C009668330ECEF80C60C6F301592B706FF039
:102D1C00FF0303EA1627B3B2D1F8B86047EA1327CA
:102D2C00AEF8047036781EB9B9F1020F00F0478185
:102D3C00B9F1030F00F043811B0A03F0070316B12E
:102D4C00002B00F03C81DFF88CC4042B9CF800C0F5
:102D5C0008BFBCF1000F00F032813EB1DFF878649F
:102D6C003678862E02D1022B40F02981BB0416D472
:102D7C00BBB203F00703022B08BFBCF1000F20D03D
:102D8C00DFF854140978862909D10020764621F001
:102D9C0017FADFF84004B64690F800C030780028E7
:102DAC004ED0BCF1000F4BD1012800F00881032854
:102DBC003FD0022844D1BEF80400400740F0FF8009
:102DCC003EE0D1F8D40090F88300022800F0808017
:102DDC0027460520147BF246A946A8F8000026F0E9
:102DEC00A7FB0546DFF8F003007886286DD1B8689C
:102DFC00016C096811B9D0F84C05804760B200210C
:102E0C00002626F04FFFB9680A6C12685077086CE0
:102E1C0000688677086C0068C477284626F034FE74
:102E2C00BAF8041099F8000001F010011CF0F0FE43
:102E3C004EE0BEF8040000F00700032840F0BF800D
:102E4C00BEF80400010700F1BA80810402D48105A8
:102E5C0000F1B5809EF80E20C2F38107012F00F01F
:102E6C00AE809609012E00F0AA80B9F1010F11D89D
:102E7C0040F0020101F0070103290BD117B93F2AD9
:102E8C0040F29D8037B9A168D1F8AC1009780029BF
:102E9C0000F095804FF6FB71B9F1020F0BEB010CB2
:102EAC0019D1CF4BD95D9B5D03EB01090023402A5F
:102EBC00B7FA87F238BF012352091A40430616D4D9
:102ECC00002A08BF09F1020915E0284626F0DCFDAE
:102EDC0025F04CFA75E0C14B402AD95D9B5D03EBA4
:102EEC00010908D3420648BFA9F1020903E0002AF0
:102EFC0018BF4FF00209C0F300205FFA89F11FFAE6
:102F0C008CF30A1A8EF801009A4258DC6044039143
:102F1C00B346401AA168AEF806007430D1F85012CE
:102F2C0080B28847A6490028886048D07421CDE932
:102F3C00019725F0C3FFA24F0020B870A548007878
:102F4C0020B9387900F020008AF8000078789AF8D7
:102F5C000010DFF878C24FF000092E4600299A497C
:102F6C003DD000284FF000003AD1B88800F007009F
:102F7C00032807D0012832D18868D0F8D40090F803
:102F8C00820060B3C8684069007818B125F028FE4B
:102F9C00FE280DD08C488068D0F84C02804738B998
:102FAC0089488068D0F844028047002800F0F780F8
:102FBC00834F0120B870DFF814C22E4610E025F0C4
:102FCC0077FC26F0B5FA814900240A6813681C7155
:102FDC0012680A6026F058FD09B0BDE8F08F002099
:102FEC00BC6804F1740184F830B06160A165797833
:102FFC00BB88FA880029A381029B228184F83A308D
:10300C00337808BF994697F80EB084F84990019D23
:10301C00A4F85C20FF22B8F80030A273CBF301199E
:10302C005E1A797BA8F8006001F0780160F38201E8
:10303C0001EB09002074280600F0AE80DCF80000DB
:10304C0004AF039A10FA86F000F10801384626F016
:10305C0051FE56FA85F0CBF38105A8F80000207CD0
:10306C0000F04008CDB3B9F1020F06D1B8F1000F52
:10307C0003D0B4F8440004AF06E0BDF810000237EA
:10308C00A4F84400A4F84200564EF189884203D0BB
:10309C004FF6FF7188425ED1032D11D104F132003D
:1030AC00394626F066FD464CF11CA068323024F0FF
:1030BC00F6FA454900284ED094F80EB008370EE0C9
:1030CC0037F8020BB1898842608606D04FF6FF7143
:1030DC003B4C88423C493ED101E03B49384CBBF16A
:1030EC00400F20D3B9F1020F06D16DB9B8F1000F22
:1030FC000AD13348806803E0A068017C490603D4F8
:10310C0039880237A0F84210BBF1C00F06D32C4C03
:10311C003946A068283026F02CFD03E0284C38886E
:10312C00A168088528498968A088D1F8AC20127854
:10313C00B2B1B9F1020F13D200F00700012802D08E
:10314C0003282FD11E4C6DB9264AA368D289B3F837
:10315C004230934206D018F058FE19F04FF830E781
:10316C0000F00700032806D0012815D1D1F8D400AF
:10317C0090F8820080B1A068D1F848128847104AB4
:10318C0050B90020D17B9070907BC1F3011100F0FD
:10319C00780008449168087408F042FA11E7084F67
:1031AC00B87808E7064CDDE7AC88002034880020AE
:1031BC00B1880020A6860020AF880020AE880020B1
:1031CC0024250020748800200C010020C0870020DA
:1031DC00BF880020BE880020B488002058BC0200A4
:1031EC0054BC0200E88600202DE9F04F97B0DFF8C0
:1031FC0010850546DFF80C6598F800000328307040
:10320C0040F04C81002088F8000030700DAC204656
:10321C0026F0BBFC2046002124F069FEDFF8E89480
:10322C00B0603A21484625F049FE4FF0FF30A9F82E
:10323C001400C9F81000C9F80C0022F0B9FD0020E8
:10324C0029461DF0F1FF06F11001F06026F02BFC71
:10325C00D6E90502DFF8B474B0FBF2F1C9B2032968
:10326C0028BF032189F800103970B2F5005F40F0D7
:10327C001281B0EB413FC0F00E81F068002800F0E5
:10328C000A814FF40050FF224FF000084FF0885B8A
:10329C00A9F80600FF2089F8032089F8058005901D
:1032AC000020089000200B9000200990002007902F
:1032BC000020069000200A9000200C90FF20029025
:1032CC00FF200490FF200390CCB2A04580F0E98051
:1032DC005FFA88F6002116AA0423304625F01AFF5F
:1032EC00DFF830443046002115AAA04730460121B2
:1032FC0014AAA0473046022113AAA04716996FF0D2
:10330C006F0050FA81F2C8B20E2A06D8012303FAD4
:10331C0002F245F201131A4203D1A0F1FE02022A75
:10332C0004D242F28352B2EB914F1ED0304614F0CD
:10333C0021FADFF8D0130028087040F0D280304614
:10334C00002116AA042325F0E5FEDFF8C843304619
:10335C00002115AAA0473046012114AAA0473046E7
:10336C00022113AAA0471699C8B208EB4802CA4614
:10337C003D4609EB8209C1F30142090A4C46FD287E
:10338C0004F8160F61709DF85610E270A17001D907
:10339C00102135E0BDF854104FF6FF7291422FD139
:1033AC000EA820F051FC304600214FF088524FF40B
:1033BC0000534FF4005725F0ADFE6FF0030313FAE2
:1033CC0087F7B8B250F80B104A1C01D10328F6D875
:1033DC0001220126D3B2042B06D8CBB2FF2B18BF87
:1033EC0016460132090AF5E740F80B10CA480E9947
:1033FC0000684268C948904757FA86F081B2207835
:10340C00A9F81C109DF85210702889F81A10BDF8F4
:10341C005010A9F81E109DF84E1089F81B10BDF81D
:10342C004C10A9F8201011D07828D14614D07C2843
:10343C002F4616D07E281AD0FE281FD0FF2823D165
:10344C000898CDF80C800130089020E00A98D146FD
:10345C002F4601300A901AE006982F46013006904C
:10346C0015E00798CDF81080013007900FE009980F
:10347C00013009901FFA88F0029008E00B98CDF803
:10348C00148001300B9002E00C9801300C903978CC
:10349C0008F1010818E7012088F8000017B0BDE812
:1034AC00F08F0C98974E00060BD10B98C0B20128E8
:1034BC0007D80A98C0B2012803D80998C0B20128CD
:1034CC0011D99348042200240270CAB2E0B290428F
:1034DC0010D214F04FF93178013408433978307038
:1034EC00F3E7884E1BE0089BD8B2A04219D188485C
:1034FC0000220270002089F8030089F80100481EA0
:10350C007E2189F80200B9F81C00A9F806000020F9
:10351C0021F0A6F899F80200FE2121F0A1F83078EC
:10352C00BCE70A98000624D00B98059A000603D134
:10353C00039A180600F08480754802210127D5B241
:10354C0089F80220017017FA82F0B0FBF4F101FB4C
:10355C00140089F80100284614F00CF93070284644
:10356C00FE2121F07DF889F805700020FFF7DCF8CA
:10357C00D5E70B98059A000621D06548012189F8FA
:10358C000220017011FA82F0049AB0FBF4F101FBF5
:10359C00140091B2FF2989F801001FD10299FF296B
:1035AC0019BF89F8031001EB410089F8030000EB07
:1035BC00400009EB8000808BA9F80600AFE7DDE93D
:1035CC000620104300063FF47CAF22F0C5FBA0425E
:1035DC0080F085804E48032101703EE0480089F858
:1035EC00032010FA82F009EB8000818B1829A9F8CE
:1035FC00061094D30739D0B20EAA89B216F058F837
:10360C009DF843004007B0D5B9F80610BDF8462028
:10361C00002399F8030000930323891A0EAA073993
:10362C0089B206F0B5FE00287FF479AFBDF84410DE
:10363C0000293FF474AF9DF848001DF085F86EE743
:10364C0022F08AFB0621A042314838BF032103290E
:10365C00017002D0062952D061E722F07DFB0546AD
:10366C0089F80C0000EB400009EB8000408BA9F8B6
:10367C000D000CF08BFD39782844B0FBF1F202FB05
:10368C00110089F802000130C2B2B2FBF1F202FB68
:10369C00110089F801007C2020F0FCFFFF2812D1DA
:1036AC007E2020F0F7FFFF280DD1FF2020F0F2FF45
:1036BC00FF2808D1782020F0EDFF014699F8010091
:1036CC00FF2918BF0846C1B289F80300490051FA16
:1036DC0080F009EB8000808BA9F806001AE70898A7
:1036EC00000609D099F80200FE213C46374620F02E
:1036FC00B7FF2478039A40E7054806210170FEE7DE
:10370C0088270020A0230020A0800020978800207C
:10371C00A38800203B930200D80100100040034016
:10372C002DE9F84305460C46480413D4A00024D4D4
:10373C00A0075CD460057ED4200500F1068120072B
:10374C0000F13B81600040F1F68019F049FF24F054
:10375C008044F0E025F0ECFEDFF81C140F6D3FB157
:10376C00D7E90A1202F0E04201F00A01891849D0A7
:10377C0026F08AF924F48044DDE0BB48DFF8FC73C2
:10378C00016841F080010160B878012804D104205F
:10379C0020F0E8FF0020B87025F0CAFE0646042091
:1037AC0025F06EFFDFF8D8130A68904219D12A7EF3
:1037BC00BAB1FA68AAB1DFF8C003806C002800F037
:1037CC009780C16840F603020988914206D0C06810
:1037DC0040F604010088884240F08A8005F114000C
:1037EC0088E040F6C4120860C5E9042284E009F0C0
:1037FC0061FBDFF88403006C002840F09D8024F00E
:10380C00020498E0D7E90A65D7E90A12AA43B14342
:10381C00C7E90A1226F038F9B8680028AAD056EA87
:10382C000500A7D0D7F808C03869B7F93010324670
:10383C002B46E0479EE725F07BFE054623F0B0FCC7
:10384C00002800F0B780CC48876B002F00F0B280C6
:10385C00DFF828830420CB49002288F81800C648DA
:10386C0025F0C0F826F03AF9C74826F007F9C74802
:10387C000068006B8047C8F810000125042088F808
:10388C00025021F08DFD386990F82810C8F804001A
:10389C00490703D5436A04210022984701201BF0F5
:1038AC0029FCD8F80400457612F0F0FFD8F8040093
:1038BC0081680B461A465B684BB11E88A6F6030658
:1038CC00072EF7D805FA06F616F0830FF2D0537BC5
:1038DC0003F0F003013353730023FD6853602D880C
:1038EC00A5F60305012D00F28A80C8F810309FE080
:1038FC0005F110001EF0ACFA304626F0C5F821F0A8
:10390C0067FD78B12E6A28466FF4807100224FF063
:10391C000073B0479848806B10B119F061FE01E05C
:10392C0044F00204EE692846002100224FF0806327
:10393C00B04724F0005434B1974821462830BDE8F4
:10394C00F84326F081B9BDE8F8838C4EB078012895
:10395C0004D1042020F006FF0020B07021F038FDC7
:10396C0038B170686FF4807100224FF00073056AF3
:10397C00A847306950B185480068006B80473269B0
:10398C007168801A000BC860002030617A4D814943
:10399C000022284625F026F802203076286C20B12B
:1039AC007D480221283026F04FF919F019FE24F435
:1039BC000064C0E726F092F841E025F0B9FD054619
:1039CC0023F0EEFBA0B1DFF8B48198F800000007FB
:1039DC000ED498F9000000280AD4684613F0E4F9D4
:1039EC0008B1009820B1DFF8B49199F8610048B3A0
:1039FC0026F074F819F0F4FD24F008049BE7034654
:103A0C0033F8385FA5B190F8445090F8456005F054
:103A1C00F00580F8445006F0F005013580F845506B
:103A2C0000255360C5634587507B00F0F000507350
:103A3C0057480022C2610160012024F003F824F4ED
:103A4C00806478E700260127602E0FD009EB060072
:103A5C00817A31B18772407A07FA00F0C0B220F057
:103A6C009BFE2036F0E700BFCC210840032088F8ED
:103A7C001800454826F002F826F030F8444F3E4D29
:103A8C000022786900207861F968F860284644497A
:103A9C0024F0A8FF3D480068006B8047D8F80C1054
:103AAC00D8F82020411A02EB1130B0EB113F38BF8F
:103ABC004FF0FF3098F82410C8F8200021B1D8F846
:103ACC000810B0EBC12F20D923F0CCFFB8B140F6D1
:103ADC000900414621F83C0F002048804A7B02F047
:103AEC00F00201324A730A7B02F0F0020A7348605A
:103AFC00F8613960B8F83E0010F4406FFAD000203D
:103B0C00C8F82000012088F824001DF045FB25484A
:103B1C00002101600220002123F094FF022020F0FC
:103B2C0021FE102011F08CFE98F8010020B9D8F875
:103B3C000400503026F084F81B48807810B90D2012
:103B4C0011F07EFE98F8250028B1002088F8250099
:103B5C00052020F007FE002088F818001348C8F84C
:103B6C001C000220B5F85610B5F85420914208BF3D
:103B7C00072018F07DFE3DE730210020D01E0020EC
:103B8C00D426002089710200207F00208C010010B7
:103B9C0000100440D10C010070200020B87B0020E4
:103BAC0051D6010000000460ACBB0200A903010067
:103BBC002DE9F04F8DB084780226142C00F21F8270
:103BCC000546DFE814F02900150015004A008500B1
:103BDC001C021C021C021C021C021C021C021C02E9
:103BEC001C021C021C028E009C00AF00BE00CC000C
:103BFC0001206A78022C8DF83100089240F0C080C8
:103C0C00E878291D03288DF82C0040F0E18009A8E4
:103C1C00082225F0B7FAE0E010208DF824001020DF
:103C2C0025F0FCFF98B10446DFF8E0032146606004
:103C3C00E81C10F0FFFA8DF8240028B9204623F078
:103C4C0051FB8DF8240010B1204625F0E5FF00262D
:103C5C0009AB642000210122C2E10020CDF82A002A
:103C6C00ADF82E00CDF8260002208DF82C00E81CB3
:103C7C0025F0D0FFADF824006979A8798DF82D10C6
:103C8C0025F010FB8346E81D25F0C4FF95F80C9039
:103C9C008046687AAC7A95F80BA04FEA49078DF804
:103CAC003100384625F0BAFF002800F01081CDE92C
:103CBC00074806464FF0000805EB0800474570D052
:103CCC000D3025F0A7FF26F8080008F10208F3E7ED
:103CDC00E87820F065FE8DF8240009AB64200421FF
:103CEC0089E1E978032900F25281281DDFE811F0FF
:103CFC000400510155015D0118F05CFE76E1E81CF1
:103D0C0025F088FFC04C6668002E00F0E4806A79CC
:103D1C00002A00F0E4803368A91D184425F032FA1B
:103D2C000020D9E0B84EEC1C04212046376822F064
:103D3C00EFFB002F4AD0B968814200F0A0803F68A9
:103D4C00F7E7A888ADF82400E87809A924F058FA18
:103D5C008DF832000DF13203642013214BE1002663
:103D6C00E878ADF8246009A923F066FCBDF82400BE
:103D7C000DF1320314210222ADF8320064202FE140
:103D8C00E81C02218DF82C1025F044FFADF824001E
:103D9C00002005F10608ADF82E0068798DF82D008D
:103DAC0026E0BBF1000F00F0B580437B0DF1310133
:103DBC000E30CDE90496CDE9000107985946CDE9BE
:103DCC00020A09A8089A1DF089FEA4E0012000E16E
:103DDC00084625F01FFFADF82400287B8DF82D0038
:103DEC0005F10D0025F016FFADF82E0005F10F08BA
:103DFC0098F8000025F056FA054608F1010025F068
:103E0C0009FF98F8036098F804A098F805B081466B
:103E1C00022C8DF8326009D108F1060025F0FAFE6B
:103E2C00074608F1080007F10A0104E098F806704B
:103E3C0008F1070039464DB10A3189B2FB2907D385
:103E4C00DFF8C481D8F8040000286ED0022009E005
:103E5C000DF132018DE8030C09A84A463B46294670
:103E6C0003F016FF089E8DF8310006F0E0002028C4
:103E7C0040F0C4800DF1310364202146BBE0EC1D01
:103E8C00204625F0C7FE6D7A002D00F0978005F1D5
:103E9C0002098246484625F0C1FE002800F09880B1
:103EAC000026457080462A460670786800EB0A01A9
:103EBC0008F1020025F066F95FFA89F264201221FC
:103ECC0043461EF0D5FB404625F0A6FE97E0102099
:103EDC008DF8320024E010208DF8240016E0D6F87E
:103EEC0000C0F38AB28A3169757EB77E06F118007C
:103EFC00CDE900C0301DCDE9025703F0C9FE8DF8A5
:103F0C002400606825F088FE0020606009AB642006
:103F1C00112170E002208DF83200304625F07CFE35
:103F2C000DF132036420032165E007F11C0025F03C
:103F3C0075FE0028C8F8040055D000F11C010C22B5
:103F4C00016000208DF83100D8F8040009A9043074
:103F5C0025F018F9D8F804000F214FF47A72056196
:103F6C002A4DC17680F81AB080F819A00676C7825F
:103F7C00A0F814900821287825F0B6FD089E00289A
:103F8C003FF473AF287808211AF05CF86DE7022033
:103F9C002CE000781AF086F828E0007825F082F9F9
:103FAC0018B324F063FE002020E025F033FEA9793D
:103FBC0025F096FBB0FA80F0400917E03068B84263
:103FCC0001D138683060384625F026FE002000E02C
:103FDC0010200026207064201221022223466670D5
:103FEC001EF046FB0BE010203CE701208DF824006E
:103FFC0009AB6420102101221EF03AFB002630464A
:10400C000DB0BDE8F08F00BF5C2600209688002024
:10401C002DE9F04F8FB00C4608040CD4A00426D424
:10402C00DFF88853287802282DD1E10740F0018170
:10403C00A10641D558E0DFF86C0300781AF000FDBA
:10404C0090B10178DFF8602305460020602808D085
:10405C00135C08308B42F9D1104450F8041C2846EC
:10406C008847284623F0F8FE84F4004595E11DF0BE
:10407C003BFC28B10546FCF7EDFD284623F0ECFE91
:10408C0084F4005589E1A1062ED4012814D8E10648
:10409C0000F11781610600F12F81210600F13D81AD
:1040AC00E10500F13F81210500F14181E10400F1BE
:1040BC005481610400F15B81A10700F1E080A1054E
:1040CC0000F1FA80210700F11181610500F11981DD
:1040DC00E0034FF0000540F160811BF037FFB6485C
:1040EC00C57084F4803558E1AE4F202138781FF02C
:1040FC0061F8DFF8C4820125D8F80810084317D0FE
:10410C0025F05EFD054625F059FD68434FF47A71A4
:10411C00B0FBF1F0D8F80810401A4FEA500538BF40
:10412C006FF00045002908BF0D46002D00F0C2803D
:10413C0000200421002222F055FD06464FF0060A0D
:10414C004FF0FF094FF6FF780DF1080B002E4DD004
:10415C00304604210022374622F044FD06463889B9
:10416C00401B38BF002038810004EFD1B87BD0B39E
:10417C0001280AD17889400707D4386887F80DA040
:10418C00B721407B1DF068FBE0E739685A468DF893
:10419C000690ADF80480086AC97F0CF089FF0128ED
:1041AC001BD1B87BB97A8DF838000907788A40F0B2
:1041BC008002ADF8362006D540F4C070ADF836005C
:1041CC00387B8DF83A00786910B1007BADF8180097
:1041DC00584601A9002202F027FC387B87F80DA075
:1041EC0016F038F8B2E701207873AFE7DFF8C88132
:1041FC006C4F22F057FE00200121002222F0F2FC2D
:10420C0018B13878202119F01DFF0020042100225C
:10421C00002622F0E7FC002847D006890421002262
:10422C0022F0E0FCA0B10289B1B2914228BF16463F
:10423C00F4E7654890F82C100F2906D190F8260069
:10424C00022802D3002021F07BF884F00105A4E0C1
:10425C00A8B2B1B2814223D9D6FA55F0202180B24E
:10426C004200387825F040FC25F0AAFC054625F0E4
:10427C00A5FC68434FF47A71B0FBF1F615E0534896
:10428C00007818B302AD284625F0A5FB25F074F98B
:10429C004F490B784F490A7829461AF0A7FE22E0BD
:1042AC003878202119F0CEFE0026C8F8086084F07A
:1042BC00200572E000259CE715F0C8FB84F400751E
:1042CC006BE008F05DF984F0100566E03E48418B28
:1042DC00012025F099FC2878022804D131480121CD
:1042EC0000781AF07FFB84F0020556E03248012179
:1042FC0084F00805817050E00CF0D4F884F040058F
:10430C004BE0022808BF15F0A5FE2F480121808C38
:10431C0025F06CFC84F480653FE024F091F984F086
:10432C0080053AE022F0BAFA84F4807535E01BF08F
:10433C0049FB2048007801280CD11D48007848B171
:10434C004FF47A7100FB01F216484FF400610078CB
:10435C0025F0C7FB84F400651FE01748017819B1FC
:10436C00002101701BF02EFB84F4805515E01448DD
:10437C00006880B11149097801290CD18047114896
:10438C00006800B1804707484FF480414FF47A72BF
:10439C00007825F0A6FB84F4804528460FB0BDE8D4
:1043AC00F08F00BF9888002030B50200182600203E
:1043BC00BC270020BD270020E8250020BA270020BC
:1043CC008423002090230020407B0020972700208E
:1043DC00C0270020C22700202DE9FE4F8846080484
:1043EC0026D45FEAC87004BF0020BDE8FE8FE54804
:1043FC00056825F0E5FB044625F0E0FB60434FF42F
:10440C007A714FF6FF72B0FBF1F14FF6FF70002D91
:10441C0000F01A812B886C88CB1A9BB29C4240F21C
:10442C001C81E31A94B2A342B8BF1A46ED68EEE7BA
:10443C00DFF840A3CDF804809AF800001AF000FBD6
:10444C00002800F0FC8006460078012840F0EC8043
:10445C00DAF8041096F83390D6F814B096F8138066
:10446C0021B148468847002840F0DE80718896F8D4
:10447C003100022222F05EF90546002842D0287A4B
:10448C00297CA0F10108FF2900F0BB80707F4F460A
:10449C00C00718BF0027E97C287D0144B94204D825
:1044AC00E974FF2101FA00F06874A969A87C96F8F8
:1044BC003020896A10FB0710F16A24F063FE287D16
:1044CC00697CB7FBF0F202FB107001228240D2B281
:1044DC000A436A74C8457CD196F83010AB7C13FB48
:1044EC000713A9698B844FF4FF7303FA00F0C0B271
:1044FC001043FF2868746CD1287C1AF0CFFDFF2084
:10450C0028747FE0707FC00700F08E80B07F24F0AD
:10451C00C9FE002800F0888004461C2025F07EFB94
:10452C00002800F081801C21054624F0C7FCB07FD8
:10453C0002A923F081F89DF809000221287528466C
:10454C0023F0D0F8708896F8312096F8301096F851
:10455C003330A880287DEA71FF2202FA00F06874DB
:10456C0060680078A9742874302013FB010080B2B5
:10457C0022F074FD0028A8615DD004461A20B11CFD
:10458C002060708CA080A01D23F048FEF27F04F107
:10459C003000B17F96F82830C4F81CB084F819802C
:1045AC00A062307CE273744A217563750121A07599
:1045BC00928C2282F28EA285F28C6282B6F8110065
:1045CC00A4F817009AF8000085F8089019F03AFD45
:1045DC0055E725F0F5FA044625F0F0FA60434FF460
:1045EC007A71B0FBF1F0654928806348097800794D
:1045FC004843642148436249097800FB0100688004
:10460C0000E04F46E87C297D6A7C01440139B942BF
:10461C0018BFFF2A0CD186F83300708806F11C01F4
:10462C0086F8342016F0A5FF304623F015FC03E77E
:10463C00C845F9D1EFE7284623F064F8F4E7019870
:10464C0080F40040BDE8FE8F92B282424BD04948C4
:10465C000121007825F048FA45E0A879022806D116
:10466C00287CFF2837D0A86923F0F6FB33E025F02F
:10467C00A7FA044625F0A2FA60434FF47A71B0FB16
:10468C00F1F03F49288095F83800097888421BD210
:10469C0095F83620FF2A06D195F83720013085F899
:1046AC00380085F8362095F8351095F8394082F0A9
:1046BC00FF0300200126C7B2A7421DD206FA07F756
:1046CC001F4214D10130F6E7EA8BA87E95F82A1028
:1046DC00E9231EF0B9FE284623F014F825480121E1
:1046EC00007819F0AFFC88F00100BDE8FE8FFBB23A
:1046FC0001441A4385F83620AB8F95F83440C8B284
:10470C0004FB10339EB2A64203D2FF2285F836205A
:10471C0002E0FF2A08D12346184A174E1278367940
:10472C0072436426724302E095F83A2023466A806D
:10473C002A8D0E0606D022F0200244432A852A6CCC
:10474C00224404E042F020012A6C2985297A85F85C
:10475C002E10E9796A6285F82D10D9B26984054961
:10476C00496811B188470028B8D105F1100004F050
:10477C0021FAB3E73C260020407B0020B027002024
:10478C00B6270020546500207FB50138072800F2B9
:10479C004C810C46DFE810F008002C0054006E0031
:1047AC0089004901A600C900CB48007801380128CE
:1047BC0000F23B81002C00F04781002003210024F3
:1047CC001FF07CF8C64DC74E0420042132222870FD
:1047DC00307825F089F90820002107F097F8307817
:1047EC006C704FF4805104B0BDE870401AF0FAB808
:1047FC000020002524F05EFDBB480121017004203F
:10480C008DF80D0074B1B548B34C4585207801285E
:10481C0003D1072023F066F92078022802D1062064
:10482C0023F060F9AE48042132220570AD480078BF
:10483C0025F05AF9A94890F82B1001F0FE01F2E08E
:10484C00A54800780138012800F2EF80A548042122
:10485C003222007825F048F9002C00F00F819F4C93
:10486C009F48012101702069002800F0EC801FF0A6
:10487C00C7FBF8E70120002C8DF80D007BD0974882
:10488C0000219B4A80F82A10984824F0DBFE924CB9
:10489C002078012803D1072023F024F9207802285E
:1048AC0070D1062023F01EF96CE002208DF80D006B
:1048BC008A48002C73D000218D4A80F82A108B482E
:1048CC0024F0C0FE002003211EF0F8FF824C20785B
:1048DC00012803D1072023F005F92078002877D18F
:1048EC00092073E07C4D00208DF80D00002C2878F9
:1048FC007BD018B9092023F0F5F82878022806D1C6
:10490C000820002107F002F8042023F0EBF810F047
:10491C00F1FF73480021C822017070480D2180F806
:10492C002A10704825F06FF878E005208DF80D00FE
:10493C0069480078022878D1002C00F0C3806848C0
:10494C000022C178C270017042F20800002106F00A
:10495C00DDFF62480D2190F82B2080F82A10C178D9
:10496C0002F0DF02002980F82B200CBF04200D2060
:10497C0023F0B8F859E05848007818B95748022184
:10498C0080F82A105648002132220170554825F033
:10499C003AF8524890F82B1001F0FD0143E0082141
:1049AC0080F82A104C490978012911D890F82E006A
:1049BC0070B900200DF10A018DF80A0052201DF08B
:1049CC0057FB24F0F3F91EF09BFB002023F08AF830
:1049DC004348002132220170424825F014F83F4828
:1049EC0090F82B1001F0FB011DE03C4C022812D179
:1049FC0094F82E0078B194F82B00002140F02000A0
:104A0C0084F82B0005208DF80D00082006F07EFFA1
:104A1C000A2023F067F8022084F82A002F4890F827
:104A2C002B1001F0EF0180F82B102C4800220323EF
:104A3C0090F82A008DF80C002A48007803A9009100
:104A4C000A211EF012FA7FBD244C0720254D4FF48D
:104A5C00805184F82A0001208DF80D00287819F077
:104A6C00C1FF0020002622F031F82878022141F203
:104A7C00883284F82B6025F037F8D6E7174C0220E3
:104A8C0000218DF80B1084F82A001548017094F859
:104A9C002B000DF10B0100F0FD0084F82B00012020
:104AAC008DF80D0052201DF0E3FA24F07FF91EF072
:104ABC0027FB002023F016F820690028B5D01FF042
:104ACC009FFAF9E70548022180F82A1090F82B107C
:104ADC0041F02001A7E700BF18260020AC220020DF
:104AEC00088800209F880020AD270020407B0020F4
:104AFC008027002092B0DFF8EC92D9F8000010B1BA
:104B0C00002180F84510483020F02AFE24F010FDDA
:104B1C008046072011F006F917F0E0FE10B1B248FC
:104B2C0024F0AAFE1AF03EFB01AD284624F09AFBB5
:104B3C000427002029468DF8047024F09BFBAB4C15
:104B4C00206023F0E9FF0AAD284624F03BFA002050
:104B5C0029468DF8287024F03DFAA54E306023F0DC
:104B6C00E5FF06AD284624F03DFA002029468DF8D5
:104B7C00187024F03FFA31689E4D286019B99E4890
:104B8C0024F07AFE286810B99C4824F075FE206841
:104B9C0010B99B4824F070FE1CF086FDD9F800007B
:104BAC004FF0FF3438B1CDE9104410A9082223F09E
:104BBC0039FA01281BD1CDE91044082025F02EF834
:104BCC00002846D005460026052E04D824F0BEFE4B
:104BDC00A8530236F8E74FF6300029460822E88041
:104BEC00884824F0CFFA284625F016F809E0D9F8C1
:104BFC000010CDE910440029DFD08248082224F0AF
:104C0C00C1FA10AA0120082124F0F4FD092800D0D3
:104C1C00D8B921F079FD800712D4CDE91044CDE943
:104C2C000E440EAB01200021082224F02DF960B9AE
:104C3C000EA810A9082223F0F5F9002800F0CB806B
:104C4C00704A0120082124F0DBFD6E49E2201DF0A2
:104C5C000FFA12F077FB282024F0E0FF6A4E0028B0
:104C6C00306055D0694F6A4C07F10C0524F0C7FE33
:104C7C0024F018FA3068056007F1100524F0BFFE27
:104C8C0064498968D1F84C1388473068456007F14E
:104C9C00140524F0B4FE1CF00DF93068856007F1A2
:104CAC00180524F0ACFE19F05BFD3068C56007F107
:104CBC001C0524F0A4FE1FF0CFFB3068056107F142
:104CCC00200524F09CFE1EF0B1FA3068456107F116
:104CDC00240524F094FE1DF043F93068856107F13A
:104CEC00280524F08CFE23F02FFD3068C56107F1F8
:104CFC002C0524F084FE20F0BBFC3068056207F123
:104D0C00300524F07CFE387024F014F830684562CD
:104D1C0018F08CFE404841494FF00009CDF8409006
:104D2C0001603F480321119010A820F0F1FA24F003
:104D3C0091FB404624F0A8FE17F0DEFE24F02EFE78
:104D4C0001201DF095FE19F033FF3748007802283A
:104D5C0008D134480078012804D14FF400400121D7
:104D6C0006F0D4FD294F4FF48041387824F07CFCB8
:104D7C002E484FF0FF3100680DF036FCDFF8B080A4
:104D8C0078684FF0FF310DF02FFC3068002550F89B
:104D9C002510096821B9691C092D0D46F7D3EFE7D9
:104DAC0024F0CFFD316851F825100C68C1F8009043
:104DBC0024F0A3FE58F825200020214690470446F5
:104DCC0024F0BFFD316851F825100A6822430A60AF
:104DDC0024F093FED4E70B480EA9082224F0D2F954
:104DEC0033E700BF5C270020F0B50200F0870020FD
:104DFC00F4870020F88700200EB6020021B60200CE
:104E0C0034B602009E8700206C8800208821002088
:104E1C00094702000C0100209C230020A5C70100BB
:104E2C00008D1500D527002018260020488800206A
:104E3C0074B802002DE9F04F89B08A4608040DD4ED
:104E4C005FEACA7040F01D815FEA8A7000F12B8125
:104E5C005FEA0A7000F13381002042E1A24F3878FA
:104E6C0019F0EEFDDFF88892A04C06464FF0000BCF
:104E7C0048F21508002E00F001813078312838D026
:104E8C00322849D0D32840F0B380F089404573D004
:104E9C00382840F0AD80CDF820B0CDE906BB3046C7
:104EAC0006A920F03DFB9DF81C10052968D8307B25
:104EBC00002840F09D809DF81D00002800F098808F
:104ECC00052800F29580069823F0ADFD002840F0EF
:104EDC008F80707C87497870708808809DF81D00E1
:104EEC00214601388DF81D0006A890E82C002CC135
:104EFC007EE0B87803287BD899F82E10804823F0F0
:104F0C0092FD002874D1FF207C4960717088088064
:104F1C00B088794908806BE06079FF2814D00020B4
:104F2C0016F074FA0246B9F8701078783346CDF85A
:104F3C0000B012F04FFD6079002859D03878082164
:104F4C00322224F0D1FD53E099F81810706820FA41
:104F5C0001F2D2071ABF3144097A002106F1080286
:104F6C0000231B2B42D020FA03F5ED0702D0D55CB1
:104F7C00A9421ED80133F4E7304621F007FD37E093
:104F8C00FF293DD0FE2956D199F872109DF81E00CC
:104F9C00884202D860BBFF292AD11CF06BFE06990F
:104FAC0000201B2859D021FA00F2D20757D101302A
:104FBC00F7E7B9F86E004F49334608804E4802882F
:104FCC004E48018810200090002012F003FD0120B3
:104FDC00F870B87840B93C2002214EF66022B880B7
:104FEC00387824F081FDB8780130B87084F805B0B9
:104FFC00304622F031FF387819F022FD064639E7A9
:10500C0099F872109DF81E00884203D80028EFD141
:10501C00FF29EDD11CF02EFE069838B1D9F82810D6
:10502C00814203D0C9F8280022F06CFDBDF82000A5
:10503C0023F0BAFBDCE7307B0028D9D170882D49EE
:10504C00802200230880707CCDE900BBCDE902BB37
:10505C00CDE904BB11F074FBCAE71B2000E0C0B221
:10506C0099F818108142C3D02649087099F80700A6
:10507C00642100FB01F23878012162E78AF40040D8
:10508C002FE020491A4C08782076E1201CF0F0FF24
:10509C0022F038FD0020A4F87000012016F0B6F9BB
:1050AC008AF001001DE010488188B1B101394EF63B
:1050BC00602281800078022124F016FD0FE00B4C59
:1050CC00607938B12179206823F0ADFC10B9607992
:1050DC00013860718AF0080003E0002181708AF0C9
:1050EC00020009B0BDE8F08FCC24002040870020DE
:1050FC00407B00207A8700205E840020DA8000202C
:10510C0000F8FF079B8800202DE9FE4F0746086832
:10511C000024B0B1D7E9018A0E4624F009FA814681
:10512C00D8F8E800082888BF0124B068204202D1D2
:10513C007068204208D003203074484624F0A4FC48
:10514C0000242046BDE8FE8FD8F8C01069B198F84D
:10515C00F8100029EFD006213174D8F8C410C8F823
:10516C00C4604E6198F8FC100DE000210522C8E9DE
:10517C003066C8E93411C8E9361198F8FC100029DA
:10518C0008BF0122327400220129726109D1022068
:10519C004FF4E02188F8FC0098F8FB001FF0C8FFE2
:1051AC00706889490138884205D8042020F0F8F845
:1051BC00062020F0F5F8022020F0F2F898F8F8001C
:1051CC0040B9DAF83C003168814203D298F8FC000F
:1051DC0000286CD0D8E9361009B118B900E028B312
:1051EC0024F015FCDAF80000416941F0010141613D
:1051FC00484624F049FC98F8F80008B10124A0E7CF
:10520C0008F16C05D8F8EC10284624F0B3FB002804
:10521C00F4D0D8F8C00003210174384612F0EAFF2C
:10522C0028460021002424F0A5FB8AE79AF8040004
:10523C0024F0D2FC654CDAF810100222206991FAA5
:10524C00A1F1B1FA81F14368D8F8CC00406800684C
:10525C0098472069DAF8141002224368D8F8CC0079
:10526C0091FAA1F1B1FA81F14068006898479AF877
:10527C00040022F087FA9AF8040024F0AFFC24F022
:10528C00C6FB0020C8F8E000D8F8C0000068B0F5F4
:10529C00806F01D924F0BBFB98F8FE000028A1D147
:1052AC00DAF80000416841F0020141609AE798F891
:1052BC00F90020B1D8F8EC0001307FF48BAF4846F0
:1052CC0024F0E2FBB2683AB1D8F8E80002210928D0
:1052DC0038BF0121009103E008F1F4020020009096
:1052EC00746834B1D8F8E8000227092838BF0127C0
:1052FC0002E008F1F6040027DAF80000334D4168AB
:10530C0041F002014160D6F800B0D946BBF1000F64
:10531C0040D0D8F8E800019209284FF0010011D2D2
:10532C002A68B9F1000F1FD0C0071DD02178DAF818
:10533C0000009268904700281EBF3C44A9F1010967
:10534C000120EDE72A68B9F1000F16D0C00714D080
:10535C002188DAF800009268904700281EBF3C4470
:10536C00A9F101090120EDE7DAF80000D26802A9E1
:10537C009047DDE90120107007E0DAF80000D268F0
:10538C0002A99047DDE9012010800098ABF1010BD8
:10539C000244BBE7D8F8F000DAF80010CA68024003
:1053AC00102802D1002AF9D101E0002AF6D0706849
:1053BC0022F070F8D8F8C0100020C8F8C400C8F863
:1053CC00C00008741AE700BFFEFFFF0FC4010010F5
:1053DC002DE9F04F85B08846080418D4A948007808
:1053EC00012802D85FEAC87155D15FEA88714CD4A4
:1053FC00022807D1A4480078012803D15FEA48703D
:10540C0000F188805FEA087057D400202BE1DFF8A8
:10541C005CA29AF8000019F013FB002800F021811F
:10542C000546807FC8B9688C132816D190486E88C1
:10543C0000F11C09002049464F46002818BF071DE3
:10544C00086850B1014631F8042BB242F4D14468DB
:10545C003C6024F0E1FB2046F3E7A87A05F1020B4F
:10546C00022840F0E480DFF8089295F83170BBF820
:10547C00006009F11C000068A0B10188B14202D1A2
:10548C008178B94242D00430F5E7794801210170A6
:10549C0088F00200E7E07648406900B1804788F068
:1054AC000100E0E0D9F81C40002C57D001206168C5
:1054BC00002955D001300C46F9E77048DFF8B0915F
:1054CC00807BD9F81C60000760D424F079FB04467B
:1054DC0024F074FB6A4A60434FF47A71B0FBF1F02C
:1054EC00D9F818101288411A91427AD3B1FBF2FB09
:1054FC000BFB02F2511A08445E49C9F818001FFA56
:10550C008BF00978884288BF8B4641E0594909786D
:10551C00C170A3E05E495D4800224FF6FE73002483
:10552C000978023079B130F8025C9D4208D0458888
:10553C00013D45802D0406BF027020F8023C012479
:10554C0001390630EEE734B1484804214FF4FA72C1
:10555C00007824F0C9FA88F0040084E000240020CC
:10556C00454980B20988884261D2082024F056FB54
:10557C0000285CD000210680877041603D49097885
:10558C00C170D9F81C1079B360603FE04FF0010B8B
:10559C0000205FFA8BF44FF0000A071D002808BFAB
:1055AC0009F11C0796B1F078C0FA5BF1A042F170DA
:1055BC0006D8756830463D6024F02EFB2E46F1E788
:1055CC00716830460AF1010A0E46E6E75FEA0A40C6
:1055DC0007D100200821C9F818002448007819F0D8
:1055EC0001FA88F008003EE0C9F81C002348807BD3
:1055FC0000070BD424F0E4FA044624F0DFFA6043ED
:10560C004FF47A71B0FBF1F0C9F818001B48807B9D
:10561C0000070CD59AF8000008211DF0CBFD30B91D
:10562C001748082102889AF8000024F05AFA2878C2
:10563C00022810D0012811D1297EAA89EB7C05F112
:10564C001C006C696E7E8DE85A0005F110035946FA
:10565C0005F0FEF802E0284615F0A0FA284622F0E4
:10566C00FBFB88F4004005B0BDE8F08F9588002066
:10567C002C240020B52700207A270020407B002016
:10568C007E27002018260020D52700204C6D0020F6
:10569C00912700202DE9F04F87B0851C83462846C2
:1056AC0024F0E9F901AC06461821204623F006FC4B
:1056BC009BF801A004F10B002946009524F059FA3F
:1056CC006FF001009BF80A1002240122ADF81800BB
:1056DC0000208DF81A408DF80C0001F00800C1F381
:1056EC00C007890782EAD00507D4002808BF012427
:1056FC00B946A8460027002507E004244FF000090E
:10570C004FF00008002808BF03248548007850EAB1
:10571C000A000BD0834890F82600082809D123F002
:10572C0079FC00285AD0BAF1010F57D14FF0C309B8
:10573C0001E04FF0C2090025BAF1000F10D07F48EC
:10574C00007890B9BAF1010F0FD1002E55D000207E
:10575C00214601228DF81A0001A814F03BFA0AE048
:10576C0001A81BF06DF986B91CE001A82146524630
:10577C0014F030FAB6B17179BAF1020F41F040026F
:10578C00727104BF41F0600171719BF80A104906F7
:10579C0003D5717941F080017171B1790024013127
:1057AC00B17100E00124B0FA80F149090D422CD10D
:1057BC0007D1002D18BF814641F20100494618F06F
:1057CC009EFF14B9009819F061FBBDF818004FF654
:1057DC00FE71884218BF24F02BFA16E0DEB3327942
:1057EC00A24218BFBAF1020F12D1D01EC0B20128CA
:1057FC001BD857EA050020D12AE0022021460122BD
:10580C008DF81A0001A814F0E5F907B0BDE8F08F87
:10581C004FF00009009953468DF81A903088ADF876
:10582C00180024F0E5F9012586E7501EC0B20128C6
:10583C000ED849EA0800012807D1308821F0AAF9CE
:10584C0050B93088ADF8180008E0308824F0F0F931
:10585C00009819F01BFB0026BDF818004FF6FE71DE
:10586C0088421ED120F08EFF10B1BDF8180011E057
:10587C00BAF1000F04D02C4D288821F08BF930B1EF
:10588C009BF80A0000F002001FF0BAFD00E0288827
:10589C00ADF818004FF6FE71884202D14FF0C709DF
:1058AC0049E79BF80A200099534624F0A1F910B15E
:1058BC004FF001093FE71D48016811B1BDF8180010
:1058CC008847BDF818000099224606F0D9F806461C
:1058DC00174818490A6800784FF4803124F004F90D
:1058EC0001211548C17096B1AAF10100C0B201287E
:1058FC0007D81020BAF1020F08BF082071790843AD
:10590C0070714FF0000901258DF81A9014E74FF6CD
:10591C00FE7000254FF001090026ADF818000BE7CA
:10592C00F4240020407B00207427002098230020C2
:10593C0098880020B0BC0200E82500201826002022
:10594C002DE9F04F8DB0044600209A4616460F46BE
:10595C00CDE90B00CDE9090087488568804614F035
:10596C00B8FD1C2803D014F0B4FD1B281BD13088C3
:10597C0040F60201884218BFB0F5C15F03D1F07B3D
:10598C00022810D93EE043F6070188420BD196F865
:10599C002400032807D33069784940F0806020F058
:1059AC00604088422ED100206FB366B3387825FA58
:1059BC0000F0C00726D03046002124F029F97048A9
:1059CC00C4E90176006880B109A800900CA90BAA63
:1059DC000AAB304609F00CFF0B980B214FF6FF7207
:1059EC00502321F06FFFFF280CD023F0A1FD654F51
:1059FC0006467878012802D840B1012070E0304684
:105A0C0024F042F800200DB0BDE8F08F09F064FEE0
:105A1C005D480DF10409016841F0020101605B4829
:105A2C00C8F80000484623F00DFCDFF864B15A4971
:105A3C004A469BF801009BF80050039055482830CB
:105A4C001EF0F8FE554856494A461EF0F3FE4846ED
:105A5C0023F008FBDFF84C81534A19214B46029581
:105A6C0040461DF0B7FA514A08F11C001A214B466A
:105A7C001DF0B0FA4E484F4923F0D5FF4E484F4920
:105A8C0023F0D1FF4E48006810F4402F06D04D4A49
:105A9C0007F128000421002321F04CFB9BF80200A5
:105AAC0010B10D2010F03EF908F1400022F0A5FFD6
:105ABC0008F1380022F0A1FF434900200722387674
:105ACC00B8843862386181F860200521C7E902107A
:105ADC003E49F96138700420002121F0B3FF787839
:105AEC002C4941F8204001307870304623F0CCFF2F
:105AFC00BAF1000F06D10DF1040A354920225046A7
:105B0C0024F0F8F8DAE90012BAF81000DAE90635F0
:105B1C00002AB2FA82F608BF40F6C4126261216014
:105B2C0060832563760926764FF4FA76C4E903621E
:105B3C0001226276274AC4E90722C4E90923DAF86C
:105B4C000C0000B12062DAF8140000B16062DAF8DF
:105B5C00080000B1E06104F13800C82123F0AEF96F
:105B6C0004F15000002121F0ADFF1B4904F1B800F5
:105B7C0023F059FF204646E7CC2108400F000005D2
:105B8C0074260020D01E002000200940110000E0E7
:105B9C00ACBB020070200020BD80020028800020D9
:105BAC00E54901003021002051D60100ADB80100BB
:105BBC00647F002065710200207F00206980020054
:105BCC00B44F005049000200B87B0020A90301002B
:105BDC0064B90200BB2E0100259B02002DE9F04F99
:105BEC0087B000240293002A00F03D81074603A8E9
:105BFC0092460E464FF0200B10300190504610F894
:105C0C00011B25290CD0002900F02A81022EC0F09E
:105C1C00D980013E002F00F0D48007F8011BD1E0A1
:105C2C009AF801002D2806D19AF802000AF1030314
:105C3C004FF0010C03E00AF102034FF0000C302886
:105C4C000CBF13F8011B01462A2920D1029D2A689A
:105C5C00111D2960D2F8009013F8011BB9F1FF3F18
:105C6C00DCBFC9F100094FF0010C2E291ED11A46D8
:105C7C0012F8011B2A291CD1029D2A68111D2960CA
:105C8C009D1C126859782B4622EAE27821E04FF0ED
:105C9C000009A1F13002092AE7D809EB890201EBCE
:105CAC004201A1F1300913F8011BF2E74FF0FF3864
:105CBC000FE04FF00008A1F13003092B08D808EBD6
:105CCC00880301EB4301A1F1300812F8011BF2E744
:105CDC00134630284FF0000241F0200008BF4A461E
:105CEC006C2808BF13F8011B9A46692901D0642956
:105CFC000CD1029B1868011D19609045C8BF424623
:105D0C00DDF8048001686FF009031EE075290AD0E4
:105D1C00A1F16F00092858D8DFE800F005695F5F32
:105D2C00835F5F5F5F05029D2868031D2B609045B4
:105D3C004FF00803C8BF4246782908BF10237529C5
:105D4C0008BF0A23DDF8048001684046654616F05A
:105D5C00A5FBAC460546A8EB0001A9EB0100BCF184
:105D6C00000F0DD109E0022E05D3013E17B107F843
:105D7C0001BB00E00027013801340128F3DA0138B7
:105D8C000A465AB1022E06D3013E1FB12B7807F8F2
:105D9C00013B00E00027013A0135F2E70C44BCF16D
:105DAC00000F3FF42BAF0128FFF628AF022E05D3CE
:105DBC00013E17B107F801BB00E0002701380134A0
:105DCC00F1E700270134824618E7632905D1029ACE
:105DDC001068011D1160006804E0AAF10100022E98
:105DEC003AD300788DF80C00012103ADB5E7029A87
:105DFC00DDF804801023CDF800C01068011D11607F
:105E0C001099082200290168404616F047FB054608
:105E1C004FF04000DDF800C005F8010DA8EB0501BE
:105E2C009BE7029ACDF800C01068011D1160109913
:105E3C0005680F480029002D08BF0546284623F0A9
:105E4C0025FB0146804538BF414618F1010208BFC9
:105E5C000146DDF800C080E7002103AD82467CE7F7
:105E6C000FB100203870204607B0BDE8F08F00BF9E
:105E7C00C0A202002DE9FC47044601900578944825
:105E8C00465D9448E840ADF80260C00740F01E81C2
:105E9C000D2D13D1904E0DF10201B068D0F82824CD
:105EAC0053209047BDF802104FF6FD70814214D874
:105EBC00208990B14FF0000AA146AEE00C2D0ED017
:105ECC00072D13D0052D0ED1A078012800F0FE80EF
:105EDC00207C304400F1240716E0B068CDE0606807
:105EEC00C08AC0050AD44FF0000A09E0A07848B176
:105EFC00A07D00EBC00006EB800705E04FF0010A27
:105F0C00374605E006F11B07ADF802704FF0000AAA
:105F1C00384621F0A3F838B38146072D44D12078B8
:105F2C0089F80000607889F80100A07889F80200EF
:105F3C000028E17889F80310D4F80510C9F804108A
:105F4C005AD0A07D002889F8080049D0A169002901
:105F5C0046D000EBC00009F110068200304623F059
:105F6C0011F9C9F80C6040E00C2D40F0AF80A1464F
:105F7C0059F8040F002800F0A98023F0D9FA8046C4
:105F8C0055488068D0F8541348468847384621F065
:105F9C0065F88146404623F077FDB9F1000F00F01B
:105FAC00958023F08DFC38E023F08AFC052D34D14C
:105FBC0009F11806D9F804102422304623F0E2F82F
:105FCC00D9F8141099F8102009F13C00C9F80460B4
:105FDC0023F0D8F8D9F804002430C9F814001CE0D8
:105FEC00002089F80800C9F80C00A069A8B123F0BA
:105FFC0013FE0020A0750FE01B2009F110061B22D8
:10600C0089F808003046A16923F0BCF8C9F80C6087
:10601C00A06923F001FE0020A0613048016819B18D
:10602C0048468847002846D10D2D2BD16068017851
:10603C008A0720D42A4AC1F38301927C91421AD157
:10604C0040783F2817D894F83000022813D199F8DB
:10605C00470009F146011DF07FFF01984FF6FF72D2
:10606C00418E91421FD14068807902281BD348464B
:10607C0019F04CFE50B318488068D0F8541301A89E
:10608C00884723E00C2D0ED160781A280BD0D9F854
:10609C00040040B1C08AC00705D099F8100009F17E
:1060AC000F011DF059FFBAF1000F04D10D484946FC
:1060BC00007818F0F3FF0C2D08D1019850F8041F4C
:1060CC0021B105498968D1F85413D9E7BDE8FC879B
:1060DC00E0BA020019C206000C010020582700206B
:1060EC00407B0020988800202DE9F04F8DB00646AB
:1060FC00806A447874B18D4909788C4280F01281A1
:10610C008B49023022462AB130F8023B013A21F881
:10611C00023BF8E78748C18A708988422FD18348AF
:10612C000078A04240F2FE80B589814A214628467B
:10613C0022F020F8284616F089FE06468248077899
:10614C00BE4204D14FF6FE7016F080FE0646BE42EB
:10615C0080F0E880DFF8F48108EBC6094F4657F869
:10616C00040F08B123F058FD002C00F0B180600042
:10617C0023F054FD0028386040F0AC80D2E0B27CB3
:10618C00002A00F0CF806A4F0025AC4205D037F8CA
:10619C0015208A4203D00135F7E7A04600E0A84657
:1061AC00002113F057FE002800F0AD8081464079A5
:1061BC00012840F0A88099F8060010F0180F00F0A4
:1061CC00A280B9F80210204622F0C2F8A54202D3F0
:1061DC00002800F098805848CDE90498B6F80C9047
:1061EC004FF6FE7A00780890544800780A90002008
:1061FC0006960B9052481130099052480430079083
:10620C0000200C90DDE909564FF0000BF6B135F883
:10621C00117C574518BF4F4502D1013E1C35F5E79F
:10622C002046394622F094F80028F6D12878013817
:10623C000528F2D80C980BF1010BC007EDD00B9888
:10624C005FFA8BF1C0B28142E7D356E0DDE90786F5
:10625C002EB338F8047C574518BF4F4503D1013E87
:10626C0008F12408F4E72046394622F071F800289A
:10627C00F5D198F8050001380528F0D898F80000F9
:10628C0001380228EBD30C980BF1010BC007E6D0B8
:10629C000B985FFA8BF1C0B28142E0D32DE05FEA3C
:1062AC000B6028D00B98000625D101205FFA8BF5E6
:1062BC000B90012D4FF001000C90A3D023F046FB66
:1062CC00C0B2B0FBF5F101FB15000B90012098E773
:1062DC00002038601E4989F80140A9F8025009785D
:1062EC0008F83610F4B1E8B1114962000DB0BDE800
:1062FC00F04F22F047BF4FF6FE770498069EDDF86C
:10630C00148047800A4FB37CF47CB269B1890125B3
:10631C00581EB07470895FFA88F68DE8D00003952A
:10632C0010F058FB0DB0BDE8F08F00BFDBBC0200D5
:10633C00F0850020407B0020E6BC0200D5BC0200AA
:10634C00DC5B0020B05400209ABC0200E027002047
:10635C00CE2700202DE9F04F87B005462C200E46A5
:10636C0023F05CFC002844D0778B044623F016F90C
:10637C000021E1840121874208BF02212170707B3A
:10638C00A0703169081A6060204618F087FB3178DC
:10639C00834F01F00301387B012908BF0520607091
:1063AC00C0B222F03FFF4FF0FF316077A182217F16
:1063BC00326908440A44317D3261081A3075E07044
:1063CC00A069013017D0207C032816D8DFE800F034
:1063DC0002170209062021466082284616F0A2FF09
:1063EC0010B3042021466082284607F0A5FB054621
:1063FC001BE01025CFE0A32517E0A12515E0002018
:10640C00B3256082F87A80B997F8410001280CD145
:10641C00A07D4FF6FF7619F039FE0025A082B04220
:10642C0008BF6FF05E0500E000252078022807D138
:10643C0004F1080622F0DEFB0146304623F099FBFE
:10644C00280640F0A580574F3878013801281AD813
:10645C0094F8260010B994F82700A0B1A078E17840
:10646C00227F08441044043023F0D8FB58B1A178A3
:10647C00E2780646207F114408446168021D3046CC
:10648C0022F080FE00E0002620460EF083F905463F
:10649C003878012802D12DB9002575E0022873D176
:1064AC00002D71D0002E73D00DF1080800274FF08D
:1064BC00010B4FF4D00908F1080A94F8260018B91A
:1064CC0094F8270000285FD0A178E278207F11444F
:1064DC0008443146021D606822F054FE94F82600F0
:1064EC0020B184F82670C4F8129007E094F82700C5
:1064FC0020B12D4884F82770C4F8120020460EF005
:10650C0049F910B10021054639E04046142122F02A
:10651C00D5FC608A8DF819B0F0B9A08A40F203114D
:10652C00884216D0682817D16068C17B052929D10B
:10653C002A30FF21082222F081FA18B34FF0FF30E5
:10654C006946CDE900001948006823F012FBFC20D5
:10655C0000E0FF208DF81800504669460022002507
:10656C0013F022F801469DF8000038B104201422E3
:10657C0043461FF01FFF0321002500E003210329E0
:10658C009BD101E00221FAE716B1304623F044FB1F
:10659C00204623F041FBE8B207B0BDE8F08F00BF06
:1065AC00407B00201826002000000301DC8700201F
:1065BC0014F04AF88848DFF824B2DFF824A2DFF898
:1065CC002482894D894E0027006817F07BFFDBF889
:1065DC0000004FF0FF310CF007F823F0B2F99AF8F5
:1065EC0002109AF80420D8F800409AF806308AF87D
:1065FC0002708AF804708AF80670002918BF44F0FB
:10660C000404002A18BF44F08004002B18BF44F087
:10661C000204C8F8004023F070FAD8F80000010614
:10662C0044BF20F08000C8F80000287818F008FA61
:10663C00002848D0DAF80C10044651B19AF8010041
:10664C00012804D0022804D1204688473BE020468C
:10665C008847204617F0E3FAA8B304460C20B1464D
:10666C002F4623F0DBFA80B1064623F06AF9054683
:10667C002078B46098B1304623F0CEFA606821F0EF
:10668C00EBFB204623F0C8FA16E0606821F0E4FB2F
:10669C00204623F0C1FA3D464E46002713E0D9F8B8
:1066AC000000314623F0D6F8D8F8000040F0100076
:1066BC00C8F8000023F09FF928463C464E460027B8
:1066CC0023F01BFA2546D8F80000C10631D53068F6
:1066DC0023F0BAF8F0B922F085FFD8B9A94623F017
:1066EC0030F90446306823F0A9F878B10546806883
:1066FC004188406817F046FCA868406821F0ACFB64
:10670C00A86823F089FA284623F086FA204623F05D
:10671C00F4F94D46306823F097F830B1D8F8000002
:10672C0020F01000C8F8000003E023F064F9D8F85A
:10673C00000081070FD508F00BFD21F0D3F820B134
:10674C0023F059F9D8F8000005E0D8F8000020F043
:10675C000200C8F80000010725D5706823F06EF818
:10676C0090B1DAF80810044641B19AF8000028B14B
:10677C00022826D0012804D1A0688847A0681AF006
:10678C002FFD204623F048FA706823F05DF830B1F5
:10679C00D8F8000020F00800C8F8000003E023F04F
:1067AC002AF9D8F8000041077FF511AF20F004005A
:1067BC00C8F80000306823F047F800287FF407AFD2
:1067CC0002E0A0688847DCE7D8F8000040F0100031
:1067DC00C8F800005846F7E6488800204C8800208E
:1067EC003425002050880020B98800202426002061
:1067FC002DE9F04F93B004461EF0C0FA08B11120F9
:10680C0006E1207F4FF6FE75B8B183480078810011
:10681C0041EA401061882077FF2020F043F90021E5
:10682C0080B1E08A05F1010B012640F00400E08202
:10683C00207F40F00100207707E0002000264FF673
:10684C00FE7B08E000264FF6FE7B74480078022899
:10685C0038BF012188010490678838461DF084F9FF
:10686C0008B10020607694F81AA0BAF1000F04D198
:10687C006B4890F800A084F81AA094F90000C5B2F7
:10688C00B0F1FF3F07DDE07E40B966480178E17664
:10689C000131017002E005F003052570207EDFF860
:1068AC008491012805D199F80B0010B90DB900207D
:1068BC002076DFF8688198F80000012831D899F823
:1068CC000E0080072DD5E6B1E08A410606D5BAF157
:1068DC00010F03D120F00400E08222E0A188E07EC9
:1068EC00627DADF822708DF82AA0ADF824108DF8D9
:1068FC002B0006A803F0E2FE00283FF480AF2578B9
:10690C000FE038461DF030F958B1002DDCD020696D
:10691C0000780A2805D8012101FA00F010F4836FE1
:10692C00D2D14FF6FE7A012D07D1206900780228CA
:10693C0003D1E08A40F04000E082EEBBE08A10F028
:10694C00400039D198F80000012835D899F80E008C
:10695C00800731D5049DA71D6188607E3A462B4681
:10696C0013F0B8FA28B100206076E08A40F02000DD
:10697C00E082387870B1618804F108001CF066FB85
:10698C0083466088834504BF00203870E08A40F05D
:10699C004000E0822078012804D0A18860882A4633
:1069AC000FF07CFCA18860882A460DF0B7F818B16E
:1069BC00E08A40F02000E0820DF11701204605F03E
:1069CC007DFA06461FFA8BF0504508BFB4F802B0AA
:1069DC00EEB12078617D94F82C50B9F816209DF812
:1069EC00173007948DF81800608DADF81A00E08A06
:1069FC0006ACCDE90254CDE900101FFA8BF13046FC
:106A0C000BF006F9102803D1304623F005F91020BD
:106A1C0013B0BDE8F08F00BFB3270020182600206C
:106A2C00CFBC0200407B00202DE9F04F99B012AF93
:106A3C008A4604461C219346384622F03FFA2046EB
:106A4C0039460CF0C5F99DF855009DF85C100843CB
:106A5C0007D09DF8480041060CD560891DF084F8DC
:106A6C0030B140F2351010F04EF919B0BDE8F08F8E
:106A7C009DF84800C0F3401900F00C0510F0200FF1
:106A8C0018BF042D21D1E08D9DF8483010F0800105
:106A9C000CD15A060AD59DF84920920706D143F02D
:106AAC00040202F00C020C2A40F0CA804FF00008DD
:106ABC00012213F003031ED0012B46D0022BD4D19C
:106ACC00A08912A91AF038FECFE7A68922F066FD3C
:106ADC00864202D1E08D010609D4A68922F05EFD22
:106AEC00864200F08B80E08D010600F18780000665
:106AFC0079D4A0897BE0544EF37A012B02D1A3798F
:106B0C00002B78D00223A7898DF84430ADF83C7067
:106B1C0081BB042D75D1207C4E4D8DF85E0028680C
:106B2C000028A2D022F03AFD87429ED1E08D217937
:106B3C0094F830202D684346CDE903028DE8020A13
:106B4C000FA812A95246A8478FE7002918BF0121A8
:106B5C0052EA010003D1A08912A914F00AFDA08900
:106B6C000797ADF81800A0798DF81A0006A819F04F
:106B7C009DF97AE7ADF8300016989DF84A109DF80B
:106B8C004B208DF8203094F832300B9060898DF8C2
:106B9C002310DDF84E108DF8222094F830208DF85B
:106BAC003830ADF81800B08CCDF826109DF85C107C
:106BBC008DF83720ADF82400207CADF82A10A17C8C
:106BCC008DF8320020798DF834109DF85F108DF817
:106BDC0033009DF85D008DF836108DF8350006A851
:106BEC0001F0E8FF41E7A089ADF86200608912A9C5
:106BFC001EF0DEF910B14FF49A7034E74FF0010932
:106C0C0041E71AB912A9384614F0B3FC10480078C1
:106C1C00022809D10D480078012805D1204611F031
:106C2C0033FB00283FF421AFA07CE17CB28C5346AF
:106C3C008DE8020A039012A80FA90EF0C3FF14E707
:106C4C004FF00108002234E7407B0020D5270020BC
:106C5C00182600203C2400202DE9F04F97B0044664
:106C6C0080690DF15B0200214FF0000890F800B034
:106C7C009C200BF09BF97B480078012808D8002059
:106C8C0004211CF0E5FE80469DF85B00404400E0CA
:106C9C000120C1B200258DF85B0059457DD9A0EBD0
:106CAC000B060221F0B2022828BF0E461A207043B0
:106CBC00C0B222F0B3FF0027002800F0BF80099477
:106CCC000BA907965FFA86FACDF814805FFA88F65E
:106CDC000446D8464FF000090690CDF820B0043198
:106CEC000A915FFA89F050455DD25FFA88F0B042A4
:106CFC0056D21FF05BFD00284AD05B490546888CB4
:106D0C0039312080A01C22F034FF4FF60270A4F819
:106D1C00170028888DF82C706082ADF82E00A97AA7
:106D2C0061760BA812F010F9014604F10A00012952
:106D3C0003D10A9922F01DFF03E04FF0FF314160AF
:106D4C000160287948B1484991F83810013102287E
:106D5C00217612D80221012811E04348022190F833
:106D6C0038006175298800290A4618BF012222754E
:106D7C0018BF411E2176002008E00121032821754F
:106D8C0002D16775012001E001206075A0751A34ED
:106D9C0008F1010809F10109A3E7002600274DE0DD
:106DAC000598CBFA50F830480FAD4FF0020BAE1CE3
:106DBC0000F139075FFA89F050453AD25FFA88F151
:106DCC0087202A460BF0F2F8BDF8460039462080A1
:106DDC00A01C22F0CEFE04F10A00314622F0C9FEBE
:106DEC00BDF83C001F49204B012209F1010908F1B3
:106DFC00010860820978022938BF022293F83830E2
:106E0C006275A3F1010238BF4FF0FF3202294FF037
:106E1C000001227638BF012184F817B04900A17512
:106E2C00002818BF01209DF84E10207561761A3489
:106E3C00C0E7069FDDE908B4079E0025607CF1B22F
:106E4C009DF85B300022CDE90275CDE900B1A11CA3
:106E5C000AF01EFB17B1384622F0DEFE17B0BDE873
:106E6C00F08F00BF18260020407B00202DE9F04752
:106E7C008AB0DFF8C0810446D8F80000416E02A841
:106E8C008847DFF8B4A1DAF80800016C096811B979
:106E9C00D0F84C058047694801210170DAF80C00E4
:106EAC00C068007830B9DAF808000021D0F858240E
:106EBC000120904722F0FFFC476805893878C0F321
:106ECC00401128460FF040FADFF874910790D9F87A
:106EDC00101019B122F0EFFC0C308847D9F80800DB
:106EEC0008B18047089057480078F0B1D9F82010C5
:106EFC00B9B1884755490028554B0A4608BF02329C
:106F0C0012781A708DF82420CA1C002818BF4A1C4D
:106F1C0010788DF825004C481978022908BF0230EA
:106F2C0000E0494801880131018016F05FF84A48B9
:106F3C00484E0078F57350B122F0BDFC007D30B1A5
:106F4C00284621F047FF1FF0EBF800286BD00025F6
:106F5C003761758022F0ECFA07467580059524B1EF
:106F6C00012C31D13D483E49C1613C483949027B35
:106F7C00437BC47D416045804D6002F0F00202739A
:106F8C0003F0F0020232427304F0F0020432C275D4
:106F9C004A7B22F00F02531C4B73DAF808301B6C3F
:106FAC001C6864682478A40608D52E4C42F00202B2
:106FBC004C601B685B689B784A73A3732A4E7060A5
:106FCC00707B00F0F00070732848D8F8001008228D
:106FDC00274B0C6D00210068CDE9002102AA314637
:106FEC00A0472449B0F1FF3F088007DD224819492A
:106FFC000160224801780131017010E0D9F800409D
:10700C0044B1DAF80800002100220023006C00686B
:10701C000C30A047012041F2883114F043F9384676
:10702C0022F032FD02E0E1200BF050FB0AB0BDE88B
:10703C00F08700BF308800200C010020A32700201F
:10704C0024B802001C25002094860020A68700206E
:10705C00A6880020A885002090270020A08300206F
:10706C00006A18003086002074250020D8260020E5
:10707C00E99200008A880020202500201925002094
:10708C00B0B5784C20780E2850D8DFE800F0E34FEC
:10709C004F5E084F4F4F4F4F584F0808080073482A
:1070AC000078B0B1A078012830D1E0780130E070E0
:1070BC00C0B2032851D870484FF6FF71808C8842BB
:1070CC004FD06C48012101704FF44170A4F80100BD
:1070DC0049E06C480021E170017000201CF0B0FE0A
:1070EC0018B120780D38012862D861480078022840
:1070FC0003D10820012104F009FC052020F0F2FC4A
:10710C0042F21070BDE8B04020F092B803282AD1AA
:10711C0057480078022826D15648012101700320D7
:10712C000021A070544880F826101CE015F0F6FEE3
:10713C00554810210078BDE8B04016F083BF4A488E
:10714C00008800F007000128A9D148480078F8B160
:10715C000020BDE8B0401AF013BB48480078012865
:10716C0001D10020A07019F07FFE20F07BFB3E487F
:10717C008078000703D54248007801286AD1A078AE
:10718C00032867D108200121BDE8B04004F0BEBB44
:10719C003D481021007816F055FF00201CF050FEE1
:1071AC00334D297810B361B3207801292AD036E009
:1071BC00062020F097FC2C4CA078000704D54FF447
:1071CC000040012104F0A2FB29480078012809D8CD
:1071DC00208800F00700022804D0002000210022A3
:1071EC0021F078FFBDE8B04015F098BE022903D11C
:1071FC000820012104F08AFB052020F073FC0120FB
:10720C00A7E720780A280AD11748008800F0070061
:10721C00022813D01848082180F826100EE0032805
:10722C000CD115F07BFE19480078022806D10120FC
:10723C001FF04CFC02200121FDF7A6FA062020F0DD
:10724C0051FC2878012805D80748008800F0070071
:10725C00022800D1B0BD002000210022BDE8B040C2
:10726C0021F038BFC426002026870020BB880020D0
:10727C00182600209E880020407B00209388002048
:10728C00BA270020AE220020998800200888002010
:10729C002DE9F04F93B01C9C08901D4606928B462E
:1072AC0020461EF035FB074620461EF019FB002633
:1072BC000790002F00F0E780002D18BF01254FF03C
:1072CC000008680100F14001BBF1000F08BF690123
:1072DC0005914FF6FE754FF00A0108BF0821049185
:1072EC0009A90431019100F108010C3003910290BD
:1072FC00207C804580F0C280380600F0BF8004EB13
:10730C00C80B9BF81C00C00740F0B28060480078A6
:10731C00012802D89BF81600D8B34FF0000A9BF84E
:10732C0016000F96CDE90D6678B15A49BBF81800D6
:10733C0091F86810012923D1FF21ADF8340003988E
:10734C0041F208098BF81A103EE0BBF81800A8426D
:10735C0036D104208DF824009BF81D00ADF83000C8
:10736C0009A818F0CBFD089C0198002100220023ED
:10737C00ADF83450A58016F055FFDDE9049024E0FB
:10738C00089C4FF00C09A080681CADF834000298E2
:10739C001BE0BBF8180022F01AFB0028BDD00079C6
:1073AC0040F002000328B8D19BF81C0040F080008C
:1073BC008BF81C00079800065DD04FF0010AAEE771
:1073CC00ADF83400DDE90490089C8DF836000120FE
:1073DC008DF83900207D8DF838000DA808F0F0F8F4
:1073EC009DF8480078BB109806994176417DA0F82D
:1073FC0016908BF81B109BF8161019B1254991F8B3
:10740C00681001771C9A51890185518A4185117D3B
:10741C0080F82C10517980F83A109BF81A1080F8EB
:10742C003B102189A0F84010617D80F849106268FA
:10743C002169C263406C227D21F0A4FE0DA81BF0D3
:10744C0057F89DF848009BF81C1041F001028BF88E
:10745C001C2020B141F009008BF81C0004E00798B7
:10746C00013FA0EB0A0007901C9C4FF6FE7500260E
:10747C0008F101083CE700200790F9E720460021BD
:10748C0017F00EF90646304613B0BDE8F08F00BF7A
:10749C0018260020407B0020BFB581780446481E8A
:1074AC000B2812D8DFE800F006525C6A267885902B
:1074BC00A430B23900208DF80400E0780F28C0F019
:1074CC00B28002208DF80400B3E0FF2940F0D38095
:1074DC000025E01C04218DF803501FF019F86C49AD
:1074EC0008606C48058011F083FE0DF103036F20DA
:1074FC00FF21BDE000208DF80800E07802F0AAF82A
:10750C0002AB6F200521B3E020F02CFB8DF80E00B0
:10751C000DF10E036F200A21AAE000208DF80F0058
:10752C00E01C22F077FB0546601D04211EF0F0FFE5
:10753C00014628460DF0CCF8504A3520282122F07F
:10754C005FF90DF10F036F200C2191E000208DF8F5
:10755C000600E0780F2870D302208DF8060072E048
:10756C00E07847490DF10703002818BF0120087087
:10757C00002003218DF807006F2079E0E2780020CD
:10758C00211D8DF80A0004F10C00022A68D0012A92
:10759C006AD117F0E3FE65E000208DF80C00E0786E
:1075AC00002818BF012020F055FE03AB6F200621E8
:1075BC005EE0E078211D19F0DBFA8DF80D000DF17D
:1075CC000D036F20072153E00020E57804218DF88E
:1075DC000900201D1EF09CFF002D014618BF01253F
:1075EC00284621F0D9FB0DF109036F2008213FE05B
:1075FC0000208DF80B00E078002818BF012022F045
:10760C00B7F80DF10B036F20092131E000208DF844
:10761C000500E07804281BD21B4A01211070512070
:10762C0022F0EEF817E0194A01211070522022F0D6
:10763C00E7F801AB6F2001211AE0124A012110700A
:10764C00532022F0DDF80DF106036F2002210FE02C
:10765C0002208DF805000DF105036F200B2107E0CA
:10766C000BF0A6F88DF80A000DF10A036F20042127
:10767C0001221AF0FDFF002004B0B0BDF082002002
:10768C00AE270020C2270020CC270020C8270020CE
:10769C00082500200425002070B590B004468078A1
:1076AC0021F0E2F8002800F0D38005466078A0F1C4
:1076BC00E101E873102906D91A2818BFCD2808D083
:1076CC001D2806D04BE0012202FA01F16C4A11424E
:1076DC00F2D06C4E3078012802D8688900056CD441
:1076EC002846002108F0BEFBC0B3307801282BD807
:1076FC006548807B800727D52968086A20B3C97F35
:10770C0003AA09F0D5FC6078E92808D12868E27B47
:10771C000123418900880093E92301F077F8286858
:10772C00BDF8161001809DF81120BDF81810BDF899
:10773C001600002A18BF012292010CF0EFF918B1C3
:10774C00688940F0200068816A896178288920F076
:10775C00A9FA28813078012831D971E060788DF848
:10776C001000A07B03958DF81100287C00283ED0DA
:10777C0003A812F06FFE9DF81030E92B00D03BB936
:10778C002868E27B012641890088009601F03EF8CA
:10779C003C480078012853D83B48807B80074FD564
:1077AC00687B022802D1688940073BD46078E928BD
:1077BC0046D128461BF03CFA42E0052068736078FD
:1077CC00E9283DD03148006800B18047304E306820
:1077DC00B0B32D48807B800732D52868418900885A
:1077EC001BF022FF60B361783268904728E003A851
:1077FC0005F0EEFD2348007820B19DF810300128EB
:10780C0002D0BAE79DF81030002BB6D1286800885A
:10781C001CF0AAF90028AED11C4800680028AAD098
:10782C008047A8E7286800881CF09EF9002811BF43
:10783C00032028684FF6FF71018008BF052068738C
:10784C00687B022804BF06206873A07812F002FD42
:10785C001FF028FB0B48007802280ED10D48007849
:10786C0058B900200DF10B018DF80B0052201AF0C5
:10787C00FFFB2020012104F049F810B070BD00BFBF
:10788C000101010018260020407B00207C230020F1
:10789C0080230020D52700202DE9F04F8BB0846980
:1078AC0006462588B4F8029028461CF05DF901289C
:1078BC000DD1307C717C00228023CDE90052CDE9C2
:1078CC000220B21C48F2060017F0F0FCD4E0284667
:1078DC001CF04AF920B96B480088854240F0C780FB
:1078EC0008962679651D5EB1700022F097F938B1C3
:1078FC000246304629460A9221F036FB054602E044
:10790C00002000260A9015F8017B57B1780022F070
:10791C0085F930B1024638462946099221F024FBFC
:10792C0002E0002000270990B8191421DFF85CB19F
:10793C004FF6FF754FF0000801EB4000C0B2079006
:10794C007800069070000590DBF800B0BBF1000FDA
:10795C0069D0DBF8040001780029F5D09BF80E20E3
:10796C00D207F1D0DBF808401CB10120A0478246B9
:10797C0001E0D0F808A0BAF1000FE5D0BAF8020087
:10798C00814518BFA94526D1DAF808309AF80720A6
:10799C000A9930461EF0D4F840B9DAF810309AF84B
:1079AC000C20099938461EF0CBF8A0B107981FF0AF
:1079BC0055FB38B30546D2202870089840882F73A1
:1079CC002E7168804EB10A99059A05F11400A860D1
:1079DC0021F0D8FB03E014BBB6E70020A86047B148
:1079EC0005EB46000999069A1430286121F0CAFB70
:1079FC0001E000202861DBF804002946406800788B
:107A0C0017F04CFB9AF80000214A5FFA88F108F154
:107A1C000108002C4FF6FF7550543FF495AF5046BB
:107A2C0022F0FAF890E7089C0A9D5FEA086011D0F2
:107A3C0014485FFA88F3227C617C0088CDE900034E
:107A4C0013480023CDE90202A21C48F2060017F0ED
:107A5C002DFC01E0207B90B115B1284622F0DCF81A
:107A6C00099848B10BB0BDE8F04F22F0D5B80648E4
:107A7C00007802283FF41DAF0BB0BDE8F08F4FF03B
:107A8C000008D5E7708700201826002020880020E9
:107A9C00148100202DE9F04788B004464FF0FF30E8
:107AAC0002214FF6FE79CDE90200E089002808BFDB
:107ABC000821A66916F801A030B1714835880088F4
:107ACC00854213D16F4E06E06E4831461FF0E7FD3C
:107ADC0090B36B4805884D4518BF002E29D1207BEB
:107AEC00002840F0C9806948406843E06648007847
:107AFC0001281CD8284621F06AFFC0B10179002664
:107B0C0001292DD140880DF110088DF81060ADF8C9
:107B1C001C00404618F0F2F90646002818BF08F180
:107B2C000406BAF1000F18BF4FF0FF3AD3E7002656
:107B3C0016E05648406825E05348007801280DD8D7
:107B4C00304621F098FF48B101790139012905D857
:107B5C00BAF1000F18BF4FF0FF3ABBE74FF6FE75B6
:107B6C00207B002840F08880484840684D4518BF6D
:107B7C00002E07D1E1894FF0810881B100F8018B0B
:107B8C0002AE11E05FFA8AF1022902D24FF000082E
:107B9C0007E0217B01296FD04FF0800801E009F14B
:107BAC00010500F8018B0EB1314600E002A921F06D
:107BBC00E0FF0570064605803348007838B10B2786
:107BCC0001284BD15FFA8AF0012804D046E05FFA15
:107BDC008AF0012824D10B27B8F1000F3ED1284898
:107BEC00A9B20088814239D100250DF107008DF82A
:107BFC00075016F0E3FDA8B1E1890322002908BF64
:107C0C000922A1698B5C9DF8072000EB43019A4285
:107C1C000BD9D21A0D258DF8072005EB420708E089
:107C2C000B271BE00C27B57018E000220D278DF8F0
:107C3C000720F370331DB27012060DD011F8022B11
:107C4C0003F8022B11F8012C03F8012C9DF80720E6
:107C5C00013A8DF80720EFE721F0DEFFE2890B4DAA
:107C6C001020A11CFBB2A87004F1110042F40042D8
:107C7C0017F0CCFB0020A87008B0BDE8F08700BF5F
:107C8C0070870020C8870020182600207C26002042
:107C9C002DE9F04F8BB0002900F0EA80DDF858A0F8
:107CAC000746007A0D46994690465FEA0A718DF8B0
:107CBC00060012D4387A02240F2800F2DA8001214F
:107CCC00814011F00B0F19D003288DF8100024D12E
:107CDC0002A8394621F04DFF22E0022840F0C8806E
:107CEC003C8821F05BFC8442E4D0388801210322DB
:107CFC0013F0E8F90028DDD0CD24BAE048F20400F6
:107D0C00014200F0B68038881BF02EFF002800F0EE
:107D1C00AB800F2038728DF810003888ADF8080051
:107D2C005FEA8A7014D40020ADF81800534800683C
:107D3C0088B14168A942FAD1826862B129780220DF
:107D4C00904768B10188ADF8181021F065FF07E085
:107D5C004FF6FF7002E0A86810B14088ADF818002B
:107D6C00CAF380129DF810301798DDE9141B8DF8BA
:107D7C00052010225C1E02EADA0218BF01240F2B28
:107D8C00134618BF43EA84035FEACA6458BF13461C
:107D9C000AF0400243EA92125FEA4A73ADF82020DF
:107DAC0044BF4032ADF820208DF824000791ADF887
:107DBC001A90ADF8168000229BF800007C7A7E8920
:107DCC005FEA8A618DF804202D498DF8220028780D
:107DDC008DF81340ADF8146009788DF8120048BF87
:107DEC0004218DF8231020F003FD28B1016919B18D
:107DFC0002A888477C7A7E893046214621F070FCA7
:107E0C0028B120F0CFFE48450DD2022413E001A882
:107E1C0020F0A4FF48450AD21A4801680029F4D082
:107E2C0002A8884706E002A806F0D8FB02E002A8E8
:107E3C0000F0C0FE04469DF8100002280CD1BDF8DD
:107E4C00086021F0ABFB864206D19BF80010287825
:107E5C00424623461BF0F8FA5CB99BF8000000245C
:107E6C0001308BF8000004E0387A0F287FF42CAF37
:107E7C00022420460BB0BDE8F08F00BF2088002004
:107E8C00E71D0020F42600202DE9F04F8DB00746A9
:107E9C00C08914468946073086B2304610F084FA01
:107EAC000546FF280AD13046FAF73EFCB04205DA07
:107EBC0070480778002F08BF0527A3E06D4E307877
:107ECC00C0B91CB1022C15D1FF2D13D1387A002268
:107EDC0003238DF81C007868009206906648C188D0
:107EEC00C07805AA02F054FA9DF824003874BDF845
:107EFC002000B881DFF880B1002104239BF80340F7
:107F0C00BBF806A00CAA204621F004F99DF830001D
:107F1C007E2805D120467C211CF0A2FB9DF8300068
:107F2C007C286BD1FD8905F107081AFA88F0B0F5A9
:107F3C00005F65D8BB88C5F385120490F888494664
:107F4C001FFA88F94FEA850C8DF82DC042EA83128E
:107F5C008DF82A00C0F301208DF82C209A088DF89A
:107F6C002B203A7A05EB0A07B9F10D0F40EA820093
:107F7C008DF829004AD23F482A460197CDF80CC00B
:107F8C0000F11C06304621F0B5FEDDF82900711910
:107F9C0000220027029170519DF82D000871681D78
:107FAC0081B2304621F024FBDDF8291032464B46D5
:107FBC00715196212F4D8DF82F10039921F0E1F975
:107FCC0002998DF82E000B98C1F8030020465146FB
:107FDC001BF056FE04EB4401049A28700BEB810154
:107FEC008A83BBF806104144ABF8061050B10198D7
:107FFC0081B2204618F0A8FB2F7803E0012700E09F
:10800C000527377038460DB0BDE8F08F8946084615
:10801C002946002221F0ECFA0DF12901052220F06D
:10802C0035F996214A462B468DF82F109DF82D10C8
:10803C0021F0A7F951468DF82E0020461BF020FEAA
:10804C003070B9B220460DF1290207231BF018FE3F
:10805C00317851EA00073770D4D104EB440004990D
:10806C0000270BEB80008183BBF806004044ABF883
:10807C000600C7E7A0230020A08000202DE9FC47C4
:10808C00D0E900588246D8F80000D0F8409019F496
:10809C00F06FC0F8449035D05FEA495117D5D5E957
:1080AC001401411A50461DF0F1FED8F80000816908
:1080BC00C90605D401688DF807109DF80710F6E77E
:1080CC00296801312960A97B09B90121A973696C5F
:1080DC0040684FF0004600F00F0404EA0100B0FACB
:1080EC0080F126FA01F1014005D02F6C1FB12A68EE
:1080FC00AB6C5046B847B4FA84F026FA00F0204036
:10810C004042A863D5F85801D8F83C1009F0400754
:10811C0040680068D0F804251140394347D0DAE9AB
:10812C000064504614F0C6FED7B1F07C90B90BE059
:10813C00316F69B10068B16EB26F8854306FB16F36
:10814C0001310138B167306720688169C906EFD504
:10815C00F07C28B1D6E91401411A50461DF096FE68
:10816C0096F86400E0B13079022819D017B1B179D2
:10817C00012901D0316F99B90024B16E01283467FF
:10818C0086F86440B46607D1B36CB26FD6F8CC6095
:10819C0050460094B04703E006F17C0021F050FDFE
:1081AC00504609F0E5FAD5F858014068006800F22D
:1081BC0004500068D8F83810084228D0D5F8F800D8
:1081CC0028B3DAE90076504611F0C4FE50460CF0A4
:1081DC001DFD7879012812D1D7F8F40078B997F8F9
:1081EC00E80060B1002087F8E800BB6CD7F8EC1011
:1081FC00D7F8FC20D7F8504100905046A047D7F84C
:10820C00F80020B93068816B41F4006181635FEA4A
:10821C00095023D5D8F8000081690907FCD4016BFB
:10822C0021F480710163297A91B10020287295F8AC
:10823C004400800606D52C6C24B1AB6C5046202132
:10824C000022A047504601211EF0A1F9D8F80000E9
:10825C00816B21F400618163687908B1BDE8FC870A
:10826C0005F58070BDE8FC4721F0EABC2DE9FE4F16
:10827C001D4614460F46814621F05AF9DFF8C0A17D
:10828C0083464FF6FD78DAE90010494518BF0846D9
:10829C0060B1B83021F098FC40B19AF82400CAF8CB
:1082AC00209040F004008AF824009FE01FF0AAFB05
:1082BC00002868D006466348CDF808B0DDE90CB854
:1082CC0021F0DCFB604908F0200EB1F854000130BD
:1082DC006FF31F30A1F85400B5605C480025C6E967
:1082EC0003792268D4F80C8086F83250C6E9085518
:1082FC000BEA000C207C72632279C6E906CEC6F824
:10830C00408086F8440086F83820B1F8541086F87E
:10831C003350D4E905533186A168C6E91253F16391
:10832C00A18BA6F8501028B9B8F1000F1CBF012082
:10833C0086F844004AB9387B00F00F00022804D1BB
:10834C00012086F83800B8687063DDF808B00822A0
:10835C00FF2353FA82F23C46D0B2851A18BF01258E
:10836C007F680FB1002DF4D1208800F47C40B0F56B
:10837C00305F0BD196F833000022082340F0100038
:10838C0086F8330004E008F101082FE000220223F4
:10839C004CEA03004EEA02012B4DC6E90601DAF85D
:1083AC002000484507D19AF82400C1071CBF00F0F3
:1083BC00FE008AF824002648046854B1A96CEA6CC3
:1083CC0005F1400005F1380300903046A04703301A
:1083DC0013D1FD209AF82410CAF820904FFA80F897
:1083EC0041F004018AF8241020F0ACFE584621F02C
:1083FC004BFB0FFA88F0BDE8FE8FB6F83080B5F86D
:10840C005410414501D020F09DFEC0B2012801D886
:10841C00FE20DFE7002089F8FC0096F8330040F0DE
:10842C00800086F83300A86BB04205D0F068007B62
:10843C0000F00F000228D9D115F0D2F8D6E700BF12
:10844C0070200020207F002030210020FFEFFF9FB4
:10845C00842600202DE9FF41DFF8BC810020039029
:10846C000290D8F83840B4B3D8F84C0010B9D8F80A
:10847C00480070B3D8F8480060B12069D8F84810AB
:10848C000969814206D194F83300C00602D5D8F8A8
:10849C004C0090B1002702A887F0010103AA10F04C
:1084AC001FFE0546FFB9F5B10299002900F09D8029
:1084BC005A4820F031F9002714E0D8F84800C06879
:1084CC0040880028F9D0D8F84800C06840880128B6
:1084DC00F3D00127DFE752480221283021F0B4FB0A
:1084EC000027002500242CB34E48466816B302988A
:1084FC00B0FA80F04009284001281BD1D8F8480078
:10850C00D8F84C10039A87F00103CDE9003208F13A
:10851C00380208F14003B047012868D0022809D17D
:10852C00D8F84800012201230069D8F84810B1F9A5
:10853C00301065E02046002C18BF0120384001287F
:10854C0051D1394821694068814203D034484FF4F5
:10855C00806145E00298002818BF012028400128BE
:10856C0006D1D8F8480018B9D8F84C0000284DD0DE
:10857C0008201FF08FFD94F833004C25C00658BF1F
:10858C00482508F138001FF013F848F80500274B70
:10859C00D4E90601C2439A60DA681043D860C84334
:1085AC00186058680843214658600820E5681FF099
:1085BC0049FA28461FF076F9288843F60601411A35
:1085CC00022906D3B0F5C15F03D040F60201884200
:1085DC0003D1012029461FF035FA11484FF0804194
:1085EC00283021F031FBBDE8FF8100277BE70398A1
:1085FC00002818BF0446B4F930102069012200236A
:10860C000092002206F03AFABDE8FF8108201CF027
:10861C00C3F8BDE8FF8100BF30210020647F00203B
:10862C007020002084260020D01E0020081004405A
:10863C002DE9F0478AB0684D2868416E02A888473A
:10864C00664FF87918B1B87908B10020C0E020F075
:10865C006FFFDFF88CA1804600249AF80000800799
:10866C004FF0000005D47D2000210DF06DFE8DF83B
:10867C0018408DF80C4002945A4C0790616911B166
:10868C009AF800008847E06808B180470890387A6B
:10869C0098B1606A88B180475349544B8A1D0028B1
:1086AC0018BF0A1D12781A708DF82420CA1D0028D4
:1086BC0018BF4A1D10788DF825004D4EDFF8349107
:1086CC0000200590317BF27EB0607080D9F80800F4
:1086DC0001F070018031317302F08001D0F8282450
:1086EC00F4206331F17603218DF8181006F11C018A
:1086FC009047387980B99AF8000080060CD5286824
:10870C00C06B8047317BB060029001F0F001023108
:10871C00317301218DF80C1029683748344E384BD1
:10872C000D6D4FF08071006801913449009102AADF
:10873C003146A84705463348B5F1FF3F058035DD86
:10874C00B879002100240130B87178790130787142
:10875C00FE60F8790130F871022012F0A3FD3C7133
:10876C002948D9F808200188D2F8AC30D2F8D420A6
:10877C001C7841EAC411D48C0180D2E9117193F8B0
:10878C0000C0538D7486C481C0F80710C0F8037004
:10879C008381508DC6E90A710CF001013086308B53
:1087AC0020F0800040EAC110308309E0626812B109
:1087BC00002000219047022041F2883112F072FD16
:1087CC00404621F061F90020B5F1FF3FC8BF012000
:1087DC000AB0BDE8F08700BF3088002014250020C7
:1087EC00AD88002024B80200A6870020A5880020B0
:1087FC00E87F00200C010020D82600202000430038
:10880C00C90E010088880020E88600202DE9F84375
:10881C00994617460C4680461AF006FF089D0646F8
:10882C003DB936B9404621463A46BDE8F84318F002
:10883C00F5BA6EB3002D3ED0624C207808B10128F9
:10884C0003D16148806800B18047B9F1000F4BD06B
:10885C002078012800F2A5805C48807B800740D5F9
:10886C005948C26812B13046494690475848317849
:10887C000078884224BF01313170C9B20024814292
:10888C0030D140461AF014F87470012701242EE000
:10889C004C4800240127B9F1000F007829D0012D94
:1088AC0027D1012825D84948807B800719D5404617
:1088BC0019F0FEFF15E0B078B9F1000F0AD1C1191B
:1088CC004808022938BF01207178B07011B94149AC
:1088DC000978717040490978884202D90027002430
:1088EC0005E00024012702E00027002437703548FA
:1088FC000078012D08BF02282BD084F001010F4213
:10890C004DD1012812D83148807B80070ED54046C6
:10891C0021F05DF850B11FB9417901F0FE014171B0
:10892C00ECB3417941F00101417100E0BCB3254C3D
:10893C002078012821D82548807B80071DD540460A
:10894C001FF012FEC8B100204146BDE8F84321F0EB
:10895C005BB9A9F119010229CFD3B9F1000F08D0E5
:10896C00B9F1E10F18BFB9F1F10FC6D0B9F1EB0FA6
:10897C001AD1154900220A70BFE71448408B4045B4
:10898C000DD10120414621F03FF92078022806D173
:10899C004FF400500121BDE8F84302F0B7BFBDE829
:1089AC00F88300240127A4E7074A0C4913780978B7
:1089BC000133DDB28D4228BF0023137028BF012480
:1089CC009BE700BF1826002074230020407B00206A
:1089DC00D1BC0200D0BC020093270020C627002087
:1089EC002DE9FE4FD0F80080994614460E4682467B
:1089FC0013B10020C9F8000020F09AFD834698F8C6
:108A0C00070038B198F8640048B121F04FF86FF0C6
:108A1C000805B3E021F04AF86FF00E05AEE0002C2B
:108A2C004AD0504614F046FA00200121C8E91A64D5
:108A3C00C8F87040C8F87800C8F8380088F80C00FE
:108A4C0088F80A00504688F864101BF0C1F95046AB
:108A5C0008F08EFE08F14C0402AD204629461EF0AB
:108A6C00C9FDD8F870100746D8F878008F4288BF37
:108A7C000F46029930443A4621F03CF920463946DB
:108A8C001DF030F8D8F87000D8F87810C01B3944B5
:108A9C00012FC8F87000C8F8781001DB0028DCD171
:108AAC0098F8041002290CD10020C8F8680088F846
:108ABC006400C8F870001BE020F0F8FF6FF00905A7
:108ACC005CE0A8B90020D8F86860012988F8640037
:108ADC00C8F868000CD10124584688F8104020F0E2
:108AEC00D3FF98F80F0000284BD020F021FD8346CF
:108AFC0020F0DCFF98F8040008B100252FE0D8F82E
:108B0C00701008F17C0031B30C9920F033FF10B1D8
:108B1C00012088F80C0020F00BFD0446504614F0A0
:108B2C00C9F90020C8F86800C8F8700088F864001B
:108B3C00504608F01DFE98F80A6098F80C50204634
:108B4C0020F0A2FF002D18BF6FF00C05002E18BFEF
:108B5C006FF00D0503E00021002520F00BFF20F045
:108B6C00E7FCB9F1000F07D098F8041001291CBFDD
:108B7C00D8F87810C9F8001020F086FF2846BDE818
:108B8C00FE8F002598F810000028AED020F0D0FC05
:108B9C00A8F80F4020F078FFD8F84830D8F87820A3
:108BAC00D8F8CC70504631460095B84788F80F502D
:108BBC00E8E77047F0B587B004466F48007878B1A5
:108BCC00228B0020E57A01210390CDE901008DF87C
:108BDC000910500706D402F008030121002008E018
:108BEC00BA20AAE0402012F008038DF8060008BF56
:108BFC000321402606EA82064BB1C02093068DF86D
:108C0C0006004FF0010358BF02238DF807305309BB
:108C1C0003EA121202F00802324342EA0106217AF8
:108C2C0003290AD8DFE801F00215112540F00407EA
:108C3C0020F0B4FC8DF8067008E00F291DD140F02F
:108C4C00080046F004068DF806002088ADF80400F4
:108C5C0013E04A4991F86810002900F080802788B9
:108C6C0040F0080006F58056FF258DF806003846C2
:108C7C007EE001A920461CF0B3F90027208BC00729
:108C8C000ED09DF8060010F00C0F58D09DF8060081
:108C9C0000F00C01042904BF40F020008DF8060000
:108CAC00A07C8DF8080001A806F08AFC9DF818003D
:108CBC00002842D10498C682B4F81B10A0F81910F1
:108CCC00217A012903D12D4991F868100177A17EF1
:108CDC00E37F0185228B80F82C301306428508D562
:108CEC00D20506D5417D94F820001DF0CEFCA17E66
:108CFC000498878780F83B5080F84A10A17A80F856
:108D0C003A10D4F80E10C0F83E10A17F80F84B102A
:108D1C00617F80F84910406C6169628A20F032FAF8
:108D2C00208B400604D51648016809B101A8884774
:108D3C0001A819F0DDFB9DF8180007B0F0BD2088E4
:108D4C0016F094FE48B19DF8060040F020008DF816
:108D5C000600208BC00799D1A2E7BB20EDE740F0BD
:108D6C000C00278846F004068DF806004FF6FD70BF
:108D7C00ADF8040082E700BF2C240020407B0020CB
:108D8C00602700202DE9F04F89B0714F14460A4638
:108D9C00064610460492B98C1AF046FC054610B1F2
:108DAC006878002866D0B06A4FF00E09B34690F888
:108DBC000180867890F805A05FEA886158BF4FF073
:108DCC000609B0F80300039004981AF0ADFF18F0F0
:108DDC00870F4CD108F01801182948D09BF81C10AB
:108DEC00894544D100EB0A020021BBF80C00B146C6
:108DFC000091D1B292460E46049B494632460EF083
:108E0C0051FD032836D008F07801B8BB18F0180FC4
:108E1C0062D05FEAC86088464FF0030058BF01205B
:108E2C0040EA0108BBF80C00414611F013F888B178
:108E3C00817911F0180F0DD0417901290AD14DB16A
:108E4C00B98C40881AF0F0FB20B1407810B16978E9
:108E5C0088420FD320F087FA88B94FF0FF3020807A
:108E6C009BF8080000286BD0DBF8181069E0D320C1
:108E7C000DF049FF002009B0BDE8F08F884620882E
:108E8C004FF6FF718842F5D10121BBF80C00324638
:108E9C0000914946049B0EF005FD0398414685B2AE
:108EAC00284618F075FAF98A88420CD1284620F029
:108EBC008EFD20B300790138012820D805A9284659
:108ECC001CF086FD21E0DBF8280080F805A009B035
:108EDC00BDE8F04F1EF096BC787B884608B120F0B8
:108EEC0042FA03984FF6FE710022434680B203F01B
:108EFC00EBFD0028C3D14FF6FF702080C4E71FF0B4
:108F0C0079FE014605A820F034FE9BF808000128E4
:108F1C0004D1DBF8181007A820F02BFEDBF8281082
:108F2C00BBF80C00497805AA07ABCDE9003200224A
:108F3C004B4641F030010291294608F0DDFE99E7DD
:108F4C000021BBF80C00324620F04CFE97E700BF26
:108F5C00407B002070B58AB000F116050446284607
:108F6C001AF0DEFF67480078013801282BD8002062
:108F7C001021012214238DF8110005AE0DF1110002
:108F8C00CDE90210CDE900620DF11201042000229E
:108F9C001BF04EF950B15C48006804A905AE32468E
:108FAC0010F002FBC728ADF812000CD806F108002F
:108FBC002946082220F0E6F8BDF8121004201422ED
:108FCC0033461DF0F7F92846FF2108221FF036FD25
:108FDC0010B14E480121017028461BF0ADFC2079E0
:108FEC000138052800F28B80DFE800F00389345C3F
:108FFC008903A01D0021102913D0425C0131002AE5
:10900C00F9D061791EF0F0F84348424D90F84100D8
:10901C0008B12878D8B160790DF066FF002028706F
:10902C0015E03D4890F8410088B905AC002062215C
:10903C000025224610F086FC204600211EF0D4F8B4
:10904C0000200DF051FFCDE90755CDE905551FF076
:10905C00BBF854E00DF1120128461DF0C2FA60B1C4
:10906C000DF112024FF6FE7029461CF093FF2846B4
:10907C0000210022002315F0D5F8BDF8126005A9D7
:10908C0030461CF0ADFA059828B905A81AF0A0F9DD
:10909C0008B905980680A11D284610F05BFD13F059
:1090AC00F5FC2CE01A4E307848B30DF1120105AAEC
:1090BC00284610F079FA01469DF81200F8B1002507
:1090CC0001201422ADF8240006958DF82650059544
:1090DC0005AB04201DF06EF906344FF4817010219D
:1090EC00224620F087FB28B94FF4817010212246CC
:1090FC0020F086FB01200321357018F065FB0AB0C7
:10910C0070BD00BF18260020DC8700209C88002042
:10911C00B0220020AF220020407B002070B58CB024
:10912C00044600208DF82C00CDE906000890A078AC
:10913C00411E052925D82220DFE801F00321212C2E
:10914C0023036248007820BB20F000FB40B9604D3F
:10915C00A168082205F1180020F014F82088288056
:10916C005C480078022814D1A0680DF1030101AA13
:10917C0010F01AFA9DF8140038B1B1206CE01B20E5
:10918C0008E0B3208DF82C0059E09DF8030000286E
:10919C00F3D023208DF81C000120A17B8DF81A0040
:1091AC0020888DF81D102169ADF81800607B08919E
:1091BC00012804BF21208DF81A0006A806F000FA39
:1091CC009DF82C00D8BB0998456C05202870A07818
:1091DC006870A81C616819B110221FF0D3FF04E05D
:1091EC000021C160816041600160A078062801D037
:1091FC00012803D1E078A874133500E01235A1687A
:10920C00284620F086F8A17805F1080006290AD82E
:10921C00012202FA01F111F0520F04D02E49096813
:10922C0020F0A7FC01E0217B017020881AF09CFC47
:10923C0010B109980421C1829DF82C0070B123480B
:10924C00007838B920F082FA20B921480021C0E911
:10925C00061101809DF82C000CB070BDA07804287C
:10926C0014D1A06801AD0DF103012A4610F09CF950
:10927C0006469DF8030018B94FF6FF708642DED003
:10928C00206968B106A80EF045F90CE0206918B108
:10929C0006A80EF03FF9D2E706A819F029F9CEE797
:1092AC0006A819F025F9A16805F1080008221FF09D
:1092BC0069FF0120314614222B46ADF81400002022
:1092CC00CDE9010004201DF075F8B8E71826002040
:1092DC0050240020AC270020DC870020F8B5634E1A
:1092EC0001211D461446F068C068017060480021D9
:1092FC00017060480170B068016C096811B9D0F850
:10930C004C0580475C48076847B15C4822462B46B1
:10931C004188B068006C00680C30B84715F0E24F1B
:10932C0014D057480178013901705448406818B17D
:10933C005448C1890131C181B068006C0068406833
:10934C00007880066FD41CF0B1FF6FE020070CD4BE
:10935C004A48406818B14B48C1890131C18148481D
:10936C000178013901701D205EE0454C42F2054246
:10937C002078013820704448418841F00400904224
:10938C0018D13E48406818B13E48C2890132C281AA
:10939C003C4842890132428142F20542E12091422D
:1093AC0008BF1C2009F092F9207800284AD094F9C3
:1093BC00000040E0314842F606024188914212D04A
:1093CC00B1F5105F49D140693349086019F010FCC0
:1093DC002E48007850B32F480168013138BF016026
:1093EC000021018122E0406818B12648C189013171
:1093FC00C18126480078C8B125480421007802288C
:10940C00204808BF0621425A013242522148416885
:10941C00013138BF41600189428901318BB2018130
:10942C00934288BF4181E92009F050F91448017832
:10943C0041B190F9000000280ADCB068D0F84C0566
:10944C00804705E0B0680021D0F8582400209047F0
:10945C00F0680021C0680170F8BD406800283FF436
:10946C0082AF0848C1890131C1817CE70C01002021
:10947C0017250020A327002024B80200A88500206F
:10948C001925002094860020A08300201C25002094
:10949C00A68800204C87002044880020FEB5044696
:1094AC002C2020F0BBFB002820614BD02C211FF07E
:1094BC0005FD256920884FF6FF760DF10301AE827C
:1094CC0011F0A8FB48B30DF1030069461EF0CCFF68
:1094DC00BDF80020B24220D0584902EB4200AA82CB
:1094EC0006226A82002251F820302A744FF47A72D4
:1094FC00AB6151F820300133B3FBF2F541F8203069
:10950C0005FB12324AB901EB8000012101724C4873
:10951C004FF40061007814F095FD21692088083122
:10952C0011F078FB1FF076FD256970B14FF4D00077
:10953C00C5F812000220287442480168A961013163
:10954C00016021E010202075FEBDA88AB0421BD11D
:10955C003D4F05F1080039681EF0A1F858B93D6877
:10956C001FF048FB014628461EF099F818B91FF069
:10957C0051FD00285FD02169208802F0EDFB2569A0
:10958C0000B1AE8200202874A88AB04231D12F4895
:10959C00C17A11BB90F8410001281ED10DF10B02CC
:1095AC00002001213A2301271EF004FD08B1AE82F0
:1095BC0013E09DF80B002F74A8754FF46810C5F8D4
:1095CC001200234801684A1CA961026029B91C4891
:1095DC004FF40071007814F035FD2569A88AB0426B
:1095EC0007D1A1202075284620F016FB0020206111
:1095FC00FEBD287C012801D10E210CE0A06808B129
:10960C000D2108E01FF006FD0D2118B9A078C00748
:10961C0008BF052125690D482977A17801F00301C0
:10962C00007B012908BF05206870C0B21FF0FAFD4D
:10963C0021694877FEBD2569A6E700BF1883002085
:10964C0099880020FC260020DC870020407B00202D
:10965C0008250020F0B587B0624C054694F82B0025
:10966C0028B9614F0421387819F0A4FD30B35F4854
:10967C00407808BB5E480078022803D194F82B0090
:10968C00800619D494F82E0005F0C60668B1A80718
:10969C000BD594F82B00C00607D41EF00AFC04204E
:1096AC000121FBF771F886F0020694F82B1006F0F6
:1096BC003F00084384F82B0007B0F0BD94F82B0052
:1096CC0005F006062178304384F82B0051B1E0B345
:1096DC004648002101703878042107B0BDE8F040FD
:1096EC0014F0B0BC012004F12E03002101222070E3
:1096FC0055201FF0C9FB94F82E0080B33C4800782D
:10970C000138012809D83B4D0021082228681FF098
:10971C0095F910B91FF07EFC20B334480721017075
:10972C0094F82B000021304340F0100084F82B00FB
:10973C00002005F07BF80028BED000201DF0C6F9F3
:10974C0007200021FBF720F8B6E728480721017015
:10975C000720002107B0BDE8F040FBF715B894F8DE
:10976C002B00B4E728680DF11B0101AA0FF01CFFB8
:10977C000546214800780028CFD09DF81400FD281C
:10978C00CBD00228C9D01D480088854217D201AE23
:10979C00142130461FF092FBFF2029461422334639
:1097AC008DF8140004201CF005FE154905EB45004E
:1097BC00002241F8202001EB80004272426000251B
:1097CC005520012104F82E5F224620F019F8FF20C5
:1097DC0003211AF073F8054804210570387814F049
:1097EC0031FC69E7AC2200209F880020088800200B
:1097FC0018260020DC870020AA270020C6BC020007
:10980C00804300202DE9F04788B00646109C0020CC
:10981C00DD099A461746C3F3C308E060A060606098
:10982C002060E9B1E9462146102248461FF0AAFC07
:10983C002046314610221FF0A5FC484620F039F98D
:10984C000020102805D0315C225C5140215401309D
:10985C00F7E70AF1800A1FFA8AF04FEA102901E0B3
:10986C004FEA1A296E46280418D030462146102299
:10987C00013D1FF087FC2046394610221FF082FC68
:10988C00304620F016F90020102805D0395C225CF7
:10989C00514021540130F7E70744E4E7B8F1000FD9
:1098AC0025D06846214610221FF06CFCB8F10E0F33
:1098BC0040D30025204639464246E560A5606560E8
:1098CC0025601FF05FFC80202146102204F8080060
:1098DC0004AE30461FF056FC684620F0EAF8102D16
:1098EC0048D0705D615D484060550135F7E76E46C4
:1098FC002146102230461FF045FC002780201FF027
:10990C00EEFF21461022C4F80170C4F80570C4F8AB
:10991C0009706773207004AD28461FF033FC304685
:10992C0020F0C7F8102F42D0E85DE15D4840E055CB
:10993C000137F7E70026204639464246A681A66045
:10994C00666026601FF01EFC80202146102204F861
:10995C0008001FF0C4FF04AD28461FF013FC684636
:10996C0020F0A7F8102E22D0A85DA15D4840A0558C
:10997C000136F7E76F462146102238461FF002FCED
:10998C0000253046214610221FF0A9FF2560656096
:10999C00A560A5811FF0F6FB384620F08AF8102D43
:1099AC0005D0705D615D484060550135F7E708B042
:1099BC00BDE8F0872DE9F84FD0E90158D8F8001030
:1099CC00CA690A62D20740F0A480D8E9040105F103
:1099DC00C8094FF0000A4FF0000B0843D5F8CC1023
:1099EC0049680968C1F8040505F130000090BBF125
:1099FC00010F00F29780D5F8C000002800F092808B
:109A0C00D5F8E0C0D5F8CC70DC2224232024BCF19E
:109A1C00000F08BFD82208BF1C2358F8033008BF1A
:109A2C0018247F68D8F8146058F804403F68D7F8B9
:109A3C000415314211D0A16849070ED10168D5F83F
:109A4C00D0408C4209D1416939B9D8F800104C6A20
:109A5C0024F002044C62C7F804659968490702D0E7
:109A6C000BF1010BC3E7AB58002BF9D045F802A062
:109A7C00D5E934121A44BCFA8CF35B09C5F8D4202E
:109A8C005B01C5F8E0300368994228BF9A420CD2BA
:109A9C002846414602F0AAF895F8FE000028DFD0CF
:109AAC001FF0BCF818BF8862DAE7D9F800204B46E3
:109ABC0080F810A02AB153690BB11A46FBE702F1EA
:109ACC0014031860C5F8D4A0BCF1000F4169C0F8AC
:109ADC0014A04FF0D800C5F8C01008BFDC202858DF
:109AEC00C5F8D00059B12846414602F07FF895F8E8
:109AFC00FE0050B11FF092F818BF886205E0D8F84C
:109B0C000000416A21F003014162009820F09EF8A8
:109B1C00A6E7D5F8C0203AB103211174BDE8F84F7F
:109B2C000EF068BBBDE8F88F486820F00200486072
:109B3C00486A20F003004862D8E904021043D5F8C3
:109B4C00CC2052681268D062C2F80405486920F033
:109B5C0001004861012008624046BDE8F84F1DF045
:109B6C007BB970472DE9F04F8BB0DFF8A08104462C
:109B7C00D8F80800D0F80001807AC00020F04EF828
:109B8C000028099000F0B5804FF000091FF0D0FCC0
:109B9C00009001AEFF270025D8F80800EAB2D0F8F3
:109BAC000011CB7A9A422CD2D0F88824D02031469E
:109BBC008DF80650ADF80440904700BB9DF810009E
:109BCC0020B101281BD19DF80F1001E09DF80B105E
:109BDC00A9B100284FF0080008BF042000218142E1
:109BEC0003D272180131D770F9E73044314680F84E
:109BFC000390D8F80800D0F89424D0209047013571
:109C0C00CAE74FF6FF7701AE0DF1140A4FF0FF3B98
:109C1C004FF00009C9885FFA89F291426BD9ADF80F
:109C2C000620D0F88824D1203146ADF80440904766
:109C3C0030B1D8F8080009F10109D0F80011E9E7B2
:109C4C00BDF80800B842F4D0ADF81400D8F80800FC
:109C5C005146D0F88824D4209047002841D10025C3
:109C6C00D8F80820D2F80001C1888D4216D2D2F85B
:109C7C008824D1203146ADF80650ADF80440904709
:109C8C0028B9BDF81400BDF80810814201D0013587
:109C9C00E6E7D8F80800D0F80001C1888D42C8D199
:109CAC00CDE907BB099AADF81A70ADF81870807A37
:109CBC00C1000020814214D0131808309B88A342A5
:109CCC00F8D11118002241F8082C09990844514682
:109CDC0020F8047CD8F80800D0F89424D4209047BD
:109CEC00A7E700981FF0D0FE09981FF095FF1920E8
:109CFC0008E01A2006E000981FF0C6FE09981FF035
:109D0C008BFF00200BB0BDE8F08F00BF0C010020D2
:109D1C00FEB50C4615F032F8A00600F18280200446
:109D2C0000F1AF80E00607D52E208DF804006048C6
:109D3C001FF075FE01A88847E00707D025208DF895
:109D4C0004005B481FF06BFE01A88847A00707D5ED
:109D5C0026208DF8040056481FF061FE01A88847A4
:109D6C00600707D527208DF8040051481FF057FED7
:109D7C0001A88847200707D529208DF804004C48F6
:109D8C001FF04DFE01A88847600607D52D20ADF8C1
:109D9C00040047481FF043FE01A88847200607D55A
:109DAC003020ADF8040042481FF039FE01A8884766
:109DBC00E00507D53520ADF804003D481FF02FFE17
:109DCC0001A88847200505D53720ADF8040001A867
:109DDC001FF092FFE00405D53820ADF8040001A86F
:109DEC001FF08AFF324CA068D0F898000068B0B120
:109DFC001FF09EFBA168D1F898100A68029200220D
:109E0C000A601FF041FEA068D0F8981002984860D4
:109E1C00A168D1F840138847A0681FF00DFC002002
:109E2C00FEBD234E02ADB068C06B04301CF0DBFFEE
:109E3C00002802903FF473AF1FF07AFBB168C96B36
:109E4C000A7B013A0A731FF01FFEB1680298D1F821
:109E5C009810077848608DF80470417839B1162F46
:109E6C000BD1B068D0F8541328468847DBE7B168AB
:109E7C00D1F840138847162FD5D0B0681FF0DCFB03
:109E8C00D1E70B4DA868D0F89400007814F0D8FDF9
:109E9C00002802903FF446AFA968D1F898104860AA
:109EAC00A968D1F840138847A8681FF0C5FBE9E7FB
:109EBC000C0100202DE9F04706680446307B02288F
:109ECC0012D196F823006568D6E904A79146884616
:109EDC0080B1B16858481FF04DFD40B100206FF0C3
:109EEC00010786F8250055E06FF0060752E00120C7
:109EFC0086F82600002052492246F0614F48C6F8E9
:109F0C00008086F821901EF06DFD297827201EF028
:109F1C0035F850463946062203F0DAFF58B196F868
:109F2C00260098B344481FF08BFE002086F82600CC
:109F3C0086F825002AE0434D434FD5F8800320F0E6
:109F4C000200C5F8800396F82000042804D157F8C5
:109F5C004C0C4169272088470220C5F8FC02386860
:109F6C00416806208847C0B14020286080202860C6
:109F7C0096F8260038B130481FF062FE002086F8B3
:109F8C00260086F825000020C5F8FC024FF0FF30B3
:109F9C00F061F7693846BDE8F0870220BA461BF03D
:109FAC00FFF90027B9F1020F0AD0B9F1040F4FF0F5
:109FBC00000006D0B9F1060018BF0120800000E0B7
:109FCC000020C5F84C010123D8F80C10D8E9010287
:109FDC00C5F85011C5F8547186F82430DAF8003001
:109FEC001D690B46A847256895F8200002281BD050
:109FFC000428CFD1DAF80000816915488847B0F100
:10A00C00FF3FDCBF4FF0FF30E8610020EF6985F8BF
:10A01C00240095F821100339022928BF85F8250062
:10A02C00204619F0C1FCB5E708484FF0FF311FF08E
:10A03C00A1FCEF69AEE700BF307E0020B4840020A5
:10A04C0089C5010004440240FC010010807E002000
:10A05C00010000802DE9F0415A4E04465A4DB0687B
:10A06C00D0F8D41091F88380297819B1D0F84C0528
:10A07C008047B068016C096811B9D0F84C0580476D
:10A08C00524F0120062C3C7028701ED8DFE804F0DB
:10A09C00040422252B5140004E4800214170B06829
:10A0AC00026CD0F8D41010684B4AC08A40064FF0AE
:10A0BC004E0058BF2520085C107014BBC97801B342
:10A0CC00022828BF022010701BE0B068D0F84C05A5
:10A0DC0080472EE018F04CFD2BE03E4800214170EB
:10A0EC0018F070F825E03A4800213A4A0170B0683F
:10A0FC00006C006890F8691090F86A00517036494D
:10A10C00087009F0F5F8B068006C006888B940E098
:10A11C00B068324A006C016891F86D1011803049BA
:10A12C00006890F86E00002808BF0120087019F034
:10A13C00BBFF28480078A0B9B268106C016829B937
:10A14C00D2F84C058047B068006C01684968254A14
:10A15C00097801F02001117023490068406880786B
:10A16C0008703878062814D8012101FA00F010F094
:10A17C004C0F0ED01FF0DCF90446387802280AD1B7
:10A18C008320287020461FF07FFCBDE8F04119F0B9
:10A19C0077BBBDE8F0811548017819B914490978E5
:10A1AC000029EDD00221B8F1010F297004D10078FB
:10A1BC00832808BF15F0DAF92046BDE8F0411FF0FE
:10A1CC0063BC00BF0C010020B4880020B7880020BD
:10A1DC00A527002021260020B5880020AE8700206E
:10A1EC00B6880020C0880020C1880020AC880020E0
:10A1FC00AF8800202DE9F0438BB0DFF884810C464A
:10A20C00054600208DF81300D8F80010002900F046
:10A21C00AD80032D18BF022D03D191F8420090425E
:10A22C0008D1584900201BF03FFD3DB1012D03D151
:10A23C0085240BE0002099E0032D0DD10121D8F8E5
:10A24C000000032D80F8411003D114B18DF8134098
:10A25C000DE000245DB91EE0022D07D1D8F80000F6
:10A26C000CB1022100E0012180F841100024D8F843
:10A27C00000090F84190B9F1010F0ED190F8431005
:10A28C0019B1013980F8431005E090F8481011B16C
:10A29C00013980F848104FF0010990F8431049B18A
:10A2AC00426C00F12E03074602EB41018A1E00F1BD
:10A2BC0026010CE090F8481000295AD0C26C00F12D
:10A2CC000E0300F1200702EB41018A1E811D1E784E
:10A2DC00158802228DF828201CBB17B32A4A127845
:10A2EC0080F8422003208DF81C007888ADF82000FF
:10A2FC0005AC20461FF03DFC7878BB7BCDE90054C3
:10A30C00CDE902602120B9F1010F08BF222008A974
:10A31C00BA1D11F093FE1D481A4900881BF0C4FCAD
:10A32C0023E041880DF1130448F220020123ADF81B
:10A33C0020104178CDE9004108A917F06DF9D8F843
:10A34C00000090F8401002290DD1418C48F22002F7
:10A35C000123ADF8201090F821102030CDE90041F8
:10A36C0008A917F059F915F057FB01200BB0BDE8FF
:10A37C00F08300214FF6FF75FF260027A9E700BFE9
:10A38C0038270020959902007C2600202E7E002084
:10A39C002DE9F04F89B08246129803F0F00403F0D7
:10A3AC000F0B002818BF01200392103C0025B4FAB3
:10A3BC0084F464092040D4880290107A92886FF358
:10A3CC009F2400F03F0024036FF39F2244EA0060B7
:10A3DC00544C104400905248007804AEC2B2ABB258
:10A3EC00934280F09580A27801355FFA8AF7974204
:10A3FC0073D08AB20195172A6DD3A1F1070938469B
:10A40C0032461FFA89F421460FF052F99DF81B8051
:10A41C0008F00300022826D1BBF1030F00F27D8067
:10A42C000398007ADFE80BF0140205109DF8181061
:10A43C0007E09DF81810884215D10398BDF8161046
:10A44C00C088884204D00EE00498009981420AD159
:10A45C000298002854D012980021836882893046D3
:10A46C0015F0F2FF60B15FEA48701CD5BDF81E0014
:10A47C0084421CD9A9EB000188B21728BDD228E070
:10A48C0012988088E0B3129BDA8819689B681A448A
:10A49C000B7815789D42E6D1013802F1010201F1E9
:10A4AC000101F5D12CE01F4C0120607104E038460D
:10A4BC00214616F049F91B4C00200025F8F734F919
:10A4CC001748E17800780131B1FBF0F202FB101A69
:10A4DC0003E013480078134C019D5FFA8AF1C2B275
:10A4EC0051FA80F1013991FBF2F303FB121A5FFA76
:10A4FC008AF1490051FA8AF104EB8101898B6DE7ED
:10A50C00039D96E81F001FC5002009B0BDE8F08F21
:10A51C000399002088810A20F7E70420F5E700BFA3
:10A52C0097880020A0800020B0B560480021604CC6
:10A53C00016094F83A01032812D002282ED0012889
:10A54C0040F0AF8094F8400111F070F9002084F8CD
:10A55C0040015948817B0220002908BF06209EE05B
:10A56C0054480168B1F5C060C4F82C01B8BFC1F5FE
:10A57C00C060D4F81011002900D5494288422ADD68
:10A58C00D4F814011CF08EFDD4F818011CF09CFDBD
:10A59C00D4F828011CF0BCFD01201DE045480568DD
:10A5AC001EF010FEC4F814011EF014FEC4F81801BD
:10A5BC001EF018FEB5F5C061C4F82801C4F81011DE
:10A5CC0009D094F830215AB1D4F81401D4F82021D0
:10A5DC00D4F82C110AE0002084F8300106205EE04B
:10A5EC00C4F82401D4E94502C4F82C110223C4F8A0
:10A5FC001C01002948BF6FF0010301EB4101194414
:10A60C00042391FBF3F111440029C4F820110FDD50
:10A61C001F2931D3D4F824212AB33E28A8BF3E20C9
:10A62C000130292928BF2921C4F81C010B3909E064
:10A63C00D4F82421032A09D111F1140FD8BF6FF0DB
:10A64C0013011531C4F82011002113E00128D8BFE3
:10A65C000120013811F10A0FD8BF6FF00901C4F8BD
:10A66C001C010B3103E0332928BF33211539C4F801
:10A67C0020110321C4F824111CF014FD01201CF03E
:10A68C0035FDD4F820011CF01FFDD4F824011CF07A
:10A69C003FFDA5F2FF510420032938BF0620C4F862
:10A6AC003C01BDE8B04005F0EBBC00BF3C500C4099
:10A6BC00D81B002008400C4090BA02002DE9F84F3E
:10A6CC00584BDD1D584B93F800B000235B4505D269
:10A6DC0015F8054C2CB108350133F7E74FF000099C
:10A6EC009DE04FF000095B4500F099804F4B0092C4
:10A6FC00504A4FF0000805F8019C1E1D4C4BB2F857
:10A70C0016A04FF6FE721F78012307B336F8044CDF
:10A71C008C4218BF544503D12436013F5B00F4E74B
:10A72C003478042C03D0012C06D0002CF4D109F180
:10A73C00010905F8019CEFE702F1010CB0F80AE001
:10A74C001FFA8CF4A64508BF48EA0308E4E73B4C23
:10A75C00DFF8E0E0384B2678BEF824700A33B6B147
:10A76C0033F80A4C8C4218BF944202D11C33013E80
:10A77C00F5E71C88BC42F9D1DC79002CF6D01C7AA8
:10A78C00002CF3D009F1010905F8019CEEE72C49E6
:10A79C005FFA89F309788B4284BF05F8011C89465E
:10A7AC00009A5FEA096102D0817C012901D1002164
:10A7BC0002E09EF80210013105F8031C9EF801100E
:10A7CC009EF80730B8F1000F05F8022C05F8041CB0
:10A7DC008189C07C05F8053C25F8071C287011D030
:10A7EC00184D194BBBF1000F0CD01E78284619469A
:10A7FC002EB14B1C051DABF1010B9642F2D1C0F8EA
:10A80C0000800A70114C4021207818F0D3FC20B93C
:10A81C002078402164221FF064F94FF0010948466A
:10A82C00BDE8F88F42760020D2BC0200B054002064
:10A83C00E6BC0200407B0020DC5B0020D5BC0200A3
:10A84C00D8BC0200C87A00204084002098880020E0
:10A85C002DE9FE4F074600789B468A46029200F08F
:10A86C000C000C2808D1B888FE211AF0B3F8FE2889
:10A87C00019008BF012019E059480568B878FF28F5
:10A88C0008D01EF00FFD40B1064600781DF0B0FF59
:10A89C00054603E02DB16E6800E00026FE20019015
:10A8AC000EE0FE2000250026019009E01EF0FAFCC7
:10A8BC00002800F09280064600781DF099FF0546AE
:10A8CC00002E00F08A80AA684AB1317802209047A5
:10A8DC004FF6FE7440B104881FF09EF904E0B06896
:10A8EC004FF6FE7400B1448839893078A14211D0FA
:10A8FC0010B909B900200DE028B14FF6FE720132F3
:10A90C0092B2914206D0A1F580714FF6013289B214
:10A91C00914244D897F80290B870387DD7F81080DF
:10A92C003030C0B21CF09AFBB8B304461A20514622
:10A93C0020707868C4F80200A01D1DF06FFCBBF8F5
:10A94C000100A4F817000C983A7D397B84F820009C
:10A95C000E986175A284E0610D986076F878E073CA
:10A96C00307820759BF80000A075788BA0857889CD
:10A97C006082029820820F9884F82E0032B104F184
:10A98C0030004146A0621EF0FDFB01E00020A062F9
:10A99C0070682146007814F081FB87F802903878B3
:10A9AC0000F00C000C280DD0B8780026FF287FF49E
:10A9BC0087AF28680025002600283FF481AF466841
:10A9CC0005467DE70199B888C9B21AF003F8FE284C
:10A9DC000146019001D0019868E7BDE8FE8F00BFE9
:10A9EC00208800202DE9FF47D0E901590E46044686
:10A9FC001EF09EFD95F8FD1021B97169102901D842
:10AA0C00032906D81FF040F80024204604B0BDE806
:10AA1C00F087012785F8FD701FF036F800204E4AAC
:10AA2C0085F8FC00C5E93000C5F8C80085F8FE00C3
:10AA3C003069C5F8E4007069C5F8E800307B85F82A
:10AA4C00F9000028317885F8F8107168C5F8EC1019
:10AA5C00B9F80E10A5F8F610317E52F8211085F8D1
:10AA6C00FA1008BF1027C5F8F07099F80C000BF01D
:10AA7C0059F9204616F0C8F899F83B00374985F883
:10AA8C00FB008A46D4E901873A6B97F83A000DF03F
:10AA9C0043FC7A6B98F8FB0051460DF03DFC98F89E
:10AAAC00F91097F83800012915D1FA6A51460DF0C2
:10AABC0033FCBA6A97F8390046F202010DF02CFC0F
:10AACC0098F8FB0026491DF03DFA98F8FB0021464A
:10AADC001EF054F80AE0BA6A46F202010DF01CFCB2
:10AAEC00FA6A97F8390051460DF016FCE8464046D4
:10AAFC001EF0B8FA99F805001A4A4346CDE9004011
:10AB0C00284699F8041018F065FA40461EF09AFB96
:10AB1C00D9F80800144942460094029005F130001F
:10AB2C0019F088FE12F0F2FD104AC5F8CC0005F1C0
:10AB3C001C00042123461CF0FDFA95F8F80008B11E
:10AB4C00B06805E005F16C0000211CF0BBFF084863
:10AB5C00C5F8BC0059E700BF30BA02000260002003
:10AB6C00CD090100C199000047650200259802003B
:10AB7C004B9A0200FEB504465A480078A04213D9FD
:10AB8C0008780D46012801D1686868B168780128F9
:10AB9C0001D1A86840B1544F57F834601EF0C8FC7E
:10ABAC00F17921B11EF070FF00242046FEBD07EBA9
:10ABBC00C40401216768F1711EF066FF002005F1E5
:10ABCC00040C7074F081B06030602988B180A98B5E
:10ABDC00C6E93D00C6E90E0086F86400B186297D01
:10ABEC002B69B1719CE80610C6F85021BCF1000F1E
:10ABFC00C6E910C34FF0FF32C6F8CC10A969C6E9FC
:10AC0C003B203163A97F86F83610296AC6E91A0001
:10AC1C00C6E91C00B16486F8E800C6F8580102D1F8
:10AC2C003249C6E9101097F840000BF07BF8D7E9D1
:10AC3C00031206F14C001EF0EDFAD7E9051206F1ED
:10AC4C00D0001EF0E7FA2A4938680968C9688847B5
:10AC5C007A6C97F8240046F202010DF05DFB254D4D
:10AC6C00BA6C97F8200029460DF056FBF8690128BC
:10AC7C000CD1FA6C97F8280029460DF04DFB3A6D73
:10AC8C0097F82C0046F202010DF046FB12F03EFD47
:10AC9C00C6F85801204605F08FFD174A06F5AE7030
:10ACAC00042123461CF046FA6D4628461EF0DAF9BC
:10ACBC00387A7968114A2B460094019006F11400F9
:10ACCC0018F088F906F17C0000211CF0FBFE06F55B
:10ACDC00807000211CF0F6FE3868D7E90C12106069
:10ACEC00486062E7CABC02003CBC0200573E01004F
:10ACFC00D001001002600020B58C02008980000099
:10AD0C002DE9F84F0CF09EFC5E480024002690F8CC
:10AD1C0000A0544510D2E0B21BF048FD50B10179AF
:10AD2C0041F00401042905D1807A1CF0ABFF002806
:10AD3C0018BF01360134ECE700241BF00FFB05466D
:10AD4C000027E0B285420AD919F0E4FF28B1807CD3
:10AD5C001CF098FF002818BF01370134F1E707EB0E
:10AD6C0006085FEA086032D04FF47F7000EA880969
:10AD7C0048461EF053FF50B34946FF2204461EF0CE
:10AD8C0097F800275FFA86F94FF0000B574529D248
:10AD9C005FFA8BF0484525D2F8B21BF007FDA0B145
:10ADAC000646007940F0040004280ED1B07A1CF05D
:10ADBC0069FF50B10146727A30885FFA88F30093CC
:10ADCC00234614F04FFF0BF1010B0137DEE7002493
:10ADDC004FF000082C48007BE0B11EF023FAC0F1C4
:10ADEC00540018E000275FFA88F9F8B28542F1D9CF
:10ADFC0019F090FF60B10646807C1CF043FF38B11F
:10AE0C000146727C30882346CDF8009014F02AFF5E
:10AE1C000137EAE76220C1B20322A2462546B1FB04
:10AE2C00F2F9B9F11F0F28BF4FF01F09C0B25FFA3A
:10AE3C0088F14446002818BF0120420102F1400766
:10AE4C0049452A4684BF47014C46E0B2394612F0C8
:10AE5C0004FA0022064617F0400008BF621E40EAC2
:10AE6C000601A8EB02080020D2B2002905EB8205EE
:10AE7C00DCD0BAF1000F02D050461EF0CDFE3046A9
:10AE8C00BDE8F88FE6BC0200407B00202DE9F84FAE
:10AE9C00814608688B469046D9E900454768068983
:10AEAC005548E1681EF066FD18B16FF00100BDE871
:10AEBC00F88F524852494FF0000A4A46C4F814B071
:10AECC0084F80980C4F804A084F802A01DF08AFD5F
:10AEDC00297827201DF052F838463146062202F018
:10AEEC00F7FF40B144481EF0ABFE4FF0FF3084F842
:10AEFC0001A0BDE8F88F434F57F84C0C416927204F
:10AF0C008847414E0220C6F8FC023868416806208A
:10AF1C00884760B1402030608020306036481EF099
:10AF2C008FFE002060704FF0FF30BDE8F88F0220DC
:10AF3C001AF036FA3A68DBF810009BF82010D26948
:10AF4C0090473A689BF820009BF821101368A8F1F1
:10AF5C000102B2FA82F252099847DBE90610C6F8F0
:10AF6C0050010020C6F85401C6F8581159B13A687E
:10AF7C00DBF80400002315690022A84738688169B2
:10AF8C00224801308847207A042804D057F84C0C0A
:10AF9C000169272088473B68DBF81C10DBE90202BB
:10AFAC001C690B46A047D9F8004001206070207A3C
:10AFBC00022815D004281BD13868144D8169284605
:10AFCC008847B0F1FF3FDCBF4FF0FF3060600020DE
:10AFDC006070A81CC6F88403484610F017FF04E004
:10AFEC000B484FF0FF311EF0C5FC6068BDE8F88FD0
:10AFFC000020BDE8F88F00BF307E0020B484002014
:10B00C00CDD20100FC01001004440240010000807C
:10B01C00807E0020F0B587B05C4E0446306848B3A3
:10B02C0090F8401001293FD1022180F840102030C7
:10B03C00214612F056FE05463068C169436B90F804
:10B04C003220007E16F058FAB5FA85F137684D09B2
:10B05C00002887F8430043D040001EF0DFFD37681E
:10B06C007864C8B397F843104A0049491EF08AF82F
:10B07C00376835E050201EF0D1FD306050B35021C0
:10B08C0005461DF01BFF2846214612F02AFE08B388
:10B09C003068012180F840103E483F49008807B0D5
:10B0AC00BDE8F0401AF000BE02200DF10F0148F28D
:10B0BC00200201238DF8180088208DF80F0060887D
:10B0CC00ADF810006078CDE9001004A9204616F008
:10B0DC00A3FA49E088201CE0882001258DF80F0098
:10B0EC007B69BA7CF96B97F8380016F005FA316871
:10B0FC0081F8480058B140001EF090FD3168C864DA
:10B10C0030B191F848104A0021491EF03BF86DB35C
:10B11C0086208DF80F0002200DF10F0548F2200259
:10B12C0001238DF818006088ADF810006078CDE927
:10B13C00005004A9204616F06FFA306890B190F8D0
:10B14C00401002290ED1418848F220020123ADF8AB
:10B15C00101002218DF818104178CDE9005104A986
:10B16C0016F05AFA14F058FC07B0F0BD306890F89D
:10B17C00431019B990F848000028C9D000200021CC
:10B18C00002207B0BDE8F040FFF734B838270020A4
:10B19C00148100202E7E00209599020070B5604D20
:10B1AC000446A8684169497F002973D0D0F8D4209F
:10B1BC00B4F84210D28C91426CD1D0F86C1304F1DB
:10B1CC0028008847002865D0A868002241694A7782
:10B1DC00D0F8D41091F8291021B1E868816A0220C6
:10B1EC008847A868006F90F82B0018B1E868816A4E
:10B1FC0001208847207CC00608D5E868816A1020A9
:10B20C008847A868D0F8281380208847E868C16B65
:10B21C0020208847A868D0F8FC14C06810308847F4
:10B22C006268A86813785278416902F00F064E766E
:10B23C00C2F300114269917603F00F0142699177D4
:10B24C001909D0F8D42082F82C10D0F8D410426907
:10B25C0091F84F30927F0F2B05D09A4203D266683B
:10B26C00F67806B91A464A730022C16881F8302074
:10B27C00D0F8D410497B0F290DD14169C97E022920
:10B28C0008D1D0F864018047A868D0F86C01BDE8FB
:10B29C007040004770BDD0F80C2520469047A96837
:10B2AC004869C07E022814D1C868D1F8FC148847BC
:10B2BC00AA684FF47076D2F8D430D2E90301D2F8F0
:10B2CC00F0245B7B31F8131006FA03F3591A9047FC
:10B2DC00A968D1F8D400D1F8B431228990F82C1097
:10B2EC0002209847A968D1F8D400427B90F82C0032
:10B2FC0090420FD04869D1F8FC148847A86841697E
:10B30C00D0F87C018860A868D0F8F02440694169C5
:10B31C009047A968D1F828131020BDE87040084761
:10B32C000C0100202DE9F84F0446B0F82490C17BA5
:10B33C00008A1EF0D5F948B9A07B032806D009F184
:10B34C00140A1FFA8AF0F128C0F0A28009F11E0A33
:10B35C001FFA8AF0FB280BD309F110001EF05EFCDB
:10B36C0050B3834610304FF01E0ACBF8040001E0B6
:10B37C004FF0000B4FF0820801251FFA8AF01EF0E7
:10B38C004DFCA0B10746A0783870E0787870207931
:10B39C00B8706079F8708DB1A07BA11D3871A07B5D
:10B3AC00032813D1781D08221DF0ECFE12E0BBF12E
:10B3BC00000F01D05F4666E0BDE8F88FA079FE1D56
:10B3CC003871E0797871E07BB8710BE008787871AE
:10B3DC004878B871E07B07F110067873207CB8735D
:10B3EC00607CF873207D3070607D7070A07DB070D3
:10B3FC00607EF070301DE1691EF079FB0020307228
:10B40C002DB14FEA192006F10B05B07201E006F1DF
:10B41C000A05BBF1000F86F809901ED01F48204E7C
:10B42C004FF47A720168CBF800100F21C0F800B00D
:10B43C0030788BF80C1008211EF056FB18B13078C0
:10B44C00082112F0FFFDE069A16A4A46CBF808001A
:10B45C00DBF804001DF096FE05E0A16A28464A467A
:10B46C001DF090FE4D4494F82C005FFA8AF2414690
:10B47C003B46287094F82D00687094F82E00A87044
:10B48C00442017F0F5F83846BDE8F84F1EF0C4BB61
:10B49C0000254FF081084FF0000B6EE75C26002072
:10B4AC0096880020F8B50446007D50B15A4994F9AD
:10B4BC001800C968D1F880108847013004BFE82013
:10B4CC00F8BD554EE27BB568D5F80011E86B0978EC
:10B4DC000AB1807A00E0C07A81429CBFF120F8BDAD
:10B4EC00636A94F8392094F83810A08DD5F88C52F2
:10B4FC00278C0097A84700285ED00546002028809E
:10B50C006868A16AA28D1EF0F5FB04F1300005F10C
:10B51C0084010CC80CC1028880788870B0680A80DD
:10B52C002146D0F8442505F1900090476089B36816
:10B53C00A5F89A00207B85F89C00607B85F89D001F
:10B54C00A27DD4F80E00D4F81210D3F848359847E1
:10B55C00A5F89E00E07D85F8A000207E85F8A1006E
:10B56C0094F83C0085F86C00228CA5F8A8202AB32E
:10B57C00E169D5F8A4001EF0BDFB1DF0EBFDB5F89C
:10B58C00A800E8B1D5F8A400D0B16868411E696084
:10B59C00F82100F8011C6868411E6960002100F860
:10B5AC00011CB5F8A8006968091A6960A9652989A0
:10B5BC0008440230288103E01A20F8BD1DF0CAFDB2
:10B5CC00B5F89E10C8051DD594F83B20E8202AB18B
:10B5DC0011F0040208BF11F0010100D0F8BDB168F0
:10B5EC00486ED1F8FC14884794F83B004FF47A71FC
:10B5FC00B268484309490978B0FBF1F1506ED2F8B2
:10B60C00F4249047B0682946D0F89400007813F0E1
:10B61C0045FD0020F8BD00BF0C010020B0880020C3
:10B62C00F8B5554F554E564D38883168EC8808445E
:10B63C00224600F10801A868806D1EF05BFBA9682A
:10B64C003888504B8A6D2044388022448A65326891
:10B65C0081B20832565C811C398089B2515C1970F8
:10B66C00C11C0730398089B2515838806846009126
:10B67C0004211AF04DFF00901CF016FEA968C86357
:10B68C0000981CF0AFFAA968A1F840003E48007879
:10B69C0018B11EF095FAA968C863EA2019F002FAED
:10B6AC003A48426812B1A8680121904738480221F3
:10B6BC00384C0170E0684069007830B1A87B800993
:10B6CC0017F0A6FC08B10120A870A878A96800287A
:10B6DC000A7C70B218BF42F004020A7400210027E1
:10B6EC001EF0E0FA0146A86880F8461000F17401DB
:10B6FC00B0F85C2080F8486080F84770816501895B
:10B70C00511A426811444160417B890709D5A168EF
:10B71C00D1F808138847A868416E11B1B0F86810C9
:10B72C00F1B190F8601049B1A168D1F80C138847B9
:10B73C00A868C16C11B1B0F8501089B1A168D1F8EA
:10B74C00B820137823B1926C12B19047A868A16805
:10B75C00D1F8581288470020A8601CF007FEF8BDED
:10B76C00A068D0F8541205F1080088470020A860A2
:10B77C0010F044FDF8BD00BFA6860020C087002055
:10B78C0024250020B18800208427002024B8020042
:10B79C00AC8800200C0100202DE9F84FD0E90054B2
:10B7AC00994616468A46834613B10020C9F8000014
:10B7BC0076B11DF0BDFE0746E87968B195F8E80052
:10B7CC0088B138461EF060F96FF00800BDE8F88FBC
:10B7DC006FF00900BDE8F88F38461EF055F96FF090
:10B7EC000E00BDE8F88F0020012105F58078C5E931
:10B7FC003BA6C5F8F460C5F8FC0085F8E810E863D2
:10B80C006873E872404600211EF0B4F820461DF023
:10B81C007FFF38461EF038F91DF0D9F808B9687961
:10B82C00C0B395F84400C00606D52C6C24B1AB6CA3
:10B83C00584610210022A0471DF07AFE04465846B7
:10B84C0009F0E4F920461EF01FF9687960B90A99ED
:10B85C0040461EF08FF808B10120687358460EF070
:10B86C0079FB002085F8E800B9F1000F1CBFD5F872
:10B87C00FC00C9F80000E87A28B10020E8726FF0EB
:10B88C000D00BDE8F88F687B002818BF6FF00C0026
:10B89C00BDE8F88FDBE9005495F84400C00614D5D8
:10B8AC002F6CAB6C584610210022B8470DE0D5F830
:10B8BC00FC0031460AEB0002204618F0D5FFD5F803
:10B8CC00FC10361A0144C5F8FC10002EEFD12046AE
:10B8DC001DF0D8FC0028FAD020461DF00DFF95F87D
:10B8EC004400800605D52C6CAB6C584620210022F8
:10B8FC00A0470020B9F1000F85F8E800C8D0D5F8B2
:10B90C00FC00C9F800000020BDE8F88F7CB5584D4C
:10B91C00584E4CF6C0722B78347883F0010384F0C7
:10B92C000204234308BF1040534C00295249898C10
:10B93C000CBF21EA00000843A08401B2B1F1FF3F23
:10B94C0008DC01200DF103018DF80300522016F0E4
:10B95C008FFBA08C810400F1828081B20A042AD46E
:10B96C0001047CD04FF0FF3101913178022976D15E
:10B97C002978002973D121682346013101A908BF18
:10B98C000B46C207224608BF0B461D6852F8046FCF
:10B99C00B54298BF1A46050758BF1A46C30606D5C6
:10B9AC002546136855F8086FB34288BF2A468306AC
:10B9BC001ED4134623E0480451D504F11000226A2A
:10B9CC00016812B11268914211D02C4D20620129EC
:10B9DC00287803D1012112F035FB7CBD012113F035
:10B9EC0001F8216A28780A6801211EF07AF87CBDDA
:10B9FC002346156853F80C6FB54298BF13464204A2
:10BA0C0001D41A4606E022461D6852F8106FB54262
:10BA1C0098BF1A46C30401D4134606E023461568A2
:10BA2C0053F8146FB54298BF1346820701D41A46D7
:10BA3C0006E022461D6852F8186FB54298BF1A46A8
:10BA4C00400701D4104606E02046136850F81C5FEE
:10BA5C00AB4298BF1046884218BF0028AFD10020D7
:10BA6C00012120620548007812F0BCFF7CBD00BFAC
:10BA7C00D527002018260020F0820020988800206E
:10BA8C002DE9FF4715460F46814639B138461DF062
:10BA9C00F2FF18B10446A5F1010A4EE04A48A0F1A4
:10BAAC0024014A480678701C01386DD001F1240439
:10BABC0091F82810FF292146F6D1002C64D0E81EFD
:10BACC00C0B201280DD84248B0F80080B8F1000F80
:10BADC0007D00320042117F0BBFFA6EB080181421D
:10BAEC006FDDA5F1010A5FFA8AF001280DD83948FB
:10BAFC00B0F80080B8F1000F07D00120022117F038
:10BB0C00A7FFA6EB080181425BDD0120E846394620
:10BB1C00ADF802908DF8000008F104001DF0F9FB5F
:10BB2C00404605F015FF0020A071BDF80C006080A8
:10BB3C002948818C48461AF048F84AF60121002021
:10BB4C002571A4F80090A4F8091080212082E060EF
:10BB5C00E072E07184F8211020490978013149081C
:10BB6C0021725FFA8AF1042938BF01208000012973
:10BB7C0060710BD81A48007858B11A4951F8200056
:10BB8C00C0EB0010800006E0002409E06FF001001B
:10BB9C0004E014480068012184F82010A061E061E1
:10BBAC0000200421002517F053FF0849097888422A
:10BBBC0024BF0D48057008F04FFE204604B0BDE8C8
:10BBCC00F0870024F9E700BFB0540020E6BC020067
:10BBDC00C0BC0200C2BC0200407B0020D1BC0200F1
:10BBEC00C827002060B70200872700202DE9FC4FF2
:10BBFC00D0F8C080D0F8D0C0D0F8E820D8F8003009
:10BC0C00C346E6469C4511D3D8F814B0BBF1000FDF
:10BC1C0000F0898090F8FC3005244FF0000E002BCA
:10BC2C0008BF0124DBF800308BF81040A3EB0E05A5
:10BC3C00A2F1080AB5F5806F28BF4FF48065D0F8E3
:10BC4C00D82032B101F1200301F12402C0F8DC50FC
:10BC5C0005E0C0F8D85001F1180301F11C020026D0
:10BC6C00BAF1000FC8BF0126DBF8044012681F6848
:10BC7C00CDF800E07CB1354B53F82630BB6005FAAB
:10BC8C0006F30126BAF1000FC8BF02260EFB0633DD
:10BC9C002344013B05E02E4B53F82630BB6000F1EA
:10BCAC00F6033B6043F6F0740191D1F8009004EB7D
:10BCBC000516264009F1080EC7F804E0BC683443A9
:10BCCC00BC600024BAF1000FC8BF0124DBF8087077
:10BCDC009FB16146DFF87CC05CF824308C469360E1
:10BCEC0005FA04F30124BAF1000FC8BF022400992D
:10BCFC0001FB043139444C1E05E0154951F8241060
:10BD0C0000F1F40491605460C2F800E09168314392
:10BD1C009160C34504BF05EB0C01C0F8D01090F83E
:10BD2C00FE10019A09B1BDE8FC8FD9F8241041F03E
:10BD3C000301C9F82410D0F8CC00D2E904124068F1
:10BD4C00114300688162BDE8FC8F00BF18BA020085
:10BD5C0020BA020028BA0200F0B58BB0ADF80A0088
:10BD6C00002001F108070C468DF8080038461CF03D
:10BD7C0037F808B306AE0DF10701384632460DF020
:10BD8C0013FC05464FF6FF7085421FD09DF8070047
:10BD9C0000B39DF82800002844D0FF280AD00228C0
:10BDAC0048D0FD2806D001284DD13F4800780138F5
:10BDBC00012844D93E4844E002A80DF0C5F80128FA
:10BDCC0002D102A818F0CAFBA1205AE03848C4F8E6
:10BDDC00120055E006F10800394608221DF0D2F990
:10BDEC0040F2FF10ADF828001DF0B0FD00F00F0080
:10BDFC0000272946142233468DF82A000420CDE969
:10BE0C0006771AF0D7FA2B4905EB450041F820705C
:10BE1C0001EB80002649C0E90177C4F8121001211A
:10BE2C00417210E0052060829DF82B0000F07F002D
:10BE3C00A08208E01C480078411E022923D24FF052
:10BE4C008170C4F812001B4A05EB4501002052F822
:10BE5C0021305D1C42F82150A3610A232074B5FBEC
:10BE6C00F3F303EB8303A5EB430353B902EB81001C
:10BE7C000121017210484FF48061007812F0E2F851
:10BE8C0000200BB0F0BD30B90848C4F812009DF882
:10BE9C002A0084F8280004F11E0006F1080108228B
:10BEAC001DF070F9CFE700BF18260020000001013B
:10BEBC00000003018043002099880020F8B50D464E
:10BECC00417F0446827F1020002908BF0820607043
:10BEDC000AB108306070217F09B101306070A1791E
:10BEEC0021B1217A00EB410002306070267E474977
:10BEFC00002E18BF0E26097802290BD14249097869
:10BF0C00012907D12178012904D04149097809B1C7
:10BF1C00012100E0002184F83410217D31440844D3
:10BF2C002870217E31B13B48007B1DF07BF92978CC
:10BF3C0008442870C0B274283DD81DF06FFED0B3F1
:10BF4C00054634482178677E237F94F818E094F8EE
:10BF5C0006C0627F807C002B41EA800007F0030161
:10BF6C00A77F40EA811094F83410287018BF012381
:10BF7C0040EA032040EA4E2040EAC22040EA073063
:10BF8C0040EA8C2040EA4130000A6870A078A87022
:10BF9C00E078E8702079287160796871A07EA871CA
:10BFAC00E07EE871607F40B1216A05F108001DF068
:10BFBC00E0FD102702E0002523E00827A07F20B138
:10BFCC00616AE8191DF0D5FD0837A07970B1207AA7
:10BFDC00E855E8190237617A4170E819227AE1686C
:10BFEC0052001DF0CFF8207A07EB4007207F08B1F4
:10BFFC00F9B268546078227D2169284430441DF0E0
:10C00C00C1F82846F8BD00BFBA270020182600202A
:10C01C00CC270020407B00202DE9F04F85B007464F
:10C02C008A465818D7F80880D8F80410884202D9E4
:10C03C006FF003057BE04E4D7C68DDF838904FF0D7
:10C04C00FF319B46164628681DF094FC6068B8F8D2
:10C05C002010C5E901015FEAC97014D15FEA89704B
:10C06C0023D5D8F80C0000287AD0D8F81010002965
:10C07C0076D001228DE80700384651465B463246A1
:10C08C0013F098F90EE0A068C14300EA0B0211EA24
:10C09C000B0F1CBFD8F808100A4400EA0A013846F6
:10C0AC0006F074FF08B105463DE0D8F800005C4688
:10C0BC003546039600EB0A09ECB3384612F0D4FD72
:10C0CC0078BB384619F004FB58BB02208DF813904E
:10C0DC008DF810004FEA19208DF812004FEA194024
:10C0EC008DF811002248018938461CF0FEFE5FFADB
:10C0FC0089F0C0F58076B44238BF264604A80421E6
:10C10C0013F05CFD68B92846314613F057FD40B971
:10C11C001748A41BB144018938461CF0EFFE354486
:10C12C00CAE74FF0FF35124800681DF089FD28461C
:10C13C0005B0BDE8F08F0E98400701D40025F2E75A
:10C14C00D8F80C0060B1D8F8101049B100228DE875
:10C15C000700384651465B46039A13F02BF9A2E7C9
:10C16C00034800681DF06CFD6FF00705DFE700BFAA
:10C17C000C2400202DE9F0418AB0514F0546387847
:10C18C00022804D14D480078002800F09480DFF894
:10C19C00348198F82600082802D0042840F08B80BF
:10C1AC0007AC284621461BF0D7FF387802280BD164
:10C1BC001CF020FDA11C1BF072FA28B1BDF81C600C
:10C1CC001DF0ECF9864276D01DF03DFC0234BDF832
:10C1DC001C00214608F08EFE01286CD06E463046BD
:10C1EC001DF0F9FB304621461BF059FA68B1BDF839
:10C1FC001C601DF0C1F9864207D0BDF81C004146F9
:10C20C0021F81A0F4B2015F033FF3878012819D874
:10C21C00AD8A1DF0C3F9854214D020461DF02BFCCD
:10C22C0030B100790138012802D8204612F02EFED8
:10C23C002648016831B124480078012802D1BDF8A4
:10C24C001C008847BDF81C00002100261AF0DEFDFA
:10C25C00B8F82410BDF81C0019F0B7FCBDF81C0090
:10C26C008DF80C60ADF80E0003AD28460CF06CFE9A
:10C27C0070B1CDE900662E1D684631461BF00FFAF1
:10C28C0030B1304621461DF044F803A805F060FBA0
:10C29C00281D21461DF03DF828460FF0DFF950B15E
:10C2AC00BDF81C00BDF80E10814204D0ADF80E0094
:10C2BC0003A805F04DFB0AB0BDE8F081D52700209E
:10C2CC0018260020407B0020BA270020982300204D
:10C2DC002DE9F047012816D1DFF830A1DAF8340146
:10C2EC00012813D10220CAF8340119F077FD01207E
:10C2FC00012419F095FA60B1CAF834411BF062FBC5
:10C30C004FF0FF347FE06FF001047CE06FF0040429
:10C31C0079E09AF85A419AF859119AF85801002C78
:10C32C0018BF0124002918BF0234002818BF043498
:10C33C0001201DF0A5F9013818BF01209AF8381119
:10C34C00B1FA81F1490910EA010902D1002007F084
:10C35C00DFF9DAF808002E4D10F0010807D12D4F47
:10C36C00286A8168384688470428F9D00646404632
:10C37C001DF0F1FAB8F1000F08D1012E04D1286A92
:10C38C0001214268234890471CF014FF286841693A
:10C39C00204688479AF8540118B14FF480601DF07C
:10C3AC0075F99AF8530118B14FF481601DF06EF9CC
:10C3BC0019480121016003200021CAF834011748F3
:10C3CC000160204615F09AFC0128FAD1144E306811
:10C3DC00042019F025FA044612480125B9F1000F82
:10C3EC000560306802D1012007F092F91DF0E8F8E1
:10C3FC00082019F015FA0443CAF8345118BF4FF04D
:10C40C00FF341BF0DFFA2046BDE8F087D81B002074
:10C41C00B801001000400340282008600C200840A0
:10C42C002C2009400C4009407CB54B4EB068016C87
:10C43C00D0F8D420096892F8835019B9D0F84C057B
:10C44C008047B068D0F8B800007800B315F0BAFE99
:10C45C004349424809680068096C884705461DF045
:10C46C0067F804463F48017811B93F49097821B370
:10C47C003E4902220A700078832808BF13F076F830
:10C48C001DF01AFB1DF030FA0420884757E01DF010
:10C49C004FF804463348017811B933490978C9B3C8
:10C4AC0002223249012D0A7004D10078832808BF7A
:10C4BC0013F05CF81DF000FB41E01DF015FA0020B4
:10C4CC008847B0680DF10701D0F82824F420904774
:10C4DC009DF90700854223DB254D287800BB1DF014
:10C4EC00EBFA25480078042803D0B068D0F84C0546
:10C4FC0080471E48042101702878013028701DF0F7
:10C50C00F3F909B1032088471C48032101801DF071
:10C51C00D3FB14E01548832101701DF0CDFA0CE01B
:10C52C00124883210170002017F0F6FD1DF0C4FAAB
:10C53C001048F16880780969087017F0A1F9F06863
:10C54C00C068007800B17CBDB0680021D0F85824D8
:10C55C00002090477CBD00BF0C010020D826002095
:10C56C0030880020AC880020AF880020B4880020E0
:10C57C00A527002021260020B7880020AE870020A8
:10C58C002DE9F84F494C1021207816F013FE28B9EC
:10C59C00207810214FF47A721DF0A3FA44480178E8
:10C5AC000139017009065AD043484FF000084FF684
:10C5BC00FE790026041D41480578AE421DD2207834
:10C5CC00C0B1FF2816D001382070000612D1607857
:10C5DC00032807D134F8041C34F8020C022211F0A1
:10C5EC0063F8607801281EBFA4F8018024F8029C2F
:10C5FC0024F8049C08340136DFE73148DFF8C4A086
:10C60C00314C4FF00008002790F800B05F4519D06E
:10C61C0007EB87000AEB4005287A013828720006E0
:10C62C000ED12046294619F02BF9064610B130469A
:10C63C0019F068FE002EF4D185F80080A5F8029060
:10C64C000137E3E721482249007830B10A780AB172
:10C65C00013A0A7008310138F7E7BDE8F88F15493F
:10C66C00002209780170002005211AF0BBFA04465B
:10C67C000626002C98D020460521002225461AF0CB
:10C68C00B1FA044628890028F3D001382881000427
:10C69C00EFD16889400702D5287B18F0C9FE2868BD
:10C6AC00F0216E73407B15F0D7F8E2E798880020F4
:10C6BC0017870020DFBC0200E04C0020DABC02002F
:10C6CC00D9BC0200D07E0020A31A02009ABC020042
:10C6DC00E02700202DE9F04F85B006464D48DFF8E5
:10C6EC003C9114460D464FF6FE774FF6FE780078D7
:10C6FC00019049480078049001200290002003909A
:10C70C00474800F1110B47480430009099F800C0DD
:10C71C004FF0000E0020C00774D1049B5946C1464F
:10C72C0003B331F8118CB84518BFB04502D11C3198
:10C73C00013BF5E7A84518BFA045F8D00A78501E74
:10C74C000628F4D8072A01D1C146F0E702980EF169
:10C75C00010EC007EBD103985FFA8EF2C0B2824291
:10C76C00E5D351E0BCF1010F2AD8DDE9001ABAF18A
:10C77C00000F25D031F8048CB84518BFB04503D153
:10C78C002431AAF1010AF2E7A84518BFA045F7D059
:10C79C004B79581E0628F3D8087801380228EFD3B5
:10C7AC00072B01D1C146EBE702980EF1010EC00731
:10C7BC00E6D103985FFA8EF2C0B28242E0D323E056
:10C7CC00C8465FEA0E6002D00398000603D0012031
:10C7DC00B845A0D018E000205FFA8EFADFF83C9044
:10C7EC0002900120BAF1010F03903FF48FAF1DF0BE
:10C7FC00ADF8C0B2B0FBFAF101FB1A0003900020B7
:10C80C00029083E74FF6FE781FFA88F005B0BDE87A
:10C81C00F08F00BFE6BC0200D5BC02001826002039
:10C82C00DC5B0020B05400202DE9F04395B00446A9
:10C83C0000208DF81F00208817F096F9002840F092
:10C84C0081804B48007810B14FF0B30908E0A07814
:10C85C00042803D11CF0DEFB002876D04FF0B6097B
:10C86C0000261E201AF0FAFB0546BEB303209DF8E5
:10C87C0052108DF81E0010A808AF08303A4610F080
:10C88C00A9FF0CAE0DF11E0008213A46334612F0FA
:10C89C005DFCA068314610221BF0C4FBE0B11FFA0E
:10C8AC0088F702AE0420002214233946009619F0B2
:10C8BC006BFD9DF91B00B0F1FF3F03DC06F113008B
:10C8CC0017F08EF80220394614228DF8180002ABAE
:10C8DC00042019F06FFD01E04FF0AD09B9F1000F24
:10C8EC0017D09DF81F00012813D19DF9531000207B
:10C8FC00CDE91000002903D401208DF85100FF2050
:10C90C008DF850001FFA88F110AB0420142219F096
:10C91C0051FDBDB1092085F81D9008222870208892
:10C92C006880A0782871681D61681CF02BFCA168D8
:10C93C0005F10D0010221CF025FC0E48294600784C
:10C94C0012F0ACFB15B0BDE8F08360680DF11F016F
:10C95C0010AA0CF029FE80469DF81F0018B14FF06C
:10C96C00000901267DE74FF0AD09002679E700BFED
:10C97C0018260020998800202DE9F843DFF8308133
:10C98C000C46914607462246B8F8241013F046FC94
:10C99C00002879D0068905464FF6FE70864204BF02
:10C9AC00C320BDE8F8831CF0F9FD864204BFC22009
:10C9BC00BDE8F8832988B8F8240088421CBFA8F881
:10C9CC002410084615F020FCE87A3946013088F826
:10C9DC00380008F139001DF0CCF802208DF8010068
:10C9EC00684619F047FF002851D007460069062118
:10C9FC000126017098F80E104170BE771CF0FAF801
:10CA0C0078624020BE7687F81890F8822889788062
:10CA1C00384611F05DFF002845D1092008F11A01B4
:10CA2C0088F826002889A8F81A0098F81800A0425F
:10CA3C0018BF88F818401F4C4B20A04708F1240160
:10CA4C005020A04708F11801E120A04708F1160179
:10CA5C005320A04708200121FEF758FF4FF4005047
:10CA6C000021FEF753FF144C4FF48061207811F035
:10CA7C00B9FF1348007802280BD110480078012820
:10CA8C0007D14FF4DC6208E0CA20BDE8F88310201F
:10CA9C0009E0082010F098FF820020784FF48061A4
:10CAAC001DF022F80020074900220A70BDE8F88327
:10CABC00407B00207D20020098880020D527002094
:10CACC00182600209E8800202DE9F0474FF6FC76B2
:10CADC00B04201D100240FE0884600211D46924649
:10CAEC00002414F055FCDFF814910746680606D4B0
:10CAFC00B9F81600874202D12046BDE8F0873846C7
:10CB0C0029460DF0A7F930B9B01C002180B20DF008
:10CB1C00A1F9002860D0B11C078089B2884505F0C6
:10CB2C00010118BFA0F8028045EA8101BAF1010F9A
:10CB3C00817142D101214171334915F0180F99F8D7
:10CB4C001420097818BF0A4602714046B9F824101F
:10CB5C0016F06AFD0028BDD12A482C49DFF8B0A098
:10CB6C00274B0022007891F800C06245B2D0C2EB8E
:10CB7C00C20600270AEB8604B8420BD003EBC705AC
:10CB8C0021886D888D4201D00137F5E70132F9B269
:10CB9C008842EAD120461C211CF090F94AF601206B
:10CBAC002AF82680A4F811001A48007801304008B1
:10CBBC002074B9F8240060818CE7417901293FF495
:10CBCC0089AF114915F0180F08BF09F11301097845
:10CBDC0080F805A001717DE715F0180F0CD00949FC
:10CBEC0007480978063039B110F8082B013912F0D2
:10CBFC00180FF8D10E388EE702247DE7407B002019
:10CC0C00E04C0020DABC0200DCBC0200D5BC020007
:10CC1C00DC5B0020D1BC0200F0B58DB00546007C79
:10CC2C000F2873D36E68686908AC0021224613F094
:10CC3C0043F89DF82000002868D1287C0B2865D388
:10CC4C00307A022862D1B189C8B2FF285ED19DF832
:10CC5C00220010F0FD0F59D1404F97F8263043F0C9
:10CC6C000402062A04D13E4A1268AAB1C90B1FE07D
:10CC7C003B4A126812B19579012DF4D0082B01D0E2
:10CC8C00042B43D17589002A42D0917902293FD1D6
:10CC9C00284619F021FB39E0727C71893088002319
:10CCAC0000930023FBF7B2FDB089C10B9DF8220065
:10CCBC0032888DF80D10B17B9DF824308DF8100062
:10CCCC009DF825509DF83200ADF8082072898DF83A
:10CCDC000C109DF821108DF80E308DF813508DF836
:10CCEC001400ADF80A20727C9DF826608DF81110A6
:10CCFC00E11D8DF812208DF80F6002AD082205F1B0
:10CD0C000D001CF03FFA28461CF080FF0DB0F0BD62
:10CD1C00B98CA942FAD1012806D0E11D07F13900DE
:10CD2C001AF0BDFC0028F1D10E484FF400710078C8
:10CD3C0016F040FA0028E9D140F20120ADF80D00C0
:10CD4C00B86A029097F82E008DF80C0002A812F029
:10CD5C0021F900289CD01AF085FDD7E7407B0020F4
:10CD6C00CC26002098880020F0B59DB04668077A44
:10CD7C0010AD0446342128461CF0A0F88DF8407004
:10CD8C00294636F8020B16F09DF902201A9604F18A
:10CD9C0028018DF84100608EADF84E009DF84000E2
:10CDAC0002388DF85C0006A81CF0F9F89DF84200DA
:10CDBC0003287AD19DF843501CF0EAFB854274D1CC
:10CDCC009DF84400002870D19DF8450000286CD1D6
:10CDDC009DF84600002868D19DF85D00002864D1BC
:10CDEC009DF84700002860D19DF8480000285CD1D0
:10CDFC0009A81C211CF062F8BDF84E001A9A9DF887
:10CE0C005C30ADF82E00154615F8010B00F003014F
:10CE1C008DF82400032916D100F00C060C2E05D039
:10CE2C00082E08D101268DF8306004E0B2F80150CC
:10CE3C00ADF82850D51C35F8046BADF82A6035F8E0
:10CE4C00026CADF82C60521B0D9513445242032911
:10CE5C008DF838308DF8312027D100F00C010429E1
:10CE6C0023D010F0200108BF10F080001DD1FE204F
:10CE7C009DF85310B4F8422000238DF827000C487D
:10CE8C0040788DF8260094F846008DF81400B4F81C
:10CE9C004700ADF81500E06BCDE90013CDE90203B6
:10CEAC0009A806A905AB08F08DFE1DB0F0BD00BFAA
:10CEBC00C02600202DE9F047DFF83491D9F840A0C6
:10CECC00BAF1000F00F089800AF10C020820FF2152
:10CEDC0051FA80F0C3B21B1A18BF012312686AB151
:10CEEC0063B11388A3F60303012B01D90432EFE7D6
:10CEFC00DAF8100092E8FA003830FAC0DAF80820B4
:10CF0C000025DAE90A10CAE90A55B2B110F0E24478
:10CF1C000CD021F00F0220F0E2434FF0000852EA4F
:10CF2C00030005D01CF057FAB04701E088460446D0
:10CF3C001CF051FA42462346B0471CF0F9FA04465D
:10CF4C00B9F8560001306FF31F30A9F856004FF6B0
:10CF5C00FD70AAF8300009F140008AF833501AF03D
:10CF6C0027FB20461CF090FDB9F85600B9F8541078
:10CF7C00884232D11F48204940680D6830B190F882
:10CF8C00FC200720002A08BF052000E005204C6883
:10CF9C000FF06EFC55B195F8FC00002100284FF005
:10CFAC00000008BF286885F8FC1000E0002044B1A0
:10CFBC0094F8FC200021002502B9256884F8FC10A7
:10CFCC0000E00025A84288BF0546681C05D035B98D
:10CFDC000020BDE8F0471BF041B8BDE8F0871CF01D
:10CFEC00EDFDB5FBF0F10548BDE8F0471BF094BB37
:10CFFC0030210020D01E002070200020207F002037
:10D00C002DE9F04186B01D4614460E46022818D074
:10D01C00012818D0002876D1012E6BD0022E72D1A7
:10D02C0008201AF05FFD3E480021437B3D48026812
:10D03C0040480088CDE9021104913F49CDE90045F3
:10D04C0055E0002000E00120032E00D0F6B91BF0C3
:10D05C00E1FF032E18BF002835D102201AF042FD43
:10D06C002F48304C417B206810F0CCFE2E4989783B
:10D07C0001F00801014345D12C48017801310170C0
:10D08C00C8B2042849D12A48206046E0711E80F0BD
:10D09C00010018BF0121084335D10A201AF022FDE6
:10D0AC0026484FF48061007811F09CFC0DF11601BC
:10D0BC00502018F0B1FF2249BDF8160088840021D9
:10D0CC001CF094FD29E0164890F80D80154807686F
:10D0DC00184806881CF03AFC0121002204903046C6
:10D0EC004346CDE90045CDE9022113493A4605F006
:10D0FC00CFFB07E008201AF0F5FC20462146002261
:10D10C001BF0E8FF48B10F4801214FF47A72007808
:10D11C0006B0BDE8F0411CF0E7BC06B0BDE8F081FC
:10D12C00CC22002070880020268700208927002030
:10D13C0000F8FF0780270020B426002098880020E4
:10D14C00407B0020998800202DE9F04F8BB00C46D5
:10D15C000690C9881F460792E07816F0CFF9002890
:10D16C007ED0217D0546C0B219F0AFFE002879D0E3
:10D17C000646E188E0780597DDE9177900224FF043
:10D18C00000815F095FC8346E0787071E188A07D6D
:10D19C0086F80880227DF1807081F06821691BF08F
:10D1AC00F1FF86F8149077824FF000090027BBF14D
:10D1BC00000F4AD05FFA89F0854246D906EBC00AC7
:10D1CC009BF80110504600F8168F012904D1012755
:10D1DC000770BBF8020005E0BBF802008AF81D00DE
:10D1EC001BF076F9AAF8180022789BF80410520666
:10D1FC008AF81A1005D59AF81C2042F002028AF817
:10D20C001C20C7B9204AD28A904214D11E48A17062
:10D21C00DDE90613CDF80080828C159801901698E4
:10D22C00CDE90208204608F0CDFC9AF81C0040F02D
:10D23C0005008AF81C0009F10109E188E0785FFA21
:10D24C0089F215F035FC8346B1E7304619F0C8F881
:10D25C000599DDE9142320460096FAF719F810E039
:10D26C00B92000E010208DF82800E078A17D8DF821
:10D27C002300E0888DF82410ADF8260008A81BF0D8
:10D28C005FFC0BB0BDE8F08F407B00202DE9F84F20
:10D29C00816A91F90120002A2AD4824602F01F00EB
:10D2AC0000EB40049AF81C300234A34220D18B1CB2
:10D2BC00D2B24FF6FE784FF6FE7C08B1B1F802C040
:10D2CC00DFF804914FF0000B4FF6FE770021B9F810
:10D2DC001650814211D29C7814F0880F08D133F883
:10D2EC00037BBEB2AE4208BF04F0070B0131F0E77E
:10D2FC00D320BDE8F84F09F006BD5FEA0B6006D1FC
:10D30C001FFA8CF0B9B215F0B3FC00284FD0BAF864
:10D31C000C001CF05CFB98B10021027AC1712B4906
:10D32C0009788A4208D30131490801725FFA8BF1FE
:10D33C00072938BF0BF1010B80F809B0BDE8F88F55
:10D34C0008F10101BAF80C0089B217F0C9FC20B140
:10D35C0005461E48297C007815E016F047F930B3D5
:10D36C001C2105461BF0AAFD4AF60120A5F8110068
:10D37C00BAF80C002880B9F82400688113480078AA
:10D38C00411C49082974814208D301304008287493
:10D39C005FFA8BF0072838BF0BF1010B002085F8E2
:10D3AC0011B02873023528461AF01AFD08B1BDE8F1
:10D3BC00F88F9AF808000028F9D0DAF818102846E7
:10D3CC00BDE8F84F1CF0D5BB407B0020D1BC02005F
:10D3DC007CB50568002D6DD004464748026842B103
:10D3EC00217928469047012803D1688920F0010053
:10D3FC006881687B02282DD1688980072ED5207919
:10D40C00CD282BD0F02829D0688A00060CD5A87E10
:10D41C0050B1A8732868008816F0A6FB40B94FF4E9
:10D42C00987009F070FC03E0344800780130A87360
:10D43C002079002856D004202021687330480088B9
:10D44C002881A87B0138A876A8732E48007810F0A4
:10D45C00F9FD687B40F0040006282BD12B49288B62
:10D46C00C98A884214D02849097889B12968098861
:10D47C00ADF8000001208DF80500287BADF80210F6
:10D48C008DF8040020798DF8060068461BF0F2FC3C
:10D49C006889C0070ED0217928461BF040F86889AE
:10D4AC0020F0010068812868008816F05DFB217966
:10D4BC0008B121B17CBD39B140F2311001E040F22C
:10D4CC002D1009F020FC7CBD40F22F1009F01BFC44
:10D4DC00002560798542EDD24FF49B7009F013FC66
:10D4EC000135F6E7002660798642A4D24FF49B7092
:10D4FC0009F009FC0136F6E738240020B627002095
:10D50C007C27002098880020E9250020407B002003
:10D51C00BFB54A4D044695F82600092800F28C80C8
:10D52C00012101FA00F040F20A21084200F0848047
:10D53C006178F1B141F2030011F0E1F84048007854
:10D54C0002280ED13F4801780B2904BF0A21017033
:10D55C003D48002101703D484FF48041007811F0A6
:10D56C0041FA6178A88C1CF041FB002085F826005C
:10D57C0060E00220002111F0C2F834F8020FE882BA
:10D58C005320214614F074FD95F82600092802D08A
:10D59C00A88C14F039FE01200DF10F018DF80F004D
:10D5AC00422014F065FD04200DF1070485F82600D7
:10D5BC004A20214618F030FD05F11C0021461CF0D4
:10D5CC00D8FA204801780B2902D10621017003E01A
:10D5DC00A88C00211CF00AFB194C207802280AD2D6
:10D5EC00688B4FF6FE7188420ED00DF107010022B8
:10D5FC00FEF746FA08E007D1E98A032011F07FF81C
:10D60C00698B042011F07BF8A87B0DF10F01C0F39E
:10D61C00C0008DF80F00522014F02AFD207802284B
:10D62C0008D1A87B00074CBF4FF40040012001211A
:10D63C00FEF76CF91AF07EFEBFBD00BF407B0020E8
:10D64C0018260020C4260020CC2700209888002013
:10D65C002DE9F0418846080430D45FEAC86000F137
:10D66C0081805FEA887000F182805FEA087000F1C7
:10D67C00818018F4706F00F082805FEA085004D546
:10D68C0000201BF0C5F988F400685FEA485004D507
:10D69C0001201BF0BDF988F480685FEA885004D53E
:10D6AC0002201BF0B5F988F400785FEAC85068D501
:10D6BC0003201BF0ADF988F4807862E0324F3878A3
:10D6CC0011F0BEF900284AD0054646680078411E84
:10D6DC0005290DD91A282CD024282ED0D12833D0A6
:10D6EC00D32835D0FD2836D128461AF088FB32E0F5
:10D6FC00DFE801F0030B310F311B66B3304611F03C
:10D70C001DFC30461CF088FA25E0284614F08CFEEF
:10D71C0021E0F478701CE11CC9B21BF099F8611D72
:10D72C0056FA81F101F8010C15E028461AF064FF55
:10D73C0011E02846FDF7F6FD0DE0F0780530C1B29A
:10D74C0030461BF007FF06E028461BF00FFF02E0F7
:10D75C00284611F061F828461AF07EFBAFE788F4F2
:10D76C0000480EE01AF02EF888F0100809E088F056
:10D77C00020806E00DF002FB88F0080801E04FF00B
:10D78C0000084046BDE8F0819688002070B50C4634
:10D79C0008041CD4E00729D144480078012805D896
:10D7AC00A00745D4A00654D4600474D4E0062DD44C
:10D7BC00200744BF84F0080070BDE0053DD460072D
:10D7CC005FD400202146BDE8704009F0DDBB344E2B
:10D7DC00307811F035F930B1054607F043FC284696
:10D7EC001AF03AFBF4E784F4004070BD01201AF003
:10D7FC0079F92C480F220F2381782B48008800F0F0
:10D80C000700FFF7FDFB84F0010070BD2548007890
:10D81C0010F0D8FC28480078012806D127484FF48E
:10D82C000061642200781CF05FF984F0100070BD78
:10D83C000AF046FA84F0020070BD214890F82600E8
:10D84C00082801D0042801D11BF038FA84F4807028
:10D85C0070BD1748007860B912480078062802D1CC
:10D86C0007201AF03FF913480078012808BF19F077
:10D87C00F1FC0B481021007810F0E4FB84F0200040
:10D88C0070BDFF20032116F019F81BF093FE0D4814
:10D89C0001210160FEE714F041FB84F4804070BD6F
:10D8AC0099880020C42600202687002018260020F6
:10D8BC00BB880020BA270020BD27002098880020B4
:10D8CC00407B00207C052043F0B58DB0044603203E
:10D8DC000D468DF830000AAE30461CF04AF91BF0AC
:10D8EC0089F90146304619F0DAFE50B1287D40F036
:10D8FC000201032905D1297A09B1FF2914D182200B
:10D90C0000E084208DF82700E289207C0DF12701AE
:10D91C000123CDE9001004F11100A11C42F40042D6
:10D92C0013F07AFE0DB0F0BD032804D1A87DFF28BA
:10D93C00E5D00028E3D0304F4FF0FF300822CDE97E
:10D94C00060006A93E1D30461AF06CFB18BB2B488E
:10D95C006188C08A81421ED03878FF280AD0297A83
:10D96C00814207D078884FF6FF71884202D06989CE
:10D97C00884210D10020314608228DF8080002AFF1
:10D98C00381D1BF0FFFB38460DF068FE6088BDF8B3
:10D99C000A1081422DD1E08905F10C0621281CD1F9
:10D9AC008C206989AB7D32468DF82700287A17F0D8
:10D9BC00E7FA0028A8D11BF09CFF287D0328A3D1EF
:10D9CC0002A9304617F00CFB00289DD130460021EF
:10D9DC000022002310F026FC96E76989287AAB7D9B
:10D9EC0032461AF093FA08B188208BE71BF081FFBE
:10D9FC008AE78D2086E700BF00260020407B0020B0
:10DA0C002DE9F04F8BB04B4FB868D0F80001807AFD
:10DA1C00C0001CF003F9002809907ED00DF1040B16
:10DA2C0000264FF6FF7A0BF103051BF081FD0DF17B
:10DA3C0014090090B868B2B2D0F800110B899A4260
:10DA4C0063D201244FF00008C97A5FFA88F28A4247
:10DA5C0021D2D0F88824D02059468DF80680ADF814
:10DA6C000460904728B1B86808F10108D0F800119B
:10DA7C00EAE79DF8100000240128F4D19DF80F006E
:10DA8C000028F0D10020082806D0295C0130FF299D
:10DA9C00F9D00024E7E70CB10136CBE70024B868D5
:10DAAC00E1B2D0F80021D2888A42F5D9D0F8882486
:10DABC00ADF80610D1205946ADF80460904710BB64
:10DACC00BDF8080050451ED0ADF81400B8684946A2
:10DADC00D0F88824D420904708BB4FF0FF3049463B
:10DAEC00ADF81AA0ADF818A0CDE90700B868D0F8C9
:10DAFC009424D4209047B8685946ADF808A0D0F8C3
:10DB0C009424D12090470134C9E700981BF0BCFF46
:10DB1C0009981CF081F8002008E01A2006E0009813
:10DB2C001BF0B2FF09981CF077F819200BB0BDE878
:10DB3C00F08F00BF0C010020F0B589B00546002025
:10DB4C0001F108060C468DF80F0030461AF048F922
:10DB5C0018B9284631460DF05DF804AD0DF10F01F2
:10DB6C0030462A460BF020FD3B4E4FF6FF773178BE
:10DB7C004A1E9DF80F10012A10D879B900200DF11A
:10DB8C000F01CDE90000684604AA0BF00DFDB84268
:10DB9C001ABF01218DF80F109DF80F10B1B1B842CA
:10DBAC0014D09DF8201099B3FF2926D0022918BF54
:10DBBC00FD2912D12A4900EB400001EB8000A1693C
:10DBCC0050F8042F91420FD2A22042E0307810B9C5
:10DBDC001BF0BCFDC0B1A1203BE0012938D130784D
:10DBEC000138012806D90FE0013101603078411E5F
:10DBFC0002291ED24FF0817007E0307801380128DD
:10DC0C009CBF012084F826001448C4F812001FE0C1
:10DC1C00052060829DF8230000F07F00A08212484E
:10DC2C000078002818BF012084F8270084F826000B
:10DC3C000EE030B90B48C4F812009DF8220084F8AD
:10DC4C00280004F11E0005F1080108221BF09AFAC5
:10DC5C00002009B0F0BD00BF182600200000030111
:10DC6C008043002000000101942700202DE9F84F8B
:10DC7C001D4600928B4681461BF05AFC444A824654
:10DC8C0000214FF4A060012705F1010C002392F84C
:10DC9C006040602935D007FA03FE1EEA040F0AD053
:10DCAC00BCF1000F18BF9D4205D1561896F80A809A
:10DCBC00B8F1000F04D000F5807020310133E8E793
:10DCCC0024EA0E040125737282F8604092F86240D7
:10DCDC00B572013482F862409EB142F801902D4930
:10DCEC00BBF1020F86F808B0716011D0BBF1010FC7
:10DCFC0034D1591DB1740A2131820A998968716134
:10DD0C002CE0FE2450461BF0BFFE60B2BDE8F88F3D
:10DD1C00718A5A1D0A9B02F00F0221F4706141EACC
:10DD2C000221718221F0F8015A7902F01F0241EAB6
:10DD3C00C201718221F4C0419A7902F0030241EAD6
:10DD4C00423140F20362328271824EF6FF72114010
:10DD5C00DA7902F0010241EA023171820B9A42B186
:10DD6C0011785278920042EA411108430A4908435B
:10DD7C0000E000200099B06101B171600748416872
:10DD8C0009B9C0F804900FF02BFC747ABAE700BF05
:10DD9C00B87B0020BB2E010001000406D01E002021
:10DDAC007CB504468078022820D0012840F08C8075
:10DDBC00267D00208DF8060006F1180019F04EF9AA
:10DDCC00054610B901208DF80600607940F002007C
:10DDDC00022824D1002D4CD0E078002818BF012057
:10DDEC001BF0EBFA23D01BF0C5FA25E000208DF8D0
:10DDFC0007002C2019F032F9054610B901208DF8D6
:10DE0C000700607940F0020002280CD1002D54D09C
:10DE1C00E0781BF0D2FA31D01BF0ACFA33E00220E0
:10DE2C008DF8060025E002208DF8070045E0A01DC6
:10DE3C00042118F06DFBA860A07C32462874E07CAD
:10DE4C006874207D15342146A87505F117001BF068
:10DE5C0099F9A05DA874A019417869758178297524
:10DE6C000521C07829802946E8741848007811F0FB
:10DE7C0015F90DF106037520012122E0A01D0421E6
:10DE8C0018F046FBA860A07C04F115011022287440
:10DE9C00E07C2875207D687505F11C001BF072F97B
:10DEAC0004F12500042118F033FB0821A861074870
:10DEBC0029802946007811F0F1F80DF1070375203F
:10DECC000221012214F0D4FB00207CBDA488002088
:10DEDC002DE9F04F89B00E46834601A82021144647
:10DEEC001AF0ECFF202E08D0182E04D0102E0CBFE8
:10DEFC000127002702E0022700E0032744F2040A6E
:10DF0C004FF00108C4F2020A40F2B01908FA04F505
:10DF1C00C1F200090094CAF80054D9F8000044F288
:10DF2C00007441692720C4F2020488470320C4F816
:10DF3C008080C4F88400C4F80080C4F888004FF6D0
:10DF4C000850CFF6FF7021588F4218BF2750182E5B
:10DF5C00CAF8FC5315D101A8594618221BF0CAFE69
:10DF6C000320C4F8880000BFD4F890008007FBD1D0
:10DF7C000020C4F248200121016020260DF1040B81
:10DF8C0011E0BBF1000F18BF002E10D00320C4F815
:10DF9C00880000BFD4F890008007FBD10020C4F2A9
:10DFAC00482001210160CAF800B0CAF808600325B6
:10DFBC00CCF2000501201BF012FDD4F89000284291
:10DFCC00F8D0D4F890000540C4F88850D9F8000077
:10DFDC00016A27208847D9F8000001692720884763
:10DFEC000020B0EB957F07D1DAF800040099C0430C
:10DFFC00C84000F0010000E0012009B0BDE8F08F3E
:10E00C002DE9F04F8BB04248DFF80CB100240DF134
:10E01C001C0A4FF000084FF000090027007801900F
:10E02C0000EBC00086003B480078013040080290AD
:10E03C0046455CD01FFA89F1032000221023CDF84D
:10E04C0000A018F0A1F900284CD19DF821300BEB61
:10E05C000801BDF81C009DF820200C82CC60CC720D
:10E06C004B714AF601232BF80800BDF81E000A710B
:10E07C00A1F80930029B48800B72BDF82230CB808E
:10E08C000A9B5D1C04D081F82040C1E9063315E0E1
:10E09C00013A012A09D8214A12784AB1204B53F887
:10E0AC002220C2EB0212920004E06FF0010203E0A6
:10E0BC001B4A126881F820408A61CA614FF6FF71D1
:10E0CC0088420FD0ADF8180001208DF80C0003A881
:10E0DC0011F014FF28B11348818CBDF81C0017F007
:10E0EC0074FD013708F1240809F10109A0E70020AB
:10E0FC000421002415F0ACFC0199884224BF0A4885
:10E10C00047006F0A9FBF8B20BB0BDE8F08F00BFAD
:10E11C00E6BC0200D1BC0200B0540020C82700208D
:10E12C0060B70200407B0020872700202DE9F041DA
:10E13C00414F04467878C8B1DFF80081B8F8540034
:10E14C00B8F8561088421ED008F13801204619F054
:10E15C0040FA80B9D8F8480010B10069A04207D045
:10E16C0008F14001204619F034FA03E0BDE8F081D3
:10E17C00D8F8480038B1B0F9301020460A224FF0D8
:10E18C00E04308F035F81BF0D3F92D4D0646284630
:10E19C0002C8A14208BF28460021016078780138E6
:10E1AC007870000636D17C60387E02280ED10820AB
:10E1BC0016F0F2FA30461BF067FC04F150004FF0F9
:10E1CC00FF311BF0D7FB1BF0B3F9064605F1280015
:10E1DC001BF038FD40461BF0FDFC1A481BF032FDCD
:10E1EC0008F11C001BF0F6FC17481BF0E5FC174867
:10E1FC001BF0E2FC1648416811B107F1500088474A
:10E20C0007F1280019F0EEFB1248807810B10D20B0
:10E21C0007F016FB7868A04204BF002078603046F7
:10E22C001BF032FC04F150001BF008FD04F1B800A7
:10E23C00BDE8F0411BF0C0BCD01E002030210020F6
:10E24C007020002028800020647F0020207F002088
:10E25C0074260020ACBB02002DE9F0478EB080463E
:10E26C000E2016468A468DF81A308DF818208DF837
:10E27C00190001208DF81C003E48B8F1000F077BF7
:10E28C008DF81B7021D00AEB0605687B11F0FEFEA1
:10E29C00002403463A2802D03B2B0BD13B230DF133
:10E2AC000409002011214A4619F084FE002808BFF9
:10E2BC0009F1010428780994384305F8050B0DF190
:10E2CC002B0029461BF055FC36E001AD0020112136
:10E2DC003A2300242A4619F06DFE08B109942BE06C
:10E2EC00DFF894906C1C012101220994D9F80430B8
:10E2FC00581CC9F804000AEB06000090384612F0CE
:10E30C00CAF81AF077FC01460DF12B001BF031FC1A
:10E31C00B9F80000194901300968A9F8000080B269
:10E32C00814203D3D9F80400012805D114484FF4D5
:10E33C00007100780FF086FE0DF12B000AEB06053C
:10E34C000422691C08301AF01DFF1AF806008DF81B
:10E35C0037005CB106A90DF12B024046534606F07E
:10E36C0091F8297801F0F801297000E0A1200EB095
:10E37C00BDE8F087407B002004250020ACBC0200E7
:10E38C00998800202DE9FE431BF0D2F8DFF80C91A0
:10E39C00804699F80100B8B14148032201688260B7
:10E3AC00C80711D03F4C2068416802208847019073
:10E3BC00206841680120884702903B4801A91C3025
:10E3CC0011F084F917F04CFDD9F80450EDB1364931
:10E3DC00686A01AF01F11C06A96A884219D230465D
:10E3EC00394612F06FFA013011D0D5E90912E869FB
:10E3FC00541A08443946082C28BF082422461BF01E
:10E40C0079FC686A20446862E6E700240CE0D5E9F0
:10E41C0009010024884207D309F10400294618F0A9
:10E42C00EDF985F83240012499F8010088B9D9F842
:10E43C00040018B180681AF017FB0AE01A481C3067
:10E44C001AF0E5FF28B9194A4FF0FF30012110F0FE
:10E45C0053FB40461BF018FBF4B1A868002201687E
:10E46C00CA628A690AB10223137091F83030012B09
:10E47C0007D0022B10D101F134001BF0E1FBBDE8F9
:10E48C00FE8322B1CB6800219847BDE8FE830C695E
:10E49C00CA698B6A0021A047BDE8FE8318230020BF
:10E4AC0008800240CC0100107422002080A90300D7
:10E4BC0070B586B0454D0446A868D0F8F41091F8B4
:10E4CC004420B2F1820318BF531C81F84430D0F8B9
:10E4DC00F40090F8441000EBD10090F82C104A088E
:10E4EC0080F82C20C807A86809D1D0F8F41091F94D
:10E4FC004420531C12F1020F81F84430E7DCD0F8B1
:10E50C00F420114611F8443F802B25D8D0F8302444
:10E51C00E1209047AA6802208DF814004FF0FF30DC
:10E52C00D2F8F430ADF80C009878022823D00128EA
:10E53C0024D030BB1BF042FB4FF47A71244B0022E9
:10E54C00B1FBF0F023490BF045FCE0B3A8681A21AD
:10E55C00D0F8F400417004E0907810B91C4814F025
:10E56C0007F92A202070A868D0F84013204606B07E
:10E57C00BDE870400847D2F86814F7E708208021FE
:10E58C0001E007208321D2F8786303F149020023CC
:10E59C00CDE9003203AA4FF6FF73B047A0F1DB01BF
:10E5AC00182910D8012202FA01F10B4A11420AD0A3
:10E5BC00A968D1F8F41048702A202070A868D0F807
:10E5CC0040132046884706B070BD00BF0C010020E8
:10E5DC0058880020FD2C0100112400012DE9F04386
:10E5EC0089B004464648807860B9E07AFE2809D1A3
:10E5FC00684624211AF062FC208B10F00D0F06D017
:10E60C00B62400E00124204609B0BDE8F083207A4E
:10E61C000028F5D001288DF8080011D002281CD054
:10E62C0003281ED00F2820D102204FF000080B2603
:10E63C004FF000098DF808002088ADF8000019E0B3
:10E64C00B4F800804FF6FF700F26ADF800000220E2
:10E65C004FEA18298DF808000CE02088ADF800006E
:10E66C0003E0684621461BF084FA4FF000080326AD
:10E67C004FF0000906F00C0707200C2F08BF0920EB
:10E68C00A17C08448DF81F00C0B21BF0C7FAA0B3E0
:10E69C000890054686700C2F11BFE81C85F8049075
:10E6AC0085F80380681DA17B0170E17B4170217CA2
:10E6BC008170617CC1700430628A61691AF062FDFC
:10E6CC001AF066FF81098000033069702870B7FA70
:10E6DC0087F04009ADF80E0003208DF80C00A07EE9
:10E6EC008DF80D00A089ADF80A0068461BF026FADB
:10E6FC00044628461BF090FA85E7102483E700BFF8
:10E70C00C02600202DE9F04F85B0054691460E46F7
:10E71C00C80731D12846314612F03AFE404FF98AEB
:10E72C00884242D02846022132460CF0CBFCE0B3A2
:10E73C0028464FF6FE7102223346FEF7C5F990BB10
:10E74C004FEA152806F0DF0A70061ED402A92846E7
:10E75C0017F03EF968B9B98C284616F0C1FAA0B189
:10E76C00871C384619F03CFB78B102A839461BF0DF
:10E77C0000FA46F0200A08E0B0074CBF46F0100A39
:10E78C0046F0080A4FF0FF08FC25264800220778BF
:10E79C00791C01702248012100913946C08A034638
:10E7AC0009F080F818B1C72036E0002034E00E20C4
:10E7BC001AF0200408BF06208DF8110004A818F0E8
:10E7CC0059F840B34FF0010B064680F81EB01AF012
:10E7DC0011FA70623069002141710AF0780187707A
:10E7EC00C57080F8048080F800B041701CB1063010
:10E7FC0002A91BF0BEF96FF00300B9F1000F708095
:10E80C0005D009480078484588BF86F81A903046EC
:10E81C0010F05EF800E0102005B0BDE8F08F00BFEE
:10E82C00407B0020BC880020CFBC02002DE9FE4FAD
:10E83C008A4683461AF000FEDFF80891DFF8FC8068
:10E84C003F4E99F8001098F80200B07339B10007E8
:10E85C0013D501200DF10A018DF80A000AE0002001
:10E86C0000240EF093FCB07B000706D58DF80B400E
:10E87C000DF10B01522013F0FBFB0FF0D7F819F040
:10E88C0087FF38B105460EF0E3FD13F031FF0DF0B4
:10E89C00B5F808E009F052F80546307E012101FA7E
:10E8AC0000F0294908604FF6FE74012D2FD10FF0AE
:10E8BC0029FC1BF04BF807462448234900680860E4
:10E8CC00FF20022114F0FAFF601C7483F482B084E0
:10E8DC00002013F0CFF907F07F00584400F16406D4
:10E8EC001B480078012808D10020BAF1010F1CBF89
:10E8FC00CDE90000684615F013FB114A2120742164
:10E90C001AF07EFF0020022114F0D8FF00E0002650
:10E91C0028460CF0FFFF601C80B2834507D0012015
:10E92C0089F8000018F01EF8B0B219F025FF98F81D
:10E93C00020019F04DFB2846BDE8FE8F268700200B
:10E94C00407B0020C4260020708800206C2700200B
:10E95C00182600202DE9F0438FB014F0EFFB3F4F49
:10E96C0097F82600082806D00120C7E90C003C487F
:10E97C000078F87078710DF11408242140461AF0D3
:10E98C009DFA39480F25374EDFF8E0900DF13B0129
:10E99C008DF83B5000783570013818BF01208DF888
:10E9AC001E004620C847324800248DF800400078ED
:10E9BC008DF801001AF0ECFD8DF8020097F8380084
:10E9CC008DF80640ADF8034007F139010F2838BF28
:10E9DC0005468DF805506D46E81D1BF0CAF84FF042
:10E9EC00FF303278234EADF80F008DF8110097F8F8
:10E9FC00720031468DF81200284610F092FE452028
:10EA0C003146C84705F028FFB88D97F82F108DF8C0
:10EA1C0020408DF834408DF82940ADF81C00387E2C
:10EA2C008DF81F1007F116018DF81A00B88CADF88F
:10EA3C0018005320C84707F11A014B20C847F87932
:10EA4C00642100FB01F20C48082100781BF04CF803
:10EA5C00404606F0BFFB0FB0BDE8F083407B0020C2
:10EA6C00E6BC0200A9270020182600207D20020009
:10EA7C00D827002008870020988800202DE9F84F1F
:10EA8C004FF00056002A984617460C46824618BF8F
:10EA9C004FF080464D1C1AF04BFD814635B1504667
:10EAAC002146002213F0B2F904460FE03748816C7E
:10EABC0011B10969514506D0C16C11B109695145B3
:10EACC0003D0846B02E0846C00E0C46C34B194F924
:10EADC003300B0F1FF3F03DD042451E003244FE089
:10EAEC00DFF8A8B00A9DDBF84800844218D0DBF8A8
:10EAFC004C00844214D05046214642462B460AF024
:10EB0C0033FB0028E8D02248017E012937D0007E53
:10EB1C00042834D01F48204928301BF095F82EE0EB
:10EB2C00DBF848000022334617F008FFDBF84C00F6
:10EB3C000022334617F002FF1848002F18BF00F5CB
:10EB4C00803018F0AFFE85B1DBF848001AF0EFFE0C
:10EB5C00DBF84C001AF0EBFE20690E49086291F8C4
:10EB6C00240040F0010081F82400B8F1000F06D019
:10EB7C00DBF83810504601222B460AF0F5FA8324B4
:10EB8C0048461AF081FF2046BDE8F88F302100205E
:10EB9C00D01E002070200020020000400100010463
:10EBAC002DE9F0410546880058BFBDE8F0810020F2
:10EBBC00002410F09FFA3D493D483E4FCC6108605F
:10EBCC0040F60A008846B887FC8797F8480000F0A2
:10EBDC00F00087F848003C6497F8490000F0F0001A
:10EBEC00013087F84900284607F050FEAC68012038
:10EBFC0021460E46496849B10A88A2F60302072A43
:10EC0C00F7D800FA02F212F0830FF2D0707B00F00A
:10EC1C00F000707307F13C0070602748806B28B1DE
:10EC2C00C0680088A0F6030002281AD3284630F8E2
:10EC3C00381FB1B10021E9636987386495F8440045
:10EC4C0095F8451000F0F00085F8440001F0F00054
:10EC5C00013085F8450097F8490000F0F00087F87E
:10EC6C00490019F0EFFF1548F86197F8250030B10D
:10EC7C0017F050FE0028FBD012F042FB0BE00120F5
:10EC8C001AF0FEFC012806D0707B00F0F000013079
:10EC9C0070730B48F86100202146C8F81C00C8F8B6
:10ECAC0000400120BDE8F04118F0CCBE001004403B
:10ECBC0001010E04D01E0020302100202D37000051
:10ECCC00850802002DE9F04788B0434D0A460446FA
:10ECDC001046A98C14F0A8FC40B1417831B9072139
:10ECEC0041703E490978013149080170A06A10222F
:10ECFC004778F90658BF082217F08F0F13D1BB06BF
:10ED0C0048BF0832237F93420DD190F8029090F8BF
:10ED1C000780B0F805A0B0F80360002909D407F00B
:10ED2C00700708200DE0D32008B0BDE8F04707F0CD
:10ED3C00EABF00F1080106A81AF01BFF07F06007F4
:10ED4C001020B90606D5A16A014404A81AF011FFD7
:10ED5C0007F05007B6B24946304615F051FD204930
:10ED6C00097888421ED21F4900EB800001EB40005D
:10ED7C0010F8061F41452CD980F80080E88A86429D
:10ED8C0013D0A1891FFA8AF401223B462046FDF7D5
:10ED9C009BFEF0B904A806A90297CDE900103046F5
:10EDAC00214612E0E88A864207D1A1891FFA8AF02F
:10EDBC0001223B46FDF788FE0BE004A806A902974A
:10EDCC00CDE900101FFA8AF1304642464B4602F05C
:10EDDC0093FF08B0BDE8F087407B0020D1BC020057
:10EDEC00D9BC0200D07E00202DE9F84F0746087AE6
:10EDFC000C4640F00201032917D10025B7B1FF2FB3
:10EE0C0014D09A4616460AB903280ED00FF03AFAD7
:10EE1C00204611F021F88146207A4FF6FE71B0F1B0
:10EE2C00010B18BFB346894503D100252846BDE820
:10EE3C00F88F0138DDF82880314EB0FA80F04409A3
:10EE4C002E4801780020814230D03278BA4208D165
:10EE5C007278A24205D17288914502D132799345DC
:10EE6C0002D00E360130EEE706B32649C7B235465E
:10EE7C00B1F80090BAF1000FD8D0B8F8004028468D
:10EE8C00214619F0F5F960B92846214618F060FAC8
:10EE9C0030B1022039464A46334617F08BFA00E06F
:10EEAC00002508F10208AAF1010AE3E70DF10300BD
:10EEBC0017F0F4F805460028B8D0134885F804B0CC
:10EECC00A5F802906C702F7041460078504538BF01
:10EEDC0082464FEA4A0285F805A0A81D1AF052F99D
:10EEEC009DF80310064AC1EBC10002EB4003054834
:10EEFC000288022017F05EFA98E700BFE2BC02001D
:10EF0C0018870020C2B40200D3BC02002DE9F843DC
:10EF1C00804600683B4BD8E9012118603A480260F2
:10EF2C003A4820221AF0E6FED8F80C003849DFF8EF
:10EF3C00E89090E8FC00FCC1D8F80C00354990E84A
:10EF4C00FC00FCC1D8F81000494690E8FC00FCC15C
:10EF5C00324D402299F80C00D8F8141040F0800083
:10EF6C0089F80C0028461AF0C5FEE87BD8F8181072
:10EF7C00202240F0A500E873294D28461AF0BAFE6D
:10EF8C0040F20540697BAA7CEB7DC5F80490288291
:10EF9C0003202875287B40F08000287301F0F000D6
:10EFAC0020490230687302F0E0000A460130A87470
:10EFBC0003F0F0000130E875D8F81C0090E8F80078
:10EFCC00F8C2087BCB7B4A7B40F08000087303F0CF
:10EFDC0070008430C87302F0F000013048734FF4B5
:10EFEC0058600861D8F820000F4908600F48C068C5
:10EFFC004069007808B111F00FFBBDE8F84315F03B
:10F00C00D3BD00BF6488002068880020C083002026
:10F01C007885002090850020A8850020E87F0020BE
:10F02C00A083002030860020608800200C01002086
:10F03C002DE9F04387B0DFF8FC8081462025EFF303
:10F04C00118085F31188D8F830501DB180F31188E8
:10F05C0000256AE0C8F83090374F80F31188002003
:10F06C00C9F80C104FF48031C9F81C20C9E9120002
:10F07C00C9E90801002B18BF1F46D7E90116C9F8CA
:10F08C001810397B012905D1C9E91060C9F8146041
:10F09C0030460DE0294A002031460023002519F0A6
:10F0AC0011FFC9E910012649C9F814008E423CD859
:10F0BC000021DFF890E0C9E9160197F800C0C9F803
:10F0CC005410BCF1020F08BF0146C9F8501001AB37
:10F0DC009EE8F5001946BCF1000FF5C108F11C00C3
:10F0EC001A4ACDF808900090174808BF0246142120
:10F0FC0009F1280018F0F2F905462020EFF31181F0
:10F10C0080F3118881F3118899F8100010B94846E2
:10F11C0012F056FC35B108F12800494619F06CF98B
:10F12C004D4602E00025C8F83050284607B0BDE82F
:10F13C00F08300BFA01F002084B9020040420F00E2
:10F14C003F420F0060BA0200E9360200D192020081
:10F15C002DE9FC47434FDFF810810DF1070A4FF002
:10F16C00000918F0BFFB002800F0798050460121FF
:10F17C0014F016FD38780528F3D8DFE800F0030901
:10F18C000F1928469DF80700FE28EAD1032462E0F7
:10F19C00B8689DF80710022441705CE0B8689DF8CF
:10F1AC000710042481707878002808BF052452E0E9
:10F1BC009DF8070088F800907870033017F04EFF28
:10F1CC000028B86049D079780124017043E098F8A0
:10F1DC000000411C88F80010B96808449DF807101D
:10F1EC00C17018F07FFB054698F8000079780A1A70
:10F1FC00B9680844E9B203308A421ADA91B214F0C1
:10F20C00CFFC787888F800001FE07878BD689DF80E
:10F21C0007400330C6B22846314619F019FBA0420C
:10F22C0015D17B68B3B1304629460022002498479B
:10F23C0011E014F0B5FC98F800007978284488F8AF
:10F24C000000C0B288427FF48CAF052403E028464E
:10F25C0018F002FE00243C7083E700203870BDE8F3
:10F26C00FC8700BFF425002092880020F8B50446E6
:10F27C004048C16819B12046BDE8F84008473E4EE9
:10F28C003068074658B1054660882988814203D109
:10F29C002079A978814216D0A8692F46F2E71C2064
:10F2AC001AF0BCFC002863D01C21054619F006FEA0
:10F2BC00FF20E8724FF6FE7028813068002818BFD6
:10F2CC0007F1180635602079217A627A237BA870C1
:10F2DC0060880129AA7169712B75288005F10C00D1
:10F2EC0007BF4FF0FF31C0E9001104F10D011AF016
:10F2FC0040FC2249A07A0978884239D961790129E0
:10F30C0003D01AF029FA98B3A07AA97A884202D9C4
:10F31C00E27A102A05D3884206D1E97AE27A8A4247
:10F32C0002D20022012101E001220021144B1B78A2
:10F33C00022B01D2A31D01E005D1E31D1B7813B1F3
:10F34C0072B9228808E00F4A538B2288D31AB3FA79
:10F35C0083F35B09194203D0A872E07A2A81E87220
:10F36C00E07908B101202871A07908B10120E8707A
:10F37C00F8BD00BF3C830020E487002093270020C9
:10F38C0018260020407B00201EF0040F14BFEFF362
:10F39C00098169468869A1F1480214BF82F3098882
:10F3AC00954621ED100BF1EE102A41F8082DEFF3E4
:10F3BC00118102B400B5DFF8D8E0F047374A126883
:10F3CC00116801EA000010605DF804EB1EF0080FF4
:10F3DC0009D101BC80F311885DF8080BE1EE100A2D
:10F3EC00BDEC100B704704BC1EF0040F14BFEFF300
:10F3FC0009816946A1F1200114BF81F309888D466A
:10F40C004A604FF08070C86125488861234B1B68A7
:10F41C001868086040F201101860704702B401B41B
:10F42C00EFF3148100291CBF002282F3148802B46C
:10F43C0002B4DFF860E0F04701BC01BC00281CBF3F
:10F44C00022181F3148801BCDFF84CE0F0470F482F
:10F45C004FF08051016001BC80F3118800BF00BFE8
:10F46C00FFF7FEBF1EF0040F14BFEFF309816946CE
:10F47C0001F1200151F8080BE1EE100AB1EC100B70
:10F48C0014BF81F309888D46704700BF04ED00E07E
:10F49C00DDCB01008B9B0200919B0200B8BC0200EB
:10F4AC0028F400002DE9FE4FD0E90085994614465A
:10F4BC000F46834613B10020C9F8000074B11AF04E
:10F4CC0037F8064698F8070058B198F8E80070B17C
:10F4DC0030461AF0D9FA6FF008056DE06FF00905A7
:10F4EC006AE030461AF0D0FA6FF00E0564E00020A6
:10F4FC000121C8E93B74C8F8F440C8F8FC0088F84E
:10F50C00E810C8F83C0088F80D0088F80B00284675
:10F51C0001951AF0FDF830461AF0B6FA08F1D0064B
:10F52C000DF1080A1AF004F804463046514616F05C
:10F53C00F0FA0546D8F8F400D8F8FC10854288BFDC
:10F54C000546029839442A461AF0D4FB304629461F
:10F55C0014F022FCD8F8F400D8F8FC10401BC8F8C2
:10F56C00F4004819C8F8FC0020461AF08DFA012D59
:10F57C0003DBD8F8F4000028D4D119F0D9FF0446E5
:10F58C00D8F8FC0050B101981AF0C2F8584605F0B2
:10F59C003DFBD8F8FC0008B1002502E06FF00F0528
:10F5AC000020B9F1000F18BFC9F80000002088F83E
:10F5BC00E80020461AF068FA2846BDE8FE8F70472E
:10F5CC00F8B504460020A5782075C4E9030045F081
:10F5DC00020000F0030002280CD115F00C0005F01D
:10F5EC00030218BF042809D1022A05D1E90601D467
:10F5FC0002210FE0012619E0022106E00C2803D0BD
:10F60C000828F1D0012100E00321022A02D1EA06E8
:10F61C000E460BD448B10E1D0C2807D8012202FA55
:10F62C0000F041F21012104200D04E1D28060AD5EF
:10F63C00E078800706D0A8074FF0030058BF0220DF
:10F64C00064400E00136278819F0A8FF87420BD04A
:10F65C00A80609D51F48416920468847206918B972
:10F66C00A07800F0DF00A070207D00B1F8BD6179BA
:10F67C005020751C8DF8000020798DF8021021693E
:10F68C0028448DF8010029B10A7F497F10440844B1
:10F69C008DF80100684613F0C9FBA0B1012180F878
:10F6AC0048504176218841806188018721792269FF
:10F6BC0080F8421001692944416412B1127F11444F
:10F6CC004164E060F8BD20461AF0E1F81020207586
:10F6DC00F8BD00BF502400202DE9FF413B4E96F8A9
:10F6EC00420100286AD1012086F8420119F0D4FFAA
:10F6FC00374F86F87001374D7868C6F86C01387B47
:10F70C0086F84101A86810F4402F13D1386988B1EC
:10F71C0028686421C0F3066000FB01F41AF04EFA6D
:10F72C00B4FBF0F22C4906F19400002315F0E8FC30
:10F73C0019F038FD01AC20461AF0B3F82749A84659
:10F74C00002506F10C00002219F0FFFD20461AF0EE
:10F75C00A8F8234906F15000082219F0F6FD214AB9
:10F76C0006F1D8003221002313F034FC1E4C1F4A42
:10F77C0006F1F4002C2100232560454613F02AFCE9
:10F78C00D8F80800797BC0F3815021B1032804BF5D
:10F79C00012186F83911032803D040F00200022819
:10F7AC0010D1206840F040002060022015F0F8FDD8
:10F7BC006868400702D4002015F0F2FD002004B068
:10F7CC00BDE8F08114F094FAF2E700BFD81B0020DA
:10F7DC0090BA0200AC4F0050A79402000F7B0100BE
:10F7EC003D28020071CB01009022084035A5000095
:10F7FC002DE9F8431D46434BDDF8208043F6060601
:10F80C001C68038814F0007411D0B34227D0B3F5F0
:10F81C00C15F33D040F60206B3423ED100F1120371
:10F82C000B604169116081692960C1692EE0B342A6
:10F83C000AD0B3F5C15F03D040F60206B34203D140
:10F84C0000F11203143002E000F11A031C300B60BB
:10F85C000068106000202860C8F800004BE000F140
:10F86C001A034FF000090B60C1691160016A29602D
:10F87C00416AC8F8001000F118011CE000F11203F5
:10F88C000B6041691160416A2960816AC8F80010F7
:10F89C0000F1100190F80F900DE000F11A030B60CD
:10F8AC00C1691160816A2960C16AC8F8001000F151
:10F8BC00180190F82490286868B10E8819F068FD3A
:10F8CC00042808D8074606F0070148460EF018FF32
:10F8DC00296841F82700D8F8000060B119F058FDEC
:10F8EC00042808D805464846FF210EF009FFD8F831
:10F8FC00001041F82500002C18BF01242046BDE85B
:10F90C00F88300BF941200507CB50446007A02289C
:10F91C0003D3208814F028F910B1022630467CBDA0
:10F92C00207A032806D10DF10201204615F058FB70
:10F93C0018B9F2E72088ADF80200608A44301AF05A
:10F94C006DF9002864D04421054619F0B7FAA07A65
:10F95C00694617F071FE9DF800009DF8011085F8BE
:10F96C003A0085F839102846012117F0BBFE05F145
:10F97C0010002146242219F005FC628A616905F108
:10F98C0044002864AA8719F0FDFBBDF80200A8808A
:10F99C0020480178E971013101701AF011F906461D
:10F9AC001AF00CF970434FF47A710026B0FBF1F0A9
:10F9BC00FF218DF80460288095F8390001FA00F0D9
:10F9CC00217E85F8370085F83600207A8DF8060000
:10F9DC0001F001008DF8050001A819F0BFF9298D7F
:10F9EC00023885F83400C0B241F0080183B2298591
:10F9FC00A98F8AB2B2FBF3F202FB1010000418BFFD
:10FA0C0001322A720448012100780EF01BFB85E7B5
:10FA1C00102683E7948800203C2600202DE9F04135
:10FA2C008AB0DFF8E080D8F8000070B9364C206856
:10FA3C0028B936488068D0F84C0580472068344C8B
:10FA4C00016A204688473348E06133480068016901
:10FA5C0031B12E488068D0F8D40090F85300884714
:10FA6C002A4DA868D0F8D40090F9420010F086FB1B
:10FA7C00411C03D0294940EAE0704882274C002001
:10FA8C0060606080207B617B40F08000207301F01F
:10FA9C00F00001306073A868D0F8C403804730B917
:10FAAC001F4810210170E868142140680170D8F8D3
:10FABC000000C0B10020002714F02EFB124E30685D
:10FACC00416E02AD2846884731680597D8F800008A
:10FADC002A4600230E6D0821CDE900172146B047B8
:10FAEC00104804600AE010480C4A094B01680648AB
:10FAFC00006804680D48A047C8F800000AB0BDE8CB
:10FB0C00F08100BFD8260020308800200C01002096
:10FB1C00E083002054F100805C880020C08300202A
:10FB2C00B088002020250020648800204873002025
:10FB3C002DE9F04788B0DFF8FCA0D0F804803E4EE9
:10FB4C007F2400217F23DAF8280020EA0800CAF875
:10FB5C0028001B2915D020FA01F2D2070FD000275C
:10FB6C00324612682AB19578A94208BF013718327B
:10FB7C00F7E7DAB2FDB295423CBFCCB23B4601315D
:10FB8C00E7E7B8F1000F15D0CAF8288001AC1821AE
:10FB9C00201D19F093F90120CDF804808DF8080090
:10FBAC009AF82E008DF8090020460EF0D3FF08B00D
:10FBBC00BDE8F087204EDFF884804FF6FF793046A1
:10FBCC000768BFB13888BAF8241088420FD1B978C9
:10FBDC00A1420CD1B8F8001049451DD11AF004F817
:10FBEC00AAF82400398881423046E9D102E007F1B5
:10FBFC001800E5E78AF81840FEF7ACFE0028D6D0CE
:10FC0C0000208AF826000E4801680029CFD0C420B5
:10FC1C0008B0BDE8F047084700208AF826000848DD
:10FC2C00016809B1C4208847002008B0BDE8F0473E
:10FC3C0016F01EBA407B0020E487002080270020AD
:10FC4C00002500202DE9F04389B03F4A127882420A
:10FC5C0009D93C4A3D4F002952F8306018BF0F4675
:10FC6C0096F8521021B10025284609B0BDE8F08362
:10FC7C0002EBC009D9F804406078022826D1022092
:10FC8C0086F8520012F07EF80DF10C08404619F07F
:10FC9C0081FA3868002541468DF8145006958DF888
:10FCAC000C500490207812F0A3FD00287060DBD07B
:10FCBC0019F02CFFF87988B1B87939684843642178
:10FCCC00B0FBF1F1706819F01EFF07E000F0F2FCD8
:10FCDC00012086F85200207886F854006D4628469C
:10FCEC0019F0DFFD002000212A46CDF808908DF890
:10FCFC0000000190164813F031F9B06070B138680B
:10FD0C003060B97986F85310F87902280CD00128A4
:10FD1C0012D0A0B9484613F06AF810E070680028B9
:10FD2C00A1D019F0EDFE9EE7B8884FF6FF7241089E
:10FD3C0048460CF0EBFB02E0484613F0A5FE4D469E
:10FD4C0092E700BF24BB02008FBA02002CBC020059
:10FD5C00FD2A02002DE9F04F85B0044600880DF114
:10FD6C00060116F063FE0546182019F057FF4FF6F2
:10FD7C00FE7970B11821064619F0A0F86088182198
:10FD8C00324619F03DFD09F101006080304619F052
:10FD9C0043FF0020A4F80090002D20715DD1DFF806
:10FDAC00C0A0BDF80640DAF80000B8B3142019F072
:10FDBC0035FF98B3834604AB4C2000210222002768
:10FDCC0019F062F8009404EB440402AE0BEB44000F
:10FDDC004FEA4408851C122F17D0B84505D1DAF824
:10FDEC00000000EB440128460AE0B81C062233460A
:10FDFC0081B24C2019F048F80BEB07003146023069
:10FE0C00062219F0BFF90637E5E74C2014215A46B3
:10FE1C0019F0F6FC584619F0FFFE009C04AB4C2080
:10FE2C000021022219F030F8B8B9DAF8000050B10C
:10FE3C0004EB440130F81100484504D1BDF8100022
:10FE4C0030B1013802E0BDF810000130ADF81000FF
:10FE5C0004AA4C20022119F0D3FC05B0BDE8F08FA8
:10FE6C00E0260020F8B5067B07460D46304618F014
:10FE7C00FBFC18B104464089002726E07A893868D3
:10FE8C00314616F0FCFF0026002869D00446068196
:10FE9C0017F8100F207478886082384619F076F8BD
:10FEAC006061388961892083B87AA07621F460700A
:10FEBC004907608105D42B490978013140EAC1100A
:10FECC0001E040F0800001276081C0F3C21195B1C0
:10FEDC00022262732268D289520702D5224A128A00
:10FEEC00228169B36FF07F0220F4607002EBC111C4
:10FEFC000843608124E039B1810607D4C1060BD4D4
:10FF0C0040070FD4012013E000261AE019F01EFD63
:10FF1C0000F07F005F300BE019F018FD00F00F00CF
:10FF2C000A3005E01148058819F010FD2840023010
:10FF3C0020810F4804216173202100780EF082F893
:10FF4C0001266FB12289617B20460CF0C7F938B1CC
:10FF5C00606908B119F060FE204619F05DFE0026BC
:10FF6C003046F8BDC5270020407B0020BEBC0200F7
:10FF7C00988800202DE9F0418AB03E4E0546306845
:10FF8C0020B13D490978A94209D82DE013F094FE1F
:10FF9C003068002448B338490978A94225D94FF074
:10FFAC00FF3119F0E7FC354905EB450001EB800406
:10FFBC0067683878A8B9A568A9682A6848424B1EB2
:10FFCC001A42B8600DD16A688A420AD31040824244
:10FFDC0007D1686910B10068786029E0298B042981
:10FFEC0007D3306819F02CFE002420460AB0BDE877
:04FFFC00F08106EB9F
:020000021000EC
:1000000081000069A8B90DF10408404619F062FBAF
:10001000002041468DF810008DF80400E869059035
:10002000287E12F06BFC0028E1D0298B06EB8102C0
:100030001061786031440A7B01320A73298CC6E969
:100040000101204616F0ECFF01203870AB20318909
:100050008DF82700204618F04EFF0DF127000121F2
:100060000FF0B2FD31890546204618F04DFF15B955
:1000700020460EF0FFFD306819F0E8FDBBE700BF39
:100080000C240020F3BA0200A0B902002DE9F84FB9
:100090003C4C3D4E3D4D42F62A294FF0010A4FF0AF
:1000A000030B00274FF00508D4F83C01062833D88D
:1000B000DFE800F00433183B203D4B000F20F060D8
:1000C000C6F8109013F09AF845F804AC55F8040CF3
:1000D0008007FBD5C6F81CA094F8390190B1012027
:1000E000EF6210E02F60C4F83CB128688007FCD4B0
:1000F0000320DBE72F60C4F83C8128688007FCD42C
:100100000520D3E70320C6F800B0C4F83C012F60F7
:1001100029688907FCD4C9E7FEE70126022084F894
:100120003A6112F0ABFB2E6009E0022000E00320F0
:1001300084F83A01002012F0A1FB0120286004F1AC
:100140005000BDE8F84F19F049BD002045F8040CF7
:10015000286055F8040C8007FBD428688007FCD47D
:100160000B480025012105600A4801600D2005F0BB
:100170006DFB022014F0FCFAC4F83C5184F83B51AA
:10018000BDE8F88FD81B002000400C4058600C40A0
:100190003C500C4004800C402DE9FE4FDFF8F4B0D9
:1001A00001219BF80C4001AA204619F0C6F86A46C6
:1001B0002046022119F0C1F8DFF8DC909BF80EE030
:1001C0009BF80D00BDF800C099F800100EF1010376
:1001D0000746B3FBF1F404FB11359DF80240ADB2C4
:1001E000FEB2B5420FD0A642634618BF102372007C
:1001F00052FA87F20BEB82029383721CB2FBF1F38B
:1002000003FB1127ECE7DFF894A0002401270DF190
:10021000080857FA8EF2C9B2C5B2B2FBF1F303FB7C
:100220001121A94232D0690051FA80F00BEB800213
:1002300032F81C0F102806D1284607F0A1FA8AF8D8
:100240000000013417E028460421022313F01EFDAC
:100250008AF80000284600214246042318F060FF77
:100260009DF808007C2802D0FE2804D10DE0284625
:10027000782114F0FBF999F80010681C9BF80EE047
:10028000B0FBF1F202FB1100C3E7FEE7E0B2BDE80C
:10029000FE8F00BFA080002097880020A0230020B0
:1002A0002DE9FE4F05460F465818AE687168884222
:1002B00002D96FF0030564E0DFF8E8800C9C4FF092
:1002C000FF3199469246D8F8000019F059FBE00733
:1002D00011D1A0071ED5306851464A463844CAB1EC
:1002E00011F8013B10F8014B013A1C40A342F6D033
:1002F0006FF0060541E0D8E90101CB4301EA0902AC
:1003000013EA090F18BF02442846394009F0E8FEF5
:10031000054690BB306802970196074412F00EFC28
:10032000CB4655460090BBF1000F16D05E46BBF1A0
:10033000080F28BF082619F001F9804628463946DB
:10034000324617F071FD0446404619F0A3FB2CB964
:1003500037443544ABEB060BE5E70024009817F073
:10036000B1F8DFF84080DDE901210C9814B14FF0BD
:10037000FF3502E0400707D40025D8F8000019F047
:1003800065FC2846BDE8FE8F10680844B9F1000FEF
:10039000F2D010F8011B1AF8012BA9F101098A42C9
:1003A000F4D0E4E7DC250020B0B50C46880722D461
:1003B000600758BFB0BD354D0120A870042014F06F
:1003C000F5FF33480068006B8047E8602D48806B7C
:1003D000F0B16968046961B1A1420AD094F82800BB
:1003E000400704D5636A2046042100229847012073
:1003F00060766C600DE0FCF763FD2248006CE0B3B2
:10040000214844F002012830BDE8B04019F022BC78
:100410006C6860681F4900780860022014F0C6FF0D
:10042000102005F085FC012028761B48807810B943
:100430000D2005F07DFC6868416818488A680AB993
:10044000C96821B100218160154940F8141C154983
:1004500007220A6001680021016042684160124978
:10046000124AE9610168114301601A2019F0BCFBCE
:100470001920BDE8B04019F0B7BBBDE8B0400DF0A1
:10048000B5B800BF3021002070200020D01E002011
:100490008C010010D0210840ACBB020014100440B5
:1004A0005100070600000460ADEB00000240004070
:1004B0002DE9F84F3A48DFF8EC90DFF8ECB0DFF8C0
:1004C000EC8000264FF0060A00210078C700B742F2
:1004D00042D009EB0605A878E0B30138A870687926
:1004E00018F0C8F9A8B30446A87800B3A87948B3AF
:1004F000287970B3E9780139E970090629D19BF8A8
:10050000011001382871E970617B032921D10006AF
:100510001BD00420607319F01FFA00F00F00202197
:100520000130208198F800000DF092FD11E0607B11
:1005300084F80DA002280CD02068F021407B11F037
:1005400091F906E0607B032803D12846214610F08C
:1005500001FF01210836BAE798F8000001290BD104
:10056000402112F02DFEC0B998F80000402164220D
:10057000BDE8F84F19F0BBBA40210EF039FA0C482B
:100580000178012909D1002101700A48007806F09C
:10059000B1FCBDE8F84F12F06DBEBDE8F88F00BFAA
:1005A000D2BC020042760020407B002098880020C8
:1005B000DA270020DB27002070B58AB04FF4806175
:1005C000041D4588ADF826108189807B0894ADF81C
:1005D00024500328ADF81C1034D0022806D0B0BB3C
:1005E00040F601000026ADF826005AE032480078B7
:1005F00001285FD10DF11B0101AA204608F0DAFFA6
:1006000004469DF81B00012854D19DF814000228CF
:1006100050D101AD1421284618F056FC274904EBAF
:10062000440000222B4641F8202001EB80002146A7
:1006300042604272FF2014228DF81400042015F04D
:10064000BFFE37E0102000268DF8270029E00DF1CD
:100650001B0101AA204608F0ADFF01469DF81B00D2
:1006600001281DD19DF81400022819D1134A002336
:1006700001EB4100CDE9013342F8203002EB80006C
:1006800014224360FF208DF814009DF816000130FD
:1006900000F00F008DF8160001AB042015F090FE5D
:1006A000012607A801F050FE26B118B928462146B8
:1006B00002F044FA0AB070BDBB270020804300203E
:1006C0002DE9F047A4B018F039FF34490A78012A1F
:1006D00004D124B0BDE8F04719F0DCB94FF00109AE
:1006E00081F8009019F0D6F9FEF7FCFF082005F01C
:1006F0001FFB21AC204618F0BBFC4FF0FF30294A0D
:10070000102123462290264812F06AFC2648284DE4
:1007100000260DF1040A0478244890F8008047462A
:10072000A74212D8286850F8271021F0FF004AF895
:100730002700880707D4F8B201F0010118F088FCFF
:1007400009FA07F006430137EAE71A4806601A4833
:10075000C16801F44001B1F5800F09D10068000EB5
:1007600018BF01205AF8201041F007014AF8201064
:100770001248A4EB080204230AEB880103EB82026F
:1007800040EA880019F0BCFA0D482022016862F3A3
:100790000D21016024B0BDE8F08700BF962700203E
:1007A000608400203D1C02009FB6020045B6020096
:1007B00014BB0200D0200240A84F00500010084097
:1007C00000300940FEB5D0E9005401A818F030FC13
:1007D00095F834003649374A384E085C95F835109C
:1007E000515C354A084395F83610515C2A6B40EA53
:1007F0000103316820684F680299B847206840F2C9
:10080000F272E1692E4B2F4F426494F854209A5CA7
:1008100094F85530FB5C1A430129426311D101461B
:10082000D4E90A2351F8307FFF2A27F4004718BF84
:1008300007F50047FF2B0F6009D00A6842F4804299
:1008400008E0014651F8302F22F400420A600A689D
:1008500022F480420A60C16A41F01001C162016B5A
:1008600041F001010163E16B09B3A16BF9B1012111
:1008700018F090F8D5F85801E16B40680068C16243
:10088000C0F8041591FAA1F17268B1FA81F15368C8
:10089000022298477068A16B02224368D5F858017C
:1008A00091FAA1F1B1FA81F1406800689847FEBD64
:1008B000A8BC0200C8BC02009AB60200D001001019
:1008C00091BC02008CBC02002DE9F04186B018F00A
:1008D00079FF0446002718F075FF10B180690137D1
:1008E000FBE7DFF8CC8098F80000012831D818F039
:1008F00069FF304EB18C28B102888A4229D08069C4
:100900000028F8D11C2019F08FF910B30546B08CDF
:100910002880307EA87018F041FE6871264806F1E4
:1009200039010078A87105F10C0019F028F90DF1D2
:100930001701412015F076FB20489DF81710AC6197
:100940002C460088002908BF6FF00100013728817C
:1009500000E000251A48FBB200210278934201D240
:1009600000260BE0BE1A0020C7B2974202D2A4694B
:100970000130F9E7F0B2052828BF05261148F6B284
:10098000CDE902411049CDE900260022007803F0AC
:100990001DFD98F8000008B1012803D115B12846C3
:1009A00019F040F916F064FF06B0BDE8F08100BF11
:1009B00018260020407B0020D827002070870020C8
:1009C000C3880020C288002084870020F8B5044630
:1009D00018F036FB07464568204618F0CBF898B16A
:1009E000D7E9014618F0AAFD0546D4F8C000C8B101
:1009F00004210174384606F00DFCD4F8C800C0B1DB
:100A0000416949B10846FBE718F098FD0446D5F85E
:100A1000C000B0B310303BE0D4F8C010416101F128
:100A200014000BE03068416821F002014160284663
:100A300031E0D4F8C000C4F8C800143001680027C1
:100A40000760C4E93477C4E93677C4F8C01031B31D
:100A500020463146FBF7D0F8D4F8C000C4F8E07067
:100A60000068B0F5806F03D920463146FBF7C4F823
:100A700094F8FE0010BB3068416841F0020141600B
:100A80001CE095F8FB00002114F058FB05F1FC0078
:100A9000012101702046BDE8F84018F0FBBF94F832
:100AA000FB000021C4F8C47014F048FB012084F856
:100AB000FC003068416A21F003014162284618F0C9
:100AC000E9FF04F13000BDE8F84019F0C5B87047FF
:100AD00070B5C1680C6991F8381041F002032246E4
:100AE00003F0030302F8011B022B3BD111F00C03AE
:100AF00001F0030518BF042B2DD1022D01D1CE0624
:100B000030D4C26892F83B2062700234022D01D1C9
:100B1000CA0626D4C26892F83E202270C26892F8B3
:100B20003F206270C26892F84020A270C26892F8BA
:100B30004120E2704BB1221D0C2B13D8012505FA80
:100B400003F341F210152B420CD0C26892F83A2000
:100B50002271621D06E00C2B2ED0082BCDD014463E
:100B6000D4E72246C46801F0020394F8395005F036
:100B700003051D4309D1658D2D0606D4134E357826
:100B800084F849506C1C347001E094F8495009060F
:100B9000157010D5C16891F839105170C16891F87D
:100BA0003940A40707D091F84B1091701BB1C06871
:100BB00090F84C00D07070BDC26892F83C20627012
:100BC000C26892F83D20A27003349FE79488002009
:100BD0002DE9F8430546007F04282FD1A86A4678FE
:100BE000B0F802900E2E38D80C460127DFE806F048
:100BF00008080841414141414141412A2A38410008
:100C000031480078012833D83048807B80072FD5C1
:100C10001FFA89F80021404609F022F900283FD048
:100C2000817911F0180F3BD0AA894388698900881F
:100C30000027009200220FF0ECF81AE0D32006F013
:100C400068F829E020480078012811D81F48807BE7
:100C500080070DD519F008F80AE00127002408E004
:100C600019480078012803D81848807B80071DD4D4
:100C7000012768891FFA89F2314618F0C7FF688991
:100C800012F078FF40B1A87C022805D327B10F48A5
:100C9000A989C08A814200D100242046BDE8F8839A
:100CA00040460121012716F085F9E2E71FFA89F88D
:100CB000404617F0AFFF40460CF05AFEB0F1C507B2
:100CC00018BF0127D5E700BF18260020407B002071
:100CD0002DE9FE4F4FF4804018F00AFAA0B1354CD0
:100CE00035496068D1F8132009786FF39F5201F0FD
:100CF0000401806842EA417101AA03F047F8606884
:100D00008168012016F0A4FE2E482C4F2C4D44F291
:100D1000020B00244FF0000A00F14009BAF1020F63
:100D20003CD055F82A80D8F80000A0B3D8F80000CD
:100D3000806918F0DDF90646D8F800000023324635
:100D400015F002FE16F00A0F1ED0D8F800008069D8
:100D5000B9686BEA00000840B860D8F80000C069C4
:100D6000396821EA000038601020D8F8001016F029
:100D70006FFED8F80010484616F00AF9002044F03B
:100D80000204C8F8000006E02EB1D8F800000D49B2
:100D900044F4804408650AF1010ABFE724B10A4817
:100DA0002146283018F056FF06F0FCFEBDE8FE4F45
:100DB000F7F756BBD01E0020850300210C1004401D
:100DC00014BC020030210020702000202DE9FC47D7
:100DD0003A4D0446286810B194B1BDE8FC87122052
:100DE00018F022FF00282860F7D04FF6FE7200218D
:100DF000531C1229F0D04618425206317380F8E78E
:100E000001AB4C200021022218F044F800284CD1FC
:100E1000BDF80400002848D0032846D8182018F050
:100E200003FFDFF89C90044600264FF6FE784FF053
:100E3000020A0027032F34D028680622831907EB03
:100E400047000AEB400081B24C2018F023F828BB81
:100E50002868815B414518BF002C1FD03044002218
:100E6000182341880620009415F094FA2868D4E9E4
:100E70000423304402F2E9324188226101EB41004F
:100E800049F8202009EB8000182243600620234601
:100E900015F096FA2046182118F016F80636013794
:100EA000C8E714B1204618F0BDFE064B71200021A2
:100EB000082217F0EFFFBDE8FC8700BFE026002006
:100EC00018830020AC260020F8B53948394D01219F
:100ED000394E0768E868C0680170002002F002011E
:100EE000F07003F0E040401817D096F90600012892
:100EF00002DBB0790138B07196F90500012802DBF8
:100F00007079013870712D48426803F0807082B1A9
:100F1000D8B10020002190470CE01446D00323D420
:100F2000A0032ED4600230D5002038710BF06CF98C
:100F30002BE050B196F90700012802DBF079013867
:100F4000F0710120307117F069FF002038710BF04B
:100F50005BF97079F8B196F90500002823DCA868E0
:100F6000D0F84C0580471EE01548007820B10520D8
:100F700017F036FF13F082FD00203871F1F78CFE78
:100F800003E00020387111F0DFF8A00648BF18F028
:100F9000A7FE707938B900200021B070A868D0F899
:100FA000582400209047E8680021C0680170F8BD0F
:100FB000748800200C0100201425002024B80200B1
:100FC00090270020B0B58CB004464089ADF80000F1
:100FD00060684178821C019206298DF8021003D0C6
:100FE000042907D0012936D1817C13228DF8031002
:100FF0001B2101E01A211222851801440391029558
:1010000031D0284616F0F2FE01282CD117F0F8FD59
:101010000146284616F049FB28BB264800780128DF
:1010200024D8684618F03EFC01281FD102980DF123
:10103000160113F0DBFF012818D10021BDF81600BE
:1010400061721D496081097891B16168097805294B
:101050000ED101210DE00021029100F11201807EEC
:1010600003918DF81000684610F060FD0CB0B0BD23
:10107000002100222173CDE906220892ADF8180064
:10108000207A8DF81D108DF81C0001208DF81A00B3
:1010900006A8FEF79BFA9DF82C000028E6D10998D7
:1010A000227A6168406C18F073F806A811F026FAED
:1010B000DCE700BF18260020D02700202DE9F041F2
:1010C0000E46054610463421144617F0FDFE082E44
:1010D0004ED326702146288811F0FAFF8046688892
:1010E00008216081A888A081A879A074E87961703E
:1010F000E074E07920B1102105F1080061706061B1
:10110000207A28B101F1080029446070A16100E053
:1011100008460021616284F82010617919B1295CC8
:10112000013060706171617FF1B1421C6270295CB5
:101130000230607084F82010AA5C914284F821206B
:1011400010D9194A4F00194E1278914288BF1827BA
:101150003A462918304618F01BF860786662384421
:10116000607001E0002161772178C2B2914203D220
:1011700000263046BDE8F081B8FA88F2091A55FA1F
:1011800080F05609A2792177A062002AF1D00E30B2
:10119000A062A1F10E0020770548007B18F048F806
:1011A000217F081A2077E4E7DBBC0200F0850020ED
:1011B000407B00202DE9F04105460026806A1C4650
:1011C000174688461680007817F034FA40B16889CF
:1011D00012F0D0FC022811BF00266889388026460C
:1011E000A86A007801380A2846D8DFE800F0060C23
:1011F0001116242C45383C4A5200284641463A46AE
:10120000F7F7C6FD41E028464146FDF761FD3DE0A8
:1012100028463146FFF7DCFC37E0287F02282BD137
:1012200026B920486989C08A814228D1304629469A
:1012300000F034FF29E0688912F09CFCE0B92846F0
:10124000F4F758FF22E017486989C08A814213D118
:10125000287F022810D128460CF06AFE16E02846A6
:10126000FCF71AF812E00F486989C08A814203D15D
:1012700028460BF0BFF909E0D32005F04AFD00260F
:1012800004E0304629460FF021FF06463046BDE80F
:10129000F081054800780128F1D128460CF018FEAD
:1012A000F4E700BF407B0020BA2700202DE9F04181
:1012B000056804464FF0FF30E86218F03FF98046B9
:1012C00095F83000042809D13349497831B13349C0
:1012D00003228A604A6822F003024A602E4F6B693B
:1012E0002F4E00217A68B34204D01AB979780029C8
:1012F00018BF01210023042804D11AB17B78002BE8
:1013000018BF012341EA0300012808BF14F0AEFD15
:1013100095F8320030B1404618F0BCFB4FF0FF307A
:10132000BDE8F08195F83000042804D1381D294625
:1013300015F039FD03E0381D294615F029FE01207E
:1013400085F83200404618F0A5FB0020FDF720F894
:10135000246894F83000012812D0022813D0042801
:10136000DCD10E4DD4E90901884211D2012018F0D8
:101370003CFB28688007F9D00020FDF709F8F1E769
:101380000020BDE8F081216A04F1340018F0F8FA79
:10139000E06ABDE8F08100BF182300200880024009
:1013A00080A9030070B586B03449002808705DD16B
:1013B000344C207830B93249097819B9082016F030
:1013C00097FB207801284ED80020CDE90300CDE915
:1013D000010017F025FE002845D02B4D05F13904FA
:1013E000204617F043FD18B92849204618F0C7FBDE
:1013F00005F11601532010F041FEA87B0DF11701F5
:10140000C0F3C0008DF81700522010F037FE0820FE
:1014100085F8260003F026FA04F072FA1C480168E9
:1014200009B9012101601B484FF4407100780CF0AC
:101430000FFE01AC204614F0F1F8204600210026F2
:1014400015F0D8FE95F8410010B9002005F052FDC6
:101450001148CDE90366CDE90166807B012802D001
:10146000012014F00BFE012015F036FB0948022183
:1014700000780CF0EDFD06B070BD00BFBB88002009
:10148000C426002018260020407B00209E870020D4
:101490000825002099880020CC2200202DE9F84F53
:1014A0008A468DF8030062B13848514601234068EE
:1014B00002700DF1030048F231020DF0ADFF044659
:1014C00060E00B9F162405201E4617FB0400C0B2E7
:1014D00018F0AAFB002854D0814604220C980A99DF
:1014E00017FB04280024CB460BF8014F00F1190527
:1014F0008BF801600BF104068BF803708BF8021077
:10150000E0B2B84229D2A5F11701304618F037FBF6
:1015100006F10800A5F10F0118F031FB15F8071CC2
:10152000861D0134017015F8061C417015F8051C64
:10153000817015F8042C41EA8201817015F8032CA2
:1015400041EA0211817015F8021CC17015F8011CE6
:10155000017129781A354171D2E70C4D5FFA88F391
:101560000DF10300514648F23102C5F804B00DF008
:1015700053FF0446484618F055FB054801306860A3
:1015800000E010242046BDE8F88F00BF7C26002034
:10159000DC7D00202DE9F04742F22C0940F2100AD0
:1015A00042F20C0640F2B81715460C468046C4F2CB
:1015B0000909C4F2090AC4F20806C1F2000708F0DA
:1015C0004FFB44F20C00C4F2090000210160D9F87D
:1015D00000003868816927208847306B4FF6FF711B
:1015E000CFF6FE6108403063B06F20F48070B067C2
:1015F0003868016B4FF4806088473868016B4FF49E
:10160000816088473868016B4FF4C060884742F2B8
:101610002800C6F2080001210160C6F8804131604F
:10162000DAF80000800705D4681C08BF4FF0404579
:10163000CAF80C50D9F80000F0698007FCD500BF4B
:10164000072010F03FFB0228FAD1B8F1000F16D1A5
:1016500044F20004C4F20304386A816820468847D3
:101660000428F9D0012804D1386A032142682046B1
:101670009047D6F8180220F00300C6F81802386820
:10168000806BBDE8F04700472DE9F04385B0064682
:1016900000200D46049017F051FF334CDFF8C49042
:1016A00080462168D9F80000CB6C04AA0521984730
:1016B00001A817F0ABFE2D48019626F00106039510
:1016C00020F00107BE420AD12B490878FE281BD022
:1016D0002068826BD9F8000091F900100EE02448D0
:1016E00020F0010086421BD123494878FE280BD008
:1016F0002068826BD9F8000091F901109047812889
:1017000002D01C4818F08DF92168D9F80000002299
:10171000CB6A01A998470546B0F1FF3F07DC03E01B
:10172000144818F07EF9FE25124818F07AF9BE42E6
:1017300001D1114806E00E4820F00100864202D196
:101740000D4801300570012021680490D9F800008F
:10175000CB6C04AA05219847404618F09BF905B0C8
:10176000BDE8F083D826002030880020B161020057
:101770004D4B02000C010020142500202DE9FC47F0
:1017800006680446707A00286BD0D4F80490D6F826
:101790005801D0F80480D9F8347020460BF090FB43
:1017A000706F20B306F14C05284618F04BFA316FE4
:1017B000884221D2307902281ED0B06E002850D045
:1017C00020460BF07DFB346F284618F03BFA201AB8
:1017D000D6F868A0B46F7067284618F033FA002175
:1017E000F1740AEB040108440190706F0CE0B06ED4
:1017F00010B1306F0028D5D106F14C0001A914F0CA
:101800008EF901217067F17458B30021B173B0F5FE
:10181000806F84BF4FF48060706701990123014499
:10182000013979601049B96043F6F07101EB00109D
:101830000840B9680843B860D9F83C10D9F80000EE
:1018400091FAA1F2B2FA82F203FA02F2D8F8003069
:101850009A61D6F85821526812689162012117F0F6
:10186000A5F8BDE8FC8700BF0180000C7CB53A4DAF
:101870000446A868D0F8B810097859B194F89820AF
:1018800004F190014AB1152217F0D8F958BF25226A
:101890009A5C09E00121217514E0252217F0CEF9A8
:1018A00058BF25229A5C023284F86A20002284F80C
:1018B0006920042284F86B2004F1700248C948C2F0
:1018C00009881180214611F82C2FB1F872300F2AA7
:1018D00021F8163CB1F8743021F8113C0BD0D0F847
:1018E0000463B4F8A8000023B0FA80F0420920464F
:1018F000B04700B17CBD214611F83C0FFF2801D153
:10190000A06D30B1A868D0F8FC222046904700288E
:10191000F0D1A868B4F89A3094F89C1004F19002C1
:10192000D0F87463002000902046B0470028E1D131
:10193000A8682189D0F80021D289914205D9E520F3
:101940006070A86800F51B7001E000F51E7001686A
:101950002046884700207CBD0C0100202DE9F0477F
:1019600088B004466FF00100A081002004F1040853
:101970008DF8100004AD4146281D17F0D0FC284614
:1019800009F072FE012809D1BDF81C00BDF8121043
:10199000A0816088814222D004AD01E060880025EA
:1019A000EA46ADF8020000264FF6FE7950468DF863
:1019B000006007F0CFFA012808BF56460746B5B1C8
:1019C000A88901210125A081204610F0D1F8012F1E
:1019D00006D1ADF802903046022110F0C9F8012579
:1019E000204611F0A3FA284608B0BDE8F087012F81
:1019F00013D1BDF80C00A0810AF1040016F0F6F92D
:101A0000012817D1204609F047F905463046022142
:101A1000ADF8029010F0ACF8E2E76088484504D1D8
:101A2000404616F0E3F901280CD1204609F034F9BC
:101A30000546D5E7404616F0D9F90128CFD1204612
:101A40000321CAE70025CBE72DE9F0438FB080469C
:101A5000374800240394CDE90144077814F05AFE76
:101A60004FFA80F901ADBC4212D2E6B207200C2237
:101A70002B4631460EF07AF940B9B9F1FF3F05DC4B
:101A8000072031460C222B4614F09AFC0134EAE779
:101A90004FF0FF300C22CDE90200781E01AB85B279
:101AA000072029460EF062F940B9B9F1FF3F05DC85
:101AB00001AB072029460C2214F082FC04AD18214A
:101AC000284617F001FA822018212A4617F098FEBE
:101AD000B8F1010F08BF002804D104AA8220182100
:101AE00017F094FE0AAD1121284617F0EDF93A20BF
:101AF00011212A4617F084FEB8F1010F08BF002813
:101B000004D10AAA3A20112117F080FE0AAA3B202C
:101B1000112117F075FEB8F1010F08BF002804D19C
:101B20000AAA3B20112117F071FE0FB0BDE8F08327
:101B3000D7BC0200B0B517F00FFF2C4C02210025D6
:101B4000207040F60F70A17430492581C4E9075513
:101B50002576A0850F202071012084F86C00E072AA
:101B600040F20510A08122480078E07121480078F9
:101B7000607021480078A07020488078A0732048C9
:101B8000007820826FF00100A0846083E0821D480D
:101B90000078E0741C480078207504F1390017F0D3
:101BA000EEFF40F20F5004F16E030021022284F890
:101BB000415084F86850A4F866001548007884F80D
:101BC0006A001448007884F869001348007884F8A3
:101BD0006B00892017F05EF908B1A4F86E50002060
:101BE00010F04EF8A4F87050B0BD00BF407B00204C
:101BF000B7270020CF270020C427002026870020F9
